:100000000C94CB170C94FC170C94FC170C94FC1755
:100010000C94FC170C94FC170C94FC170C94FC1714
:100020000C94FC170C94FC170C94FC170C94FC1704
:100030000C94FC170C940A580C94FC170C94FC17A5
:100040000C94FC170C9494CD0C94FC170C94FC1796
:100050000C94FC170C94FC170C94C0590C9420A41D
:100060000C94FC170C94EA3E0C94FC170C94FC17AF
:100070000C94FC170C94FC170C94FC170C94FC17B4
:100080000C94FC170C94FC170C94FC170C94FC17A4
:100090000C94FC170C94FC170C94FC170C94FC1794
:1000A0000C94FC170C94FC170C94FC170C94FC1784
:1000B0000C94FC170C94FC170C94FC170C94FC1774
:1000C0000C94FC170C94FC170C94FC170C94FC1764
:1000D0000C94FC170C94FC170C94194C0C94DA4BF0
:1000E0000C94FC179C2FB92FEA2F07301C30453099
:1000F000B2301831C1315A366836613688368C369E
:10010000EB36833B00374C3773379A37C337193890
:100110002A383E384F3860387138833B8E3A833BFB
:10012000993A093B0F3B2F3B1D3F233F343F3F3F55
:10013000473F5C3F4B3F5C3F4F3F533F5C3F593F26
:100140004FB452B441B445B44BB489B456B45AB464
:1001500060B464B468B46EB472B476B489B47CB478
:1001600080B484B484B989B98EB998B9A2B91BBADC
:10017000ACB9B4B9BCB9C6B9D0B9DAB9E9B9F3B94F
:100180001BBAFDB907BA11BA084AD73B3BCE016E7C
:1001900084BCBFFDC12F3D6C74319ABD56833DDADE
:1001A0003D00C77F11BED9E4BB4C3E916BAAAABEED
:1001B000000000803F05A84CCDB2D44EB93836A916
:1001C000020C50B9918688083CA6AAAA2ABE000053
:1001D00000803F004E414E494E495459494E46CD4C
:1001E000CCCC3D0AD7233C17B7D13877CC2B3295EE
:1001F00095E6241FB14F0A000020410000C84200CC
:10020000401C4620BCBE4CCA1B0E5AAEC59D744352
:100210004F4D4D554E49434154494F4E004452595C
:1002200052554E004552524F525300494E464F00D0
:100230004543484F0047322F4733206261642070A6
:100240006172616D65746572730A00206F662000CB
:100250004D424C2047323920706F696E742000295E
:100260000A0059206F7574206F662072616E676591
:100270002028312D00290A0058206F7574206F66E0
:100280002072616E67652028312D004D65736820EE
:1002900070726F62696E6720646F6E652E0A00531C
:1002A00074617274206D6573682070726F62696E1C
:1002B0006720776974682022473239205331222021
:1002C00066697273742E0A004732380A4732392041
:1002D00053320053746174653A20004D6573682091
:1002E000626564206C6576656C696E672068617311
:1002F000206E6F20646174612E0A0053206F757444
:10030000206F662072616E67652028302D35292E9A
:100310000A004D65736820706F696E742063616EAA
:100320006E6F74206265207265736F6C7665640A07
:1003300000456E642066696C65206C6973740A0000
:10034000426567696E2066696C65206C6973740A22
:10035000004D31323500286E6F2066696C652900CA
:100360005344207072696E74696E67206279746597
:1003700020004E6F74205344207072696E74696E51
:10038000670A0043757272656E742066696C653A1F
:10039000200046696C652064656C657465643A008C
:1003A00044656C6574696F6E206661696C65642C68
:1003B0002046696C653A20005072696E7420746939
:1003C0006D653A20006F6E2E0A006F66662E0A0079
:1003D000473236204465627567200030022B0224C4
:1003E000021D020F026F66660044454255473A00FF
:1003F0004D3131332053006F6B002C20002C200036
:10040000544845524D414C5F50524F544543544916
:100410004F4E004155544F5245504F52545F534434
:100420005F53544154555300454D455247454E4343
:10043000595F50415253455200434153455F4C4927
:100440004748545F4252494748544E45535300541D
:100450004F47474C455F4C494748545300534F461C
:1004600054574152455F504F574552004255494CF1
:10047000445F50455243454E54004C4556454C4907
:100480004E475F44415441005A5F50524F4245002D
:100490004155544F4C4556454C005052494E545FBF
:1004A0004A4F420050524F47524553530041555412
:1004B0004F5245504F52545F54454D5000564F4C8B
:1004C000554D455452494300454550524F4D0053F8
:1004D000455249414C5F584F4E5F584F4646004683
:1004E00049524D574152455F4E414D453A4D61721B
:1004F0006C696E20312E312E392847697468756217
:100500002C20646176696472616D69726F29205371
:100510004F555243455F434F44455F55524C3A68EF
:10052000747470733A2F2F6769746875622E636FE5
:100530006D2F646176696472616D69726F2F4D61B0
:10054000726C696E2D4149334D2050524F544F43C8
:100550004F4C5F56455253494F4E3A312E30204D45
:10056000414348494E455F545950453A416E79637D
:1005700075626963206933204D6567612045585471
:1005800052554445525F434F554E543A31205555CC
:1005900049443A63656465326132662D34316132B3
:1005A0002D343734382D396231322D633535633689
:1005B00032663336376666204D41524C494E2D41E6
:1005C00049334D5F56455253494F4E3A76312E349A
:1005D0002E320A002F2F20002054002052004163A9
:1005E00063656C65726174696F6E3A2050005741A3
:1005F000524E494E4721204C6F77205A204A65724F
:100600006B206D6179206C65616420746F20756E5C
:1006100077616E746564207061757365732E0A006E
:10062000546F6F206661722066726F6D207265660E
:100630006572656E636520706F696E740A0020468E
:100640006C6F773A20000001363726032BFFFFFF3F
:100650003C3D382AFFFFFFFF2E303E12FFFFFFFF19
:10066000FFFFFF0809FF2C071A1C18FFFFFF0844B3
:100670000A2C4324221E20643A0020693A0020708C
:100680003A00496E76616C696420657874727564AD
:1006900065720A0043290A0061626C656420286D56
:1006A000696E2074656D702000436F6C64206578FE
:1006B00074727564657320617265200020643A006D
:1006C00020693A0020703A004E6F20636173652004
:1006D0006C696768740A00454550524F4D204F4B76
:1006E0000A00205A004475616C20456E6473746F73
:1006F000702041646A7573746D656E7420286D6D29
:10070000293A20003F4B2076616C7565206F757427
:10071000206F662072616E67652028302D31302988
:100720002E0A00416476616E6365204B3D00416393
:10073000746976652045787472756465723A200034
:10074000496E76616C69642065787472756465724F
:100750000A0043616E6E6F7420656E74657220735B
:1007600075626469723A20004D363030005370650E
:100770006369616C204D656E753A2046696C616DE8
:10078000656E744368616E676520526573756D654B
:100790000A005370656369616C204D656E753A207F
:1007A00046696C616D656E744368616E6765205063
:1007B000617573650A004739310A4731205A2D3077
:1007C0002E310A473930005370656369616C204DE2
:1007D000656E753A205A20446F776E20302E310AAC
:1007E000004739310A4731205A2D302E30320A471E
:1007F0003930005370656369616C204D656E753AE0
:10080000205A20446F776E20302E30320A0047394C
:10081000310A4731205A2B302E30320A4739300006
:100820005370656369616C204D656E753A205A207E
:10083000557020302E30320A004739310A473120B6
:100840005A2B302E310A4739300053706563696185
:100850006C204D656E753A205A20557020302E312F
:100860000A00473239205332005370656369616C66
:10087000204D656E753A204E657874204D6573681D
:1008800020506F696E740A0047323920533100538B
:1008900070656369616C204D656E753A20537461B3
:1008A0007274204D657368204C6576656C696E675F
:1008B0000A004D313430205336300053706563697F
:1008C000616C204D656E753A205072656865617483
:1008D000204265640A004D3530320053706563690B
:1008E000616C204D656E753A204C6F6164204657EF
:1008F0002044656661756C74730A004D35303000B4
:100900005370656369616C204D656E753A20536163
:10091000766520454550524F4D0A004D3330332007
:10092000452D312053363020433620553100537049
:10093000656369616C204D656E753A204175746F11
:100940002054756E6520486F746265642050696438
:100950000A004D31303620533230340A4D333033B3
:10096000204530205332313020433620553100535A
:1009700070656369616C204D656E753A20417574D0
:100980006F2054756E6520486F74656E6420504901
:10099000440A003C5370656369616C5F4D656E7518
:1009A0003E003C5370656369616C5F4D656E753EDA
:1009B000002F002F002F002F2E2E0A002F2E2E008A
:1009C0002F2E2E003C5370656369616C5F4D656E20
:1009D000753E0A003C5370656369616C204D656E1D
:1009E000753E003C5370656369616C204D656E75A2
:1009F0003E003C46696C616D656E744368616E676C
:100A00006520526573756D653E003C46696C616D8D
:100A1000656E744368616E676520526573756D65B8
:100A20003E003C46696C616D656E744368616E673B
:100A3000652050617573653E003C46696C616D656B
:100A40006E744368616E67652050617573653E0022
:100A50003C4C6F61642046572044656661756C7438
:100A6000733E003C4C6F61642046572044656661CC
:100A7000756C74733E003C4175746F2054756E65DF
:100A800020486F74626564205049443E003C4175C3
:100A9000746F2054756E6520486F746265642050D1
:100AA00049443E003C4175746F2054756E65204882
:100AB0006F74656E64205049443E003C4175746F0C
:100AC0002054756E6520486F74656E6420504944EB
:100AD0003E003C457869743E003C457869743E00B0
:100AE0003C5361766520454550524F4D3E003C5386
:100AF00061766520454550524F4D3E003C4E65782D
:100B000074204D65736820506F696E743E003C4ED2
:100B1000657874204D65736820506F696E743E006F
:100B20003C5374617274204D657368204C65766522
:100B30006C696E673E003C5374617274204D65733E
:100B400068204C6576656C696E673E003C50726546
:100B500068656174206265643E003C50726568653A
:100B60006174206265643E003C5A20446F776E20B9
:100B7000302E313E003C5A20446F776E20302E31AB
:100B80003E003C5A20446F776E20302E30323E00BB
:100B90003C5A20446F776E20302E30323E003C5A53
:100BA00020557020302E30323E003C5A20557020A7
:100BB000302E30323E003C5A20557020302E313ECF
:100BC000003C5A20557020302E313E0056313136CF
:100BD000004A333320004D3530300A4D3432302056
:100BE00053310A4731205A313020463234300A47D7
:100BF00031205830205930204636303030004A32CB
:100C000032004A3232004731205A352046323430E1
:100C10000A47312058313930205932302046363099
:100C200030300A4731205A302046323430004731C4
:100C3000205A3520463234300A4731205831393075
:100C400020593139302046363030300A4731205A69
:100C5000302046323430004731205A352046323475
:100C6000300A473120583139302059323020463649
:100C70003030300A4731205A302046323430004775
:100C800039310A4731205A313020463234300A4750
:100C900039300A4732380A4732390A473120583248
:100CA00030205932302046363030300A4731205A11
:100CB000302046323430004A3032004A3132004768
:100CC00031205A3130004F4B004731205A3130002B
:100CD00047393000473120452569463530300047D7
:100CE0003120452D302E31462569004731204530D1
:100CF0002E31462569004731205A2569462569006D
:100D00004731205A2D302E31462569004731205A6F
:100D1000302E31462569004731205925694625691D
:100D200000473120592D302E3146256900473120AA
:100D300059302E314625690047312058256946250E
:100D40006900473120582D302E3146256900473142
:100D50002058302E31462569004739310047323856
:100D600000473238205A004732382059004732387D
:100D70002058004132305620004731205A3130008F
:100D80004A3034004A3231004A3230004B494C4C30
:100D900045442E20004A303400454E4400464E2043
:100DA000004A3032003939393A393939004D004872
:100DB000004137562000413656202D2D2D004A3057
:100DC000320041365620005A3A2000593A20005845
:100DD0003A20004135560041345620004133562018
:100DE000004132562000413156200041305620004B
:100DF0004D3834004A3136004A3138004D333030F6
:100E0000205332303933205033303030004D3330BE
:100E100030205331353637205031303030004739AB
:100E20003000473120452D332046313830300047DF
:100E3000393100473930004731205A3130204632AD
:100E4000343000473120452D3220463138303000D3
:100E5000473931004A3134004A3030004A303100DD
:100E60004A313000696E206D6F76655F746F282996
:100E700020666565645F76616C756520666F7220BB
:100E800058593A002C2065793D0029202D3E202814
:100E900065783D002C2073793D0020436F6E6E65B0
:100EA0006374696E67207769746820766572746907
:100EB00063616C206C696E65202873783D002C207E
:100EC00065793D0029202D3E202865783D002C20A5
:100ED00073793D0020436F6E6E656374696E6720A1
:100EE0007769746820686F72697A6F6E74616C20BC
:100EF0006C696E65202873783D003F5370656369A7
:100F00006669656420582C5920636F6F7264696E3E
:100F1000617465206F7574206F6620626F756E64F2
:100F2000732E0A003F28522965706561742076612E
:100F30006C7565206E6F7420706C61757369626C7E
:100F4000653B206D757374206265206174206C654B
:100F500061737420312E0A003F2852296570656143
:100F600074206D75737420626520737065636966A3
:100F7000696564207768656E206E6F74207573698B
:100F80006E6720616E204C43442E0A003F5370650B
:100F9000636966696564206E6F7A7A6C6520746532
:100FA0006D7065726174757265206E6F7420706CFF
:100FB00061757369626C652E0A003F5370656369E1
:100FC000666965642066696C616D656E742073691D
:100FD0007A65206E6F7420706C61757369626C65E0
:100FE0002E0A003F537065636966696564207072FC
:100FF000696D65206C656E677468206E6F74207013
:101000006C61757369626C652E0A003F5072696D80
:1010100065206C656E677468206D757374206265F9
:1010200020737065636966696564207768656E2002
:101030006E6F74207573696E6720616E204C434437
:101040002E0A003F537065636966696564206E6FA0
:101050007A7A6C652073697A65206E6F7420706C83
:1010600061757369626C652E0A003F537065636930
:10107000666965642052657472616374696F6E207D
:101080004D756C7469706C696572206E6F74207038
:101090006C61757369626C652E0A003F52657472EB
:1010A000616374696F6E204D756C7469706C6965ED
:1010B00072206D7573742062652073706563696654
:1010C0006965642E0A003F537065636966696564EB
:1010D000206C6179657220686569676874206E6F3D
:1010E0007420706C61757369626C652E0A003F53E1
:1010F0007065636966696564206265642074656D06
:101100007065726174757265206E6F7420706C61A9
:10111000757369626C65202834302D313430432971
:101120002E0A0047323620636F6D6D616E64207346
:101130007461727465642E2057616974696E6720EA
:10114000666F72206865617465722873292E0A00C3
:1011500024F4D43050C38E20C2A24017828B701169
:10116000127A910D816CD90AA861E108C758660707
:10117000615143061E4B5D05C145A7041A41110488
:10118000093D9803713931034036DB026533910222
:10119000D4305402802E1D02632CEE01752AC50145
:1011A000B028A001102781018F2564012B244B0159
:1011B000E0223401AC211F018D200D01801FFC00B5
:1011C000841EED00971DDF00B81CD200E61BC60090
:1011D000201BBC00641AB200B219A8000A19A000B2
:1011E0006A189900D117910040178B00B51684003A
:1011F00031167E00B31579003A157300C7146F00DD
:1012000058146A00EE1366008813630025135E000D
:10121000C7125B006C12570015125400C111510027
:1012200070114F0021114B00D61049008D1047005E
:101230004610440002104200C00F4000800F3E00E4
:10124000420F3C00060F3B00CB0E3800930E3700D8
:101250005C0E3500270E3400F30D3200C10D310055
:10126000900D3000600D2E00320D2D00050D2C006C
:10127000D90C2B00AE0C2900850C29005C0C270032
:10128000350C27000E0C2600E80B2400C40B2400AC
:10129000A00B23007D0B23005A0B2100390B2100EA
:1012A000180B2000F80A1F00D90A1E00BB0A1E00F6
:1012B0009D0A1D00800A1D00630A1C00470A1B00CE
:1012C0002C0A1B00110A1A00F7091A00DD0919007F
:1012D000C4091900AB091900920917007B0918000D
:1012E000630917004C09160036091600200916007C
:1012F0000A091500F5081500E0081400CC081400D0
:10130000B8081400A4081400900813007D08120007
:101310006B08130058081200460812003408110028
:10132000230811001208110001081100F007100035
:10133000E0071000D0071000C0071000B0070F0032
:10134000A107100091070E0083070F0074070F001C
:1013500065070E0057070E0049070E003B070D00FA
:101360002E070E0020070D0013070D0006070D00C5
:10137000F9060C00ED060D00E0060C00D4060C008A
:10138000C8060C00BC060C00B0060C00A4060B003E
:1013900099060C008D060B0082060B0077060B00E9
:1013A0006C060B0061060A0057060B004C060A008B
:1013B00042060A0038060A002E060A0024060A0021
:1013C0001A060A001006090007060A00FD050900B2
:1013D000F4050900EB050900E2050900D90509003B
:1013E000D0050900C7050900BE050900B5050800BC
:1013F000AD050800A50509009C0508009405080036
:101400008C050800840508007C05080074050800A8
:101410006C050700650508005D0507005605080016
:101420004E0507004705070040050800380507007E
:10143000310507002A050700230507001C050600E3
:10144000160507000F05070008050600020507003E
:10145000FB040600F5040700EE040600E80406009D
:10146000E2040700DB040600D5040600CF040600F2
:10147000C9040600C3040600BD040600B704060044
:10148000B1040500AC040600A6040600A004050093
:101490009B04060095040500900406008A040500DC
:1014A00085040500800406007A0405007504050023
:1014B000700405006B040500660405006104050066
:1014C0005C04050057040500520405004D040500A6
:1014D00048040500430405003E0404003A040500E6
:1014E00035040500300404002C0405002704040022
:1014F000230405001E0404001A0404001604050059
:10150000110404000D04040009040500040404008F
:1015100000040400FC030400F8030400F4030400C6
:10152000F0030400EC030400E8030400E4030400F7
:10153000E0030400DC030400D8030400D403040027
:10154000D0030400CC030400C8030300C503030058
:1015500024F404D9201BC40C5C0E9804C4095F0257
:1015600065077101F405F900FB04B3004804870026
:10157000C10369005803550003034500BE023A0049
:101580008402310053022A002902250004022000AF
:10159000E4011C00C8011900AF01170098011400F4
:1015A00084011300710110006101100051010E004F
:1015B00043010D0036010B002B010B0020010B0035
:1015C000150109000C01090003010800FB000800D7
:1015D000F3000800EB000700E4000600DE00060050
:1015E000D8000600D2000600CC000500C7000500A8
:1015F000C2000500BD000400B9000400B5000400ED
:10160000B1000400AD000400A9000400A50003001F
:10161000A20003009F0004009B0003009800030049
:101620009500020093000300900003008D0002006B
:101630008B00030088000200860002008400030083
:10164000810002007F0002007D0002007B0002009A
:1016500079000200770001007600020074000200A9
:1016600072000100710002006F0002006D000100B5
:101670006C0002006A0001006900020067000100BE
:1016800066000100650001006400020062000100C4
:1016900061000100600001005F0002005D000100C8
:1016A0005C0001005B0001005A00010059000100CC
:1016B00058000100570001005600010055000100CC
:1016C00054000100530000005300010052000100CB
:1016D00051000100500001004F0001004E000000C9
:1016E0004E0001004D0001004C0001004B000000C5
:1016F0004B0001004A0001004900010048000000C1
:1017000048000100470001004600000046000100BB
:1017100045000000450001004400010043000000B6
:1017200043000100420000004200010041000000AF
:1017300041000100400001003F0000003F000100A7
:101740003E0000003E0001003D0000003D000100A1
:101750003C0000003C0000003C0001003B00000099
:101760003B0001003A0000003A000100390000008F
:101770003900010038000000380000003800010086
:10178000370000003700010036000000360000007E
:101790003600010035000000350000003500010072
:1017A0003400000034000000340001003300000069
:1017B000330000003300010032000000320000005E
:1017C0003200010031000000310000003100010052
:1017D0003000000030000000300001002F00000049
:1017E0002F0000002F0000002F0001002E0000003D
:1017F0002E0000002E0001002D0000002D00000032
:101800002D0000002D0001002C0000002C00000025
:101810002C0000002C0001002B0000002B00000019
:101820002B0000002B0001002A0000002A0000000D
:101830002A0000002A000100290000002900000001
:1018400029000000290000002900010028000000F4
:1018500028000000280000002800000028000100E7
:1018600027000000270000002700000027000000DC
:1018700027000100260000002600000026000000CE
:1018800026000000260001002500000025000000C1
:1018900025000000250000002500000025000100B3
:1018A00024000000240000002400000024000000A8
:1018B000240001002300000023000000230000009A
:1018C000230000002300000023000000230001008B
:1018D0002200000022000000220000002200000080
:1018E0002200000022000100210000002100000071
:1018F0002100000021000000210000002100000064
:101900002100010020000000200000002000000055
:101910002000000020000000200000002000000047
:10192000200001001F0000001F0000001F00000039
:101930001F0000001F0000001F0000001F0001002A
:101940001E0000001E0000001E0000001E0000001F
:10195000232C0000B8220000561800003A0F0000A7
:10196000B8080000B1040000710200003E01000050
:101970001000C90210012C01400122017001180160
:10198000B0010E01F00104015002FA00B002F000B3
:101990003003E600D003DC009004D2007005C800DC
:1019A000A006BE000008B400B009AA00D00BA00039
:1019B000600E960060118C000015820020197800DE
:1019C000C01D6E00A0226400B0275A00902C500069
:1019D00000314600E0343C0010383200903A2800D4
:1019E000603C1E00A03D1400803E0A00203F000025
:1019F0002CFFFFFFFFFF0001010101016265640A86
:101A0000002C2073797374656D2073746F7070652A
:101A10006421204865617465725F49443A20004240
:101A200065642068656174696E67206661696C65CC
:101A3000640048656174696E67206661696C6564FD
:101A40000045312048656174696E67206661696C84
:101A500065640048656174696E67206661696C65DC
:101A600064004B494C4C45442E200070012C0190E1
:101A7000012701B0012201C0011D01F00118011070
:101A800002130130020E016002090190020401C03C
:101A900002FF000003FA004003F5008003F000D0CD
:101AA00003EB002004E6007004E100E004DC0040E9
:101AB00005D700C005D2004006CD00D006C8008082
:101AC00007C3003008BE00F008B900C009B400B078
:101AD0000AAF00B00BAA00D00CA500000EA0005069
:101AE0000F9B00C01096005012910000148C00C093
:101AF000158700B0178200B0197D00D01B78000058
:101B00001E730040206E0090226900F024640040A3
:101B1000275F0090295A00E02B5500102E5000201E
:101B2000304B0010324600E033410090353C00104D
:101B300037370070383200A0392D00B03A2800A0A5
:101B40003B2300603C1E00103D1900903D14001026
:101B50003E0F00703E0A00C03E0500003F000040FE
:101B60003FFBFF803FF6FFC03FF1FF453120544867
:101B700045524D414C2052554E4157415900424526
:101B80004420544845524D414C2052554E415741F6
:101B90005900546865726D616C2052756E61776191
:101BA00079004531204572723A204D415854454DD7
:101BB00050004572723A204D415854454D502042D4
:101BC0004544004D415854454D5020747269676733
:101BD00065726564004531204572723A204D494E68
:101BE00054454D50004572723A204D494E54454D72
:101BF0005020424544004D494E54454D502074728A
:101C000069676765726564004D3834205820592033
:101C10005A204500202F002042403A0020403A0040
:101C2000023A004361703A00205A002059005800DF
:101C300020204D61783A2000205A00205900580099
:101C400020204D696E3A20004F6E20004F666600DE
:101C5000536F667420656E6473746F70733A2000FE
:101C60004B64200023646566696E652044454641E7
:101C7000554C545F004B69200023646566696E65AE
:101C80002044454641554C545F004B70200023646E
:101C90006566696E652044454641554C545F005069
:101CA0004944204175746F74756E652066696E696C
:101CB00073686564212050757420746865206C61B8
:101CC0007374204B702C204B6920616E64204B6430
:101CD00020636F6E7374616E74732066726F6D2013
:101CE00062656C6F7720696E746F20436F6E6669F2
:101CF0006775726174696F6E2E680A0050494420DE
:101D00004175746F74756E65206661696C656421D8
:101D10002074696D656F75740A004531205448451B
:101D2000524D414C2052554E415741590042454475
:101D300020544845524D414C2052554E415741592F
:101D400000546865726D616C2052756E61776179BF
:101D50000045312048656174696E67206661696C71
:101D60006564004265642068656174696E67206619
:101D700061696C65640048656174696E67206661BD
:101D8000696C656400504944204175746F74756EC8
:101D900065206661696C6564212054656D706572AB
:101DA000617475726520746F6F20686967680A00D6
:101DB000204B643A2000204B693A2000204B703AB7
:101DC00020000A20436C61737369632050494420EA
:101DD0000A002054753A2000204B753A2000206DEF
:101DE00061783A2000206D696E3A200020643A2024
:101DF0000020626961733A200050494420417574A3
:101E00006F74756E65206661696C65642120546528
:101E10006D706572617475726520746F6F2068698A
:101E200067680A00504944204175746F74756E6587
:101E30002073746172740A00504944204175746FB4
:101E400074756E65206661696C6564212042616409
:101E5000206578747275646572206E756D62657246
:101E60000A004F66660A0046616465204865696736
:101E700068742000426564204C6576656C696E6705
:101E800020004661696C656420746F20656E616234
:101E90006C6520426564204C6576656C696E670AE6
:101EA000004D65736820426564204C6576656C2042
:101EB000646174613A0A004D65736820706F696EE1
:101EC000742063616E6E6F74206265207265736F3B
:101ED0006C7665640A004D34323120696E636F722E
:101EE0007265637420706172616D657465722075CE
:101EF000736167650A00496E736572742066696C68
:101F0000616D656E7420616E642073656E64204D32
:101F10003130380A0053656E64204D3130382074FA
:101F20006F2068656174206E6F7A7A6C650A00496B
:101F30006E736572742066696C616D656E74206184
:101F40006E6420707265737320627574746F6E2096
:101F5000286F72204D313038290A0020746F6F20AD
:101F60006C6F6E6720657874727573696F6E207020
:101F7000726576656E7465640A0020636F6C642018
:101F8000657874727573696F6E2070726576656EB0
:101F90007465640A00486F6D696E67206661696CDC
:101FA000656400206E6F7420656E74657265642EC2
:101FB0000A0050726F7465637465642050696E0A1C
:101FC0000046696C616D656E7420757365643A20B6
:101FD0000053746174733A20002C204C6F6E676557
:101FE0007374206A6F623A2000546F74616C2074BD
:101FF000696D653A200053746174733A20002C2097
:102000004661696C65643A20002C2046696E6973EC
:102010006865643A20005072696E74733A20005308
:10202000746174733A20004A3036004A3034004AF2
:1020300030370020573A004A3038004A3039002003
:10204000573A00205A3A0020593A0020436F756EE3
:102050007420583A0020453A00205A3A0020593A54
:1020600000583A002569730025696D2025697300C1
:102070002569682025696D2025697300256964201C
:102080002569682025696D202569730025697920F7
:10209000256964202569682025696D2025697300FC
:1020A000656E7175657565696E672022005072698D
:1020B0006E7465722073746F7070656420647565EA
:1020C00020746F206572726F72732E2046697820BB
:1020D000746865206572726F7220616E642075731A
:1020E00065204D39393920746F20726573746172BF
:1020F000742E202854656D70657261747572652048
:1021000069732072657365742E2053657420697439
:102110002061667465722072657374617274696E91
:1021200067290A004E6F20436865636B73756D20E5
:1021300077697468206C696E65206E756D62657272
:102140002C204C617374204C696E653A20004E6FF0
:1021500020436865636B73756D2077697468206CC4
:10216000696E65206E756D6265722C204C617374AA
:10217000204C696E653A2000636865636B73756D0A
:10218000206D69736D617463682C204C61737420D9
:102190004C696E653A20004C696E65204E756D6223
:1021A0006572206973206E6F74204C617374204CCB
:1021B000696E65204E756D6265722B312C204C6105
:1021C0007374204C696E653A20004D313130004DFA
:1021D00033310053442072656164206572726F72FE
:1021E0000A00446F6E65207072696E74696E6720B4
:1021F00066696C650A0020496E76616C69642065C9
:102200007874727564657220000000A0C000000040
:102210000000000000000057430000574300004D3D
:1022200043454550524F4D206461746173697A652E
:10223000206572726F722E0A00290A00206279747A
:1022400065733B20637263200053657474696E6725
:10225000732053746F726564202800290A0020627D
:10226000797465733B2063726320002073746F720E
:1022700065642073657474696E6773207265747227
:102280006965766564202800202863616C63756C3D
:102290006174656429210A0020213D2000454550D4
:1022A000524F4D20435243206D69736D61746368D2
:1022B000202D202873746F726564292000205369D3
:1022C0007A653A2000496E6465783A2000204D61B5
:1022D000726C696E3D563535290A002845455052C5
:1022E0004F4D3D00454550524F4D20766572736904
:1022F0006F6E206D69736D6174636820006F706527
:102300006E206661696C65642C2046696C653A20B4
:102310000043616E6E6F74206F70656E207375621E
:1023200064697220004A3233004A3035004A323341
:10233000004D32350053442063617264206F6B0A94
:10234000006F70656E526F6F74206661696C6564B2
:102350000A00766F6C756D652E696E697420666112
:10236000696C65640A004572726F723A00534420CA
:10237000696E6974206661696C0A006563686F3A0A
:10238000004A3135004A3132004A313700202050AE
:102390006C616E6E657242756666657242797465CF
:1023A000733A20002046726565204D656D6F727925
:1023B0003A2000436F6D70696C65643A204665622F
:1023C00020323420323031390A00207C20417574AB
:1023D000686F723A2028646176696472616D69720F
:1023E0006F290A00323031392D30322D323400203D
:1023F0004C61737420557064617465643A20007692
:10240000312E342E320A004D61726C696E2D4149B5
:10241000334D00312E312E390A004D61726C696ED8
:102420000020536F6674776172652052657365741E
:102430000A00205761746368646F67205265736592
:10244000740A002042726F776E206F757420526597
:102450007365740A002045787465726E616C205251
:10246000657365740A00506F77657255700A007362
:10247000746172740A004D3234004D32332025737A
:10248000006175746F25692E67006572726F722026
:1024900077726974696E6720746F2066696C650A6B
:1024A00000205A3A0020593A0020583A00656E64DC
:1024B00073746F7073206869743A2000446F6E659E
:1024C00020736176696E672066696C652E0A004D1F
:1024D0003239007C3C3E5E2B3D3F2F5B5D3B2C2A1E
:1024E000225C00627573793A2070617573656420AF
:1024F000666F7220696E7075740A00627573793A3E
:102500002070617573656420666F722075736572E3
:102510000A00627573793A2070726F63657373692C
:102520006E670A004A3135004B494C4C45442E2019
:10253000004B494C4C2063617573656420627920BF
:102540004B494C4C20627574746F6E2F70696E0A23
:10255000004B494C4C45442E20004B494C4C2063C9
:10256000617573656420627920746F6F206D756387
:102570006820696E6163746976652074696D652091
:102580002D2063757272656E7420636F6D6D616E60
:10259000643A20004A3131005072696E74657220CD
:1025A00068616C7465642E206B696C6C28292063EB
:1025B000616C6C6564210A000000A0C0000000008E
:1025C0000000000000004842000048420000804037
:1025D000000000005761726E696E673A20486F6DA7
:1025E000696E672042756D702044697669736F72F9
:1025F000203C20310A000202040000A0400000A09C
:10260000400000004000005C430000574300004DC4
:1026100043FFFFFF486F74656E6420746F6F206323
:102620006F6C640A00486F74656E6420746F6F206D
:10263000636F6C640A0000002100240027002A0058
:102640002D003000330001010000040107010A01E0
:1026500000002200250028002B002E00310034004D
:1026600002010000050108010B0100002000230009
:10267000260029002C002F00320000010000030179
:1026800006010901050505050705080808080202F5
:1026900002020A0A080804040404010101010101FC
:1026A00001010303030303030303040707070C0CDF
:1026B0000C0C0C0C0C0C02020202060606060606A6
:1026C00006060B0B0B0B0B0B0B0B0102102020084B
:1026D000081020401020408002010201080402017D
:1026E00001020408102040808040201008040201EC
:1026F0008004020180402010080402010804020145
:1027000001020408102040800102040810204080CB
:1027100000000A0B02090C0D0E080703040100005B
:1027200000000000000000000000000000000000A9
:102730000000000000000000000000001211100066
:102740000000000000000000000000000000000089
:10275000000000000000556E6B6E6F776E20636F97
:102760006D6D616E643A202200496E73657274204B
:1027700066696C616D656E7420616E64207072654F
:10278000737320627574746F6E20286F72204D31E0
:102790003038290A002066697273740A005A005999
:1027A000005800486F6D65200047393000473120E0
:1027B0005A31204632343000473931004739300031
:1027C0004731205A352046323430004739310047EE
:1027D0003930004731205A313020463234300047FA
:1027E000393100473930004731205A3230204632E3
:1027F0003430004739310054524947474552454427
:10280000006F70656E003A20007A325F6D696E006D
:102810007A5F6D696E00795F6D696E00785F6D69D2
:102820006E005265706F7274696E6720656E6473B6
:10283000746F70207374617475730A000A4D65615A
:10284000737572656420706F696E74733A0A005A0A
:10285000206F66667365743A20004E756D20582CA3
:10286000593A20352C350A00000000010000000113
:102870000000800055555500000040003333330000
:10288000AAAA2A004992240000002000C7711C0057
:1028900099991900D1451700555515003BB1130002
:1028A0002449120011111100000010000F0F0F0039
:1028B000E3380E0043790D00CCCC0C00C3300C0083
:1028C000E8A20B0064210B00AAAA0A00703D0A00CE
:1028D0009DD80900427B090092240900DCD308003E
:1028E000888808001042080000000800F0C10700B6
:1028F0008787070075500700711C07003EEB060034
:10290000A1BC06006990060066660600703E0600DF
:102910006118060017F4050074D105005BB00500CE
:10292000B290050062720500555505007839050022
:10293000B81E0500050505004EEC040087D4040010
:10294000A1BD040090A7040049920400C17D0400C9
:10295000EE690400C7560400444404005C320400DD
:102960000821040041100400000004003FF00300AF
:10297000F8E0030026D20300C3C30300CCB5030074
:102980003AA803000A9B0300388E0300C0810300AD
:102990009F750300D0690300505E03001D530300C0
:1029A00034480300913D030033330300162903002C
:1029B000381F030097150300300C030003030300C6
:1029C0000BFA020049F10200BAE802005CE00200E2
:1029D0002DD802002DD0020059C80200B0C002005C
:1029E00031B90200DAB10200AAAA0200A0A30200D3
:1029F000BC9C0200FA9502005C8F0200DF88020096
:102A000082820200457C02002776020027700200C5
:102A1000436A02007C640200D05E02003F5902005B
:102A2000C8530200526573656E643A20006F6B00F4
:102A300020746F6F206C6F6E672065787472757389
:102A4000696F6E2070726576656E7465640A002029
:102A5000636F6C6420657874727573696F6E207033
:102A6000726576656E7465640A00FFFDFCFAF8F61F
:102A7000F4F2F0EEECEAE9E7E5E3E1E0DEDCDAD9F6
:102A8000D7D5D4D2D0CFCDCBCAC8C7C5C3C2C0BF9B
:102A9000BDBCBAB9B7B6B4B3B2B0AFADACAAA9A811
:102AA000A6A5A4A2A1A09E9D9C9A9998979594935F
:102AB00092908F8E8D8B8A8988878684838281808D
:102AC0007F7E7D7B7A797877767574737271706F9B
:102AD0006E6D6C6B6A696867666564636261605F8E
:102AE0005E5D5C5B5A595858575655545352515075
:102AF000504F4E4D4C4B4A4A494847464645444341
:102B0000424241403F3E3E3D3C3B3B3A39383837FC
:102B1000363535343332323130302F2E2E2D2C2BAA
:102B20002B2A29292827272625252423232221214A
:102B300020201F1E1E1D1C1C1B1B1A1919181817DC
:102B40001616151514131312121111100F0F0E0E65
:102B50000D0D0C0C0B0A0A090908080707060605E3
:102B60000504040303020201000048617264636FFC
:102B70006465642044656661756C74205365747483
:102B8000696E6773204C6F616465640A00D007004A
:102B900000B00400003C000000102700000000FA14
:102BA000430000F0420000C040000070420000A05E
:102BB000420000A0420000C8433333B94220286DD0
:102BC0006D290020204D36303320002055004C0068
:102BD00046696C616D656E74206C6F61642F756EF3
:102BE0006C6F6164206C656E677468733A0A0020CC
:102BF000204D393030204B004C696E6561722041A8
:102C00006476616E63653A0A002044002049002022
:102C1000204D333034205000204400204900202033
:102C20004D3330312050005049442073657474692D
:102C30006E67733A0A00205A0020204D363636005F
:102C4000456E6473746F702061646A7573746D652A
:102C50006E743A0A00205A00205900202047323969
:102C6000205333205800205A0020204D3432302089
:102C700053004D65736820426564204C6576656C31
:102C8000696E673A0A00205A0020590020204D3210
:102C90003036205800486F6D65206F666673657426
:102CA0003A0A00204500205A0020590020580020F0
:102CB000540020530020204D323035205100204553
:102CC0003C6D61785F655F6A65726B3E0020583CC1
:102CD0006D61785F785F6A65726B3E20593C6D610B
:102CE000785F795F6A65726B3E205A3C6D61785FF0
:102CF0007A5F6A65726B3E00416476616E636564FB
:102D00003A20513C6D696E5F7365676D656E745FE7
:102D100074696D655F75733E20533C6D696E5F66C7
:102D2000656564726174653E20543C6D696E5F74C4
:102D3000726176656C5F66656564726174653E009C
:102D400020540020520020204D32303420500041C9
:102D50006363656C65726174696F6E2028756E6956
:102D600074732F7332293A20503C7072696E745F0D
:102D7000616363656C3E20523C726574726163747A
:102D80005F616363656C3E20543C74726176656C70
:102D90005F616363656C3E0A00204500205A002095
:102DA000590020204D3230312058004D6178696D36
:102DB000756D20416363656C65726174696F6E2027
:102DC00028756E6974732F7332293A0A0020450002
:102DD000205A0020590020204D3230332058004D19
:102DE0006178696D756D206665656472617465737F
:102DF0002028756E6974732F73293A0A00204500E4
:102E0000205A0020590020204D3932205800537498
:102E10006570732070657220756E69743A0A0020BF
:102E2000204D3230302044300A0020204D323030E6
:102E30002044002044697361626C65640A0046693D
:102E40006C616D656E742073657474696E67733A36
:102E5000002020473231202020203B004572726F35
:102E6000722077726974696E6720746F20454550CF
:102E7000524F4D210A004D3234004739300047315E
:102E8000205A2D3130204632343000473931004D40
:102E90003130380057726974696E6720746F20662C
:102EA000696C653A20006F70656E206661696C65BB
:102EB000642C2046696C653A20006F70656E206650
:102EC00061696C65642C2046696C653A200046692E
:102ED0006C652073656C65637465640A00205369D2
:102EE0007A653A200046696C65206F70656E65648E
:102EF0003A20002066696C653A2000646F696E674D
:102F0000006672657368004E6F772000454E44205E
:102F1000535542524F5554494E450A002220706F76
:102F200073002220706172656E743A22005355421C
:102F3000524F5554494E452043414C4C20746172C8
:102F40006765743A22004B494C4C45442E2000746E
:102F50007279696E6720746F2063616C6C20737581
:102F6000622D67636F64652066696C65732077699D
:102F7000746820746F6F206D616E79206C65766562
:102F80006C732E204D4158206C6576656C206973FA
:102F90003A004FE4D4EB11241FBECFEFD1E2DEBFE5
:102FA000CDBF00E00CBF14E0A0E0B2E0EEE6F1EF30
:102FB00001E00BBF02C007900D92A833B107D9F70B
:102FC00029E1A8E3B4E001C01D92A734B207E1F7FC
:102FD00017E1CAECD7E100E006C021970109802F74
:102FE000FE010E940FF8C93CD10780E00807A9F74D
:102FF0000E9409E60C94A6F80C9400002F923F92D0
:103000004F925F926F927F928F929F92AF92BF92F8
:10301000CF92DF92EF92FF920F931F93CF93DF93A4
:10302000CDB7DEB7C354D1090FB6F894DEBF0FBEDB
:10303000CDBF21E020934011809139128D3409F4E5
:1030400059C5843511F40C94622C873411F00C941A
:10305000AE2C80913712909138128B31910509F482
:1030600003C2A4F48430910534F48230910594F5C0
:1030700097FF29C03BC58430910509F4BFC14A9729
:1030800009F034C50E94DF410C94B02C8A329105BE
:1030900009F421C444F48C31910509F415C24D970B
:1030A00009F417C223C58B35910509F49FC48C35EB
:1030B000910509F49FC48A35910509F017C510924E
:1030C00049040C94B02C8091190281110C94B52CF8
:1030D0000C94B02C20911902222311F40C94B02CE2
:1030E00011E0029709F010E00E94908219821A8282
:1030F0001B821C821D821E821F82188682E50E940E
:103100004240882309F42AC10E94C23F4B015C015E
:1031100020E030E0A9010E9496F0882309F434C130
:103120004091540450915504609156047091570495
:1031300048A759A76AA77BA76091580470915904C2
:1031400080915A0490915B046CA77DA78EA79FA7DE
:1031500080918D1190918E11A0918F11B09190114D
:1031600088AB99ABAAABBBAB409191115091921136
:1031700060919311709194114CAB5DAB6EAB7FABD2
:103180009C01AD0168A579A58AA59BA50E9496F032
:1031900081110DC02CA93DA94EA95FA96CA57DA5E3
:1031A0008EA59FA50E9496F0882309F4EDC020E02B
:1031B00030E0A901C501B4010E9496F0881F88275C
:1031C000881F181749F060E070E080E89FEB6CAF53
:1031D0007DAF8EAF9FAF08C080E090E0A0E8BFE376
:1031E0008CAF9DAFAEAFBFAF28A539A54AA55BA5F3
:1031F00068A979A98AA99BA90E9412F568AF79AF3D
:103200008AAF9BAF2CA53DA54EA55FA56CA97DA956
:103210008EA99FA90E9412F56B017C0128AD39ADE2
:103220004AAD5BADCA01B9010E94FBF02B013C0124
:10323000A7019601C701B6010E94FBF09B01AC01FA
:10324000C301B2010E9413F50E947EF72B013C01DD
:1032500020E030E040E05FE30E94FBF024966CAF9A
:103260007DAF8EAF9FAF2497A5019401C501B40136
:103270000E94FBF04B015C0124962CAD3DAD4EADA0
:103280005FAD2497CA01B9010E94FBF09B01AC011C
:10329000C501B4010E9412F50E947EF72CAD3DAD30
:1032A0004EAD5FAD0E94FBF04B015C01C701B60162
:1032B0009058A30192010E94EFF5A50194010E948C
:1032C000FBF06B017C0128A939A94AA95BA968A573
:1032D00079A58AA59BA50E9413F520E030E040E087
:1032E0005FE30E94FBF09B01AC01C701B6010E94A5
:1032F00013F528A539A54AA55BA50E9412F5698397
:103300007A838B839C832CA93DA94EA95FA96CA5C8
:103310007DA58EA59FA50E9413F520E030E040E03A
:103320005FE30E94FBF06B017C01A301920168AD99
:1033300079AD8AAD9BAD0E94EFF5A50194010E9485
:10334000FBF09B01AC01C701B6010E9413F52CA54F
:103350003DA54EA55FA50E9412F512C089E40E940A
:103360004240882331F00E94C23F69837A838B8375
:103370009C838AE40E944240882331F00E94C23F2D
:103380006D837E838F83988720E030E0A901698177
:103390007A818B819C810E9496F081110EC020E081
:1033A00030E0A9016D817E818F8198850E9496F021
:1033B000811103C0E6E6F3E20DC0412FBE016F5F4D
:1033C0007F4F8DE891E10E94C6C30C94B02C0E94FF
:1033D000138EF80184918F010F5F1F4F8111F7CF7A
:1033E000E5E3F2E084918F010F5F1F4F882311F412
:1033F0000C94B02C0E94138EF801F4CF80E50E944B
:103400004240882329F00E94218D6B017C0103C07A
:10341000C12CD12C760183E50E944240882361F0C3
:103420000E94C23F20E030E04AE754E40E94FBF0F3
:103430000E945CF66B017C010E94B07D0E9414A486
:10344000C60ED71EE81EF91E0E9414A4DC01CB0193
:103450008C199D09AE09BF09B7FD02C00C94B02CB0
:1034600080E00E942CAEF0CF0E947DB781110C94B9
:10347000B02C80E090E0A0EAB0E489839A83AB832B
:10348000BC8380E090E0ADE4B3E48D839E83AF83A2
:10349000B88780E090E0A0EAB1E489879A87AB879B
:1034A000BC8780E50E944240882319F00E94923F29
:1034B00001C060E068A3BE016F5F7F4FCE018096C0
:1034C0000E9477C10C94B02C80E00E94BD850C94C2
:1034D000B02C83E50E944240882321F10E94A23F44
:1034E000182F863070F0EBEFF2E084918F010F5FC0
:1034F0001F4F882311F40C94B02C0E94138EF801F6
:10350000F4CF833009F44AC130F4813091F1823034
:1035100009F43FC008C0843009F4ABC1853009F418
:10352000B8C101C010E00E940E84811103C0EBED10
:10353000F2E013C080915B11882319F063E173E01E
:1035400002C067E173E083ED92E00E94DBCE8AE087
:103550000E94138E0E941EC2A2C184917F019FEF20
:10356000E91AF90A882309F49AC10E94138EF70117
:10357000F4CF0E94D1C2109201021092000288EC96
:1035800092E090931807809317070E947B8E0C940B
:10359000B02C809100029091010297FF0EC0EFE9DC
:1035A000F2E084918F010F5F1F4F882311F40C9478
:1035B000B02C0E94138EF801F4CF0097A1F48091F3
:1035C000410280934A0419821A821B821C8218A22B
:1035D00019A21AA21BA2BE016F5F7F4FCE01809677
:1035E0000E949F8527C0815065E00E94DBF780FF25
:1035F00003C024E0291B922FA5E09A02F0011124B8
:10360000E80FF11D87FDFA95EE0FFF1FEE0FFF1F6C
:10361000EB55FE4E80915C0490915D04A0915E0498
:10362000B0915F0480839183A283B38380914A0425
:1036300080934102809100029091010289319105AD
:103640000CF067C0109241029C012F5F3F4F3093F6
:1036500001022093000265E00E94DBF780FF03C0B7
:1036600024E0291B922F40915C0450915D046091ED
:103670005E0470915F0448A359A36AA37BA31982D7
:103680001A821B821C82B4E08B0290011124F90182
:10369000E35AF64F4F012081318142815381F4E09A
:1036A0009F02C0011124BC016F58764F5B01DB0102
:1036B0006D917D918D919C91FE0131966F01E12C70
:1036C000F12C00EA10E40E94B18419821A821B8254
:1036D0001C82B601CE0180960E949F85F5018081F3
:1036E0009181A281B3818093540490935504A09357
:1036F0005604B0935704F40180819181A281B38173
:103700008093580490935904A0935A04B0935B0497
:10371000C8C080E090E0A0EAB0E480935C0490939D
:103720005D04A0935E04B0935F040E945A840E94DB
:10373000B07D8FEF9FEF9093010280930002EBE842
:10374000F2E084918F010F5F1F4F882321F00E94C8
:10375000138EF801F6CF83E992E09A83898304E619
:1037600010E019A308A3BE016F5F7F4FCE018096C2
:103770000E947AB88AEB92E09A83898319A308A3FE
:10378000BE016F5F7F4FCE0180960E947AB881E0C4
:103790000E94BD8581E00E943B8483C088E50E9431
:1037A00042408823D1F00E94923F1FEF160F153040
:1037B000D8F065E070E088E792E00E94C2CEE5E7CD
:1037C000F2E084918F010F5F1F4F882311F40C9456
:1037D000B02C0E94138EF801F4CF88E50E94138E5E
:1037E0000E943FE40C94B02C89E50E94424088235B
:1037F000D1F00E94923F0FEF060F0530D8F065E040
:1038000070E082E692E00E94C2CEEFE5F2E08491A1
:103810008F010F5F1F4F882311F40C94B02C0E946E
:10382000138EF801F4CF89E50E94138E0E943FE4C5
:103830000C94B02C8AE50E944240882399F00E94A3
:10384000C23F25E0129FF0011124E00FF11DEE0FA1
:10385000FF1FEE0FFF1FEB55FE4E608371838283C7
:10386000938335C08AE50E94138E0E943FE40C9436
:10387000B02C8AE50E9442408823A1F30E94C23FF7
:103880006093A1117093A2118093A3119093A4113E
:103890001EC080E00E943B840E94D1C218C012303A
:1038A000B1F460910002709101026931710514F068
:1038B00069E170E080E592E00E94C2CE69E170E0CB
:1038C0008BE492E00E94C2CE8AE00E94138E0E9496
:1038D000C17D0C94B02C80911902882311F40C94B2
:1038E000B02C89E40E944240E82E882321F00E94F7
:1038F000923F062F01C000E08AE40E944240F82E69
:10390000882321F00E94923F162F01C010E0EE2084
:1039100011F0053020F4FF2081F0153070F0E2E165
:10392000F3E084918F010F5F1F4F882311F40C94F3
:10393000B02C0E94138EF801F4CF0E944E40EE206E
:1039400091F044E00402F0011124EF58F64F808119
:103950009181A281B38180938D1190938E11A09358
:103960008F11B0939011FF2091F054E01502F001F7
:103970001124E35AF64F80819181A281B381809313
:10398000911190939211A0939311B093941180E5AB
:103990000E944240882319F00E94B33F03C080E593
:1039A0000E94F93F86E40E9442408823D9F00E9499
:1039B000C23F6B017C0120E030E0A9010E9439F791
:1039C000181684F420E030E040E752E4C701B60165
:1039D0000E94EFF560934202709343028093440289
:1039E000909345020E94D8C70C94B02C20934904B0
:1039F0000C94B02C27E5222E22E0322E36EFE32E57
:103A000030E1F32E64E574E079A768A748E3C42E9B
:103A100044E0D42E00E010E0D1018D911D010E9400
:103A20004240882309F44BC00E94C23F2B013C0155
:103A3000133049F0F60120813181428153810E9487
:103A400012F52B013C01A8A5B9A52D913D914D91F1
:103A50005C91C301B2010E9412F54B015C012DEB98
:103A600037E346E855EB0E9439F787FD0AC02DEB96
:103A700037E346E855E3C501B4010E9496F01816F5
:103A8000F4F4133051F44092600450926104609257
:103A900062047092630401E012C0A5019401F70171
:103AA00060817181828193810E9413F5D7016D93AA
:103AB0007D938D939C931397812F0E949A8C1F5F07
:103AC000B4E0EB0EF11CE8A5F9A53496F9A7E8A738
:103AD000F4E0CF0ED11C143009F09ECF002309F47E
:103AE000F6CE80E694E00E941CB7F1CE0E94AEB8FC
:103AF0000C94B02C80913712909138128537910533
:103B000011F40C94B02C0CF0C0C08C34910509F465
:103B100008C50CF058C08931910509F4E8C21CF5BC
:103B20008431910509F4C9C17CF48131910509F40E
:103B30004AC22CF4029708F4C3C10C945F2C42973C
:103B400009F4E0C60C945F2C8631910509F489C212
:103B50000CF483C28731910509F489C2489709F4AE
:103B60009CC20C945F2C8E31910509F47EC384F4C1
:103B70008B31910509F4D7C20CF4C7C28C31910581
:103B800009F469C34D9711F40C94B02C0C945F2C7C
:103B90008A32910509F46CC44CF48F31910509F413
:103BA00042C4809709F4F3C30C945F2C81339105D0
:103BB00009F492C48B34910511F00C945F2C0E948F
:103BC000F6CE0C94B02C8936910509F472C544F5F3
:103BD0008335910509F492C69CF48E34910509F45D
:103BE000A8C40CF4A2C48135910509F475C68235C8
:103BF000910511F00C945F2C109248040C94B02C99
:103C00008535910509F4B1C60CF47CC68C35910557
:103C100009F4C4C68836910509F48FC40C945F2C4E
:103C20008E36910509F4B2C4A4F48B36910509F4DB
:103C3000BAC50CF49AC58C36910511F40C94B02CCD
:103C40008D36910511F00C945F2C0E94A9860C947E
:103C5000B02C8137910509F4FFC45CF48F369105CF
:103C600009F4A7C48037910511F40C94B02C0C947E
:103C70005F2C8237910509F419C78337910511F03C
:103C80000C945F2CEFEDF4E050C78E3221E09207E8
:103C900011F40C94122A0CF082C0893C910511F4A5
:103CA0000C9496267CF58D37910509F48EC5ACF4FD
:103CB0008737910509F4E1C70CF492C7883791055D
:103CC00009F4DEC78937910511F00C945F2C10922E
:103CD0004D0F10924C0F0C94B02C8B39910509F4B8
:103CE00003C534F48C38910509F425C50C945F2C78
:103CF0008E3B910509F435C5883C910509F4C6C78A
:103D00000C945F2C833D910511F40C94A22844F58A
:103D10008C3C910511F40C94CD266CF48B3C9105F0
:103D200011F00C945F2CA7E5EA2EA2E0FA2E03EE28
:103D300015E00C94BD268D3C910511F40C9442279E
:103D40008E3C910511F00C945F2CE7E5CE2EE2E05D
:103D5000DE2EFEE4EF2EFFE0FF2E10E00C94C927CC
:103D6000823E910511F40C94202964F48C3D910558
:103D700011F40C94A5288D3D910511F40C94B228F2
:103D80000C945F2C8C3251E0950711F40C94492966
:103D90008D32914011F40C9472290C945F2C863F63
:103DA00071E0970711F40C94022B0CF043C08A3990
:103DB000B1E09B0711F40C94B02CBCF48033F1E01B
:103DC0009F0711F40C94692A14F40C94662A833624
:103DD00041E0940709F46DC08039914011F00C94D2
:103DE0005F2C0E94B07D0C94B02C8C3A61E0960759
:103DF00011F40C94DC277CF4843AA1E09A0711F4C6
:103E00000C94FC2A853A914011F00C945F2C0E948E
:103E100039620C94B02C843FE1E09E0711F40C94BD
:103E2000FF2A853F914011F00C945F2C0E94A198CD
:103E30000C94B02C8B3522E0920711F40C943E2B9D
:103E4000C4F4883F51E0950711F40C94112B14F43D
:103E50000C94052B8C3072E0970711F40C94352BE1
:103E60008835924011F00C945F2C0E94B66B0C9434
:103E7000B02C8B38B3E09B0711F40C94B02C6CF48D
:103E80008A39F2E09F0711F40C94C72B84389340D1
:103E900011F40C94F42B0C945F2C803A43E09407BB
:103EA00009F4B4C2873E934011F40C944C2C0C944A
:103EB0005F2CE6E6F3E20C94E92AE0E4F3E08FC03D
:103EC000A0903512B090361280E50E9442408823BF
:103ED00059F00E94218D6B017C0111E0672B682B4A
:103EE000692B31F410E004C010E0C12CD12C760114
:103EF00083E50E944240882311F40C94BA2C0E945E
:103F0000C23F20E030E04AE754E40E94FBF00E9408
:103F10005CF66B017C0111110BC0672B682B692BC0
:103F200039F4A114B10421F0D5018C91811102C0A2
:103F300010E001C011E00E94B07D1123B9F0EBE761
:103F4000F3E284918F010F5F1F4F882321F00E94BD
:103F5000138EF801F6CFF50181915F01882319F0E6
:103F60000E94138EF8CF8AE00E94138E83E0809324
:103F7000401181E080931E19C114D104E104F104C1
:103F8000B1F00E9414A4C60ED71EE81EF91E0E94AE
:103F900014A4DC01CB018C199D09AE09BF09B7FF40
:103FA0000EC080911E1981110C94BF2C08C0809105
:103FB0001E19882321F080E00E942CAEF8CF1092C9
:103FC0001E190C94B02C5F988A984798809108012C
:103FD000817080930601479812980C94B02C8491BC
:103FE0008F010F5F1F4F882321F00E94138EF8016D
:103FF000F6CF1092230C86ED99E00E94C9A68BE1C2
:10400000E6EDF9E0DE01159601900D928A95E1F753
:104010008091D4099091D5099C838B838DEE92E099
:104020009A83898340E050E0BE016F5F7F4F80E05C
:1040300090E00E942CA1CE0101960E94C2ADE1E366
:10404000F3E084918F010F5F1F4F882311F40C94CC
:10405000B02C0E94138EF801F4CF0E940A9F0C949A
:10406000B02C1092A5091092A6090C94B02CE091E6
:104070003512F09136128081882329F0803209F4BC
:1040800010823196F8CF40E061E080913512909136
:1040900036120E94A7DE0C94B02C80E090E0A0E0E5
:1040A000B0E489839A83AB83BC8318A219A21AA2B5
:1040B0001BA21CA21DA21EA21FA28091160788236C
:1040C00059F020E0AE014F5F5F4FBE01605E7F4F51
:1040D000CE0184960E945EBA8091A609882319F0C9
:1040E00081E08093A5090E94F6CE0C94B02C10922A
:1040F000A5090E9466E281E593E0909318078093FA
:1041000017070E947B8E0C94B02C8091A6098823FF
:1041100011F40C94B02C83E50E94424081110C9460
:10412000C42C0C94B02C83E40E94F93F882309F43A
:1041300050C0E3E8F3E084918F010F5F1F4F8823A5
:1041400021F00E94138EF801F6CF8091710B81113E
:1041500003C0E6E5F3E012C0BE016F5F7F4F8EE65D
:104160009BE00E9491A58E010F5F1F4FD8018D919A
:104170008D01882349F10E94138EF8CF84918F011D
:104180000F5F1F4F882301F10E94138EF801F6CFB5
:104190009BEDC92E93E0D92EE12CF12C20E08091EB
:1041A000FF0590E00E2C02C0959587950A94E2F7E2
:1041B00080FD2FC24FEFE41AF40A52E0C50ED11C65
:1041C00065E0E616F10459F78AE00E94138E0C941C
:1041D000B02C8091A609882339F08091A509882305
:1041E00019F0E0E6F3E003C0E2E7F3E028C08491D1
:1041F0008F010F5F1F4F882321F00E94138EF8015B
:10420000F6CF60911F0C7091200C8091210C909141
:10421000220C4AE00E944F918FE20E94138E60911F
:104220001B0C70911C0C80911D0C90911E0C4AE08F
:104230000E944F918AE00E94138E0C94B02C8491BE
:104240008F010F5F1F4F882311F40C94B02C0E9434
:10425000138EF801F4CF40E060E080913512909128
:1042600036120E94A7DE0C94B02C8091A6098823F8
:1042700011F40C94B02C8EE69BE00E94D4DC8EE608
:104280009BE00E946CA51092A4091092A309809152
:10429000A609882311F40C94B02C009135121091CA
:1042A00036120E941EA1B801CE0180960E9432A350
:1042B0008C01892B11F40C94B02C68A179A16115A3
:1042C000710511F06C5F7F4F19821C8222E0A801FA
:1042D000CE0101960E94F6AA811102C0F12C14C0F1
:1042E000CE0101960E948EA08823C1F361E0CE0129
:1042F00001960E9475A5009789F325EEFC012083A5
:104300001C820E947DDAF82ECE0101960E940D8E4D
:10431000F11003C0E0EAF3E022C0E2E9F3E08491A7
:104320007F012FEFE21AF20A882321F00E94138EF8
:10433000F701F5CFD8018D918D01882319F00E94E6
:10434000138EF8CF8AE00E94138E10921F0C1092E9
:10435000200C1092210C1092220C0C94B02C849101
:104360007F01BFEFEB1AFB0A882321F00E94138E16
:10437000F701F5CFF80181918F01882319F00E9490
:10438000138EF8CF8EE20E94138E0C94B02C809185
:10439000A50981110E94B07D8091A609882311F49E
:1043A0000C94B02C80E50E944240882319F00E94B2
:1043B000B33F03C080E50E94F93F182F482F61E00A
:1043C00080913512909136120E94A7DE83E50E94FB
:1043D0004240882381F00E94923FAB01BC01409390
:1043E0001F0C5093200C6093210C7093220C8EE6CE
:1043F0009BE00E9482A48091A609882319F081E0A5
:104400008093A50911110C94B02C6DCE80913512BA
:104410009091361221E02093A40940E060E00E94D0
:10442000A7DE0C94B02C0E9417E268A379A38AA39C
:104430009BA3BE016F5F7F4FCE0180960E94318D9E
:10444000EBE7F3E284918F010F5F1F4F882321F088
:104450000E94138EF801F6CFBE016F5F7F4F88EB8D
:1044600093E00E94DBCE8AE00E94138E0C94B02C65
:1044700083E50E944240882311F40C94B02C0E94E2
:10448000A23FE82E80E50E944240882339F00E9436
:10449000A23F182F87FF03C00C94B02C1DE089E4C5
:1044A0000E944240882341F00E94B33F81110C9446
:1044B000412DE6E4F6E00BC089E40E94F93FF6CF17
:1044C000319626E0E637F20711F40C94412D8491E1
:1044D0001813F6CF0C94152DF090440481E0F826C3
:1044E000F0924404E0EDF3E084918F010F5F1F4FE1
:1044F000882321F00E94138EF801F6CFFF2019F0D7
:10450000E5ECF3E002C0EAECF3E084918F010F5F89
:104510001F4F882311F40C94B02C0E94138EF801C5
:10452000F4CF0E9466E20C94B02C0E943DCF0C9414
:10453000B02C0E9476800C94B02C88E690E00E940B
:104540001A8E81110C94B02C8091FF0583FF02C05C
:104550000C94B02C83E50E944240882399F00E947D
:10456000C23F0E9457F6CB010E948F5A0E94C23F61
:1045700020E030E04AEA52E40E9496F0181614F067
:104580000E943DCF0E94EFD00C94B02C8EE40E948C
:104590004240882311F40C94B02C0E94923F609307
:1045A00021197093221980932319909324190C9444
:1045B000B02C83E50E94F93F882359F083E50E94DF
:1045C0004240882319F00E94A23F01C080E08093FE
:1045D000FF05EBE7F3E284918F010F5F1F4F81111D
:1045E00003C0E9EEF3E004C00E94138EF801F3CF9C
:1045F00084918F010F5F1F4F882321F00E94138E3B
:10460000F801F6CF8091FF058111C2CDE5EEF3E010
:1046100018C0BB24B394B20E222319F08CE20E947E
:10462000138EF60185919491FC0184918F010F5FA7
:104630001F4F882321F00E94138EF801F6CF2B2DF7
:10464000B9CD84918F010F5F1F4F882309F4BCCD32
:104650000E94138EF801F5CF83E50E94424081113C
:1046600003C0EBE7F3E20DC00E94A23F8D3320F4BC
:10467000809328020C94B02C8CE3809328020C9435
:10468000B02C84918F010F5F1F4F882321F00E946F
:10469000138EF801F6CF4091280250E060E070E000
:1046A00080EF93E00E9488CE8AE00E94138E0C94E3
:1046B000B02C89E690E00E941A8E811111C0E7EFBC
:1046C000F3E084918F010F5F1F4F882321F00E9438
:1046D000138EF801F6CF0E943D598AE00E94138E96
:1046E000109240110C94562D83E50E94424088237D
:1046F00011F40C94B02C0E94A23F182F8D3308F0B7
:104700001CE31093F5100E9414A46B017C01212F6F
:1047100030E0A8EEB3E00E9403F5C60ED71EE81EF7
:10472000F91EC092F110D092F210E092F310F092C4
:10473000F4100C94B02C8091FF0583FF02C00C9400
:10474000B02C83E50E944240882311F40C94B02CD5
:104750000E94C23F0E9457F6CB010E94D1410C94A7
:10476000B02C0E948B7E0C94B02C80E50E944240BD
:10477000811106C083E50E944240882361F006C093
:104780000E94A23F81110C94B02CF4CF0E94923F62
:104790006F3F710510F06FEF70E0709365046093E8
:1047A00064040C94B02C80E50E944240811106C044
:1047B00010926504109264040C94B02C0E94923FF5
:1047C000672B11F00C94B02CF3CF8CE40E94F93FCE
:1047D000882381F00E94C23F6B017C0120E030E021
:1047E000A9010E9439F787FF0BC0F7FAF094F7F898
:1047F000F09406C0C12CD12C80E8E82E80E4F82E7D
:10480000F7FAF094F7F8F094CCA2DDA2EEA2FFA2A2
:1048100080E090E0A0EAB0E489839A83AB83BC8314
:1048200080E090E0ADE4B3E48D839E83AF83B887EE
:1048300080E090E0A0EAB1E489879A87AB87BC87E3
:1048400088E50E944240882379F088E50E94424032
:10485000882319F00E94C23F03C060E070E0CB01E2
:1048600069837A838B839C8389E50E9442408823F5
:1048700079F089E50E944240882319F00E94C23FE6
:1048800003C060E070E0CB016D837E838F839887E7
:104890008AE50E944240882379F08AE50E944240DE
:1048A000882319F00E94C23F03C060E070E0CB0192
:1048B00069877A878B879C8718A219A21AA21BA2E4
:1048C000AE01405E5F4FBE016F5F7F4FCE018496A9
:1048D0000E9407B30C94B02C0E949F5A0E941EBCE9
:1048E000109265041092640468EE73E080E090E03A
:1048F0000E9417620E94702D0C94B02C20934804E3
:104900000C94B02C83E50E9442408823A1F00E94C1
:10491000C23F20E030E04AE754E40E94FBF00E94EE
:104920005CF66093290270932A0280932B02909385
:104930002C020C94B02C88E50E94F93F81110C9454
:10494000D52C89E50E94F93F81110C94D52C8AE57C
:104950000E94F93F81110C94D52C85E40E94F93F07
:1049600081110C94D52C0C94072D83E50E94F93FFE
:10497000882309F4F5C70E94C23F20E030E04AE7EF
:1049800054E40E94FBF00E945CF66093ED1070937B
:10499000EE108093EF109093F010E2C717E5C12E50
:1049A00012E0D12E01E7E02E01E1F02E10E0D60159
:1049B0008D916D010E94F93F882309F46DC0133079
:1049C00009F063C00E94C23F4B015C0120E030E06F
:1049D00040EA51E40E9496F087FF4EC0A501940181
:1049E00060917D1170917E1180917F119091801165
:1049F0000E94EFF52B013C019B01AC016091D305B6
:104A00007091D4058091D5059091D6050E94FBF058
:104A10006093D3057093D4058093D5059093D60504
:104A2000A30192016091EF057091F0058091F1056D
:104A30009091F2050E94FBF06093EF057093F005F2
:104A40008093F1059093F205609162127091631268
:104A500080916412909165120E949AF0A3019201D4
:104A60000E94FBF00E945CF66093621270936312E6
:104A7000809364129093651280927D1190927E11C2
:104A8000A0927F11B092801107C00E94C23FF7012F
:104A900060837183828393831F5FF4E0EF0EF11CC8
:104AA000143009F084CF0E9490D25AC70E94B07D82
:104AB00083E50E944240882311F40C94671C0E94F5
:104AC000923F6230710511F00C94671C0E94B2CBCA
:104AD0008BE50E94138E60913A1270913B12809187
:104AE0003C1290913D1242E00E94D49140913E12BE
:104AF00050913F1260914012709141128DEF93E0FE
:104B00000E94A5CE409142125091431260914412EE
:104B1000709145128AEF93E00E94A5CE8DE50E9428
:104B2000138E8AE00E94138E1BC784918F010F5F42
:104B30001F4F882321F00E94138EF801F6CF60E00A
:104B40008FEC94E00E947F6B61E088EC94E00E941F
:104B50007F6B61E08DEB94E00E947F6B61E08DEAFA
:104B600094E00E947F6B60E084EA94E00E947F6B97
:104B700061E08AE994E00E947F6B60E080E994E064
:104B80000E947F6B60E088E894E00E947F6B61E0A8
:104B90008AE794E00E947F6B60E08CE694E00E94DC
:104BA0007F6B60E08DE594E00E947F6B60E08FE4B6
:104BB00094E00E947F6B60E089E394E00E947F6B49
:104BC00061E088E294E00E947F6B60E083E194E022
:104BD0000E947F6B61E080E094E00E947F6BC0C622
:104BE000009135121091361283E0D12C40E08150B3
:104BF000E9F0D8019C91292F2B7F2134C1F7119620
:104C00002C912133A1F7913421F0953421F441E026
:104C100002C0DD24D39498012E5F3F4F89012F5F9E
:104C20003F4FF80190819032C9F3E1CF442369F0FE
:104C3000EBE7F3E284917F012FEFE21AF20A882377
:104C400021F00E94138EF701F5CFDD2069F0E4ED2D
:104C5000F5E084917F014FEFE41AF40A882321F0F4
:104C60000E94138EF701F5CFD8018D918D01882315
:104C700009F4AACA0E94138EF7CF0E9490C370C68F
:104C800081E080934D0F80934C0F6AC688EC90E0D2
:104C90000E941A8E811164C684E40E94F93F882321
:104CA00009F441C00E94C23F6B017C0111E020E089
:104CB00030E0A9010E9496F0811101C010E010932C
:104CC000091220E030E0A901C701B6010E9496F068
:104CD000882349F10E94C23FE0917205B4E0EB9F46
:104CE000F0011124E25FFD4E608371838283938320
:104CF00020E030E0A90160910E1270910F128091B6
:104D00001012909111120E9496F081110CC080E057
:104D100090E0A0EEBFE380930E1290930F12A09349
:104D20001012B09311120E945DBC1AC6B7E5EB2EAB
:104D3000B2E0FB2E06E612E1F70181917F010E94AD
:104D4000F93F882351F00E94C23F0E945CF6D801CF
:104D50006D937D938D939C9313970C5F1F4FB2E1DE
:104D600006371B0749F70E941FD1FAC50C5F1F4F7A
:104D7000B5E0033F1B0709F4F3C5F70181917F01FB
:104D80000E94F93F882391F30E94C23FD8016D939E
:104D90007D938D939C931397E9CF83E50E944240C6
:104DA0008823A1F00E94C23F6093DF057093E00565
:104DB0008093E1059093E2056093DB057093DC0539
:104DC0008093DD059093DE0510E001C011E080E5E1
:104DD0000E944240882359F00E94C23F6093DF0541
:104DE0007093E0058093E1059093E20510E082E581
:104DF0000E944240882359F00E94C23F60933C11B8
:104E000070933D1180933E1190933F1110E084E523
:104E10000E944240882359F00E94C23F6093DB0504
:104E20007093DC058093DD059093DE0599C5112311
:104E300009F496C54091DF055091E0056091E105C8
:104E40007091E2058EED95E00E94A5CE40913C1157
:104E500050913D1160913E1170913F118BED95E0A5
:104E60000E94A5CE4091DB055091DC056091DD05E7
:104E70007091DE0588ED95E00E94A5CE8AE00E9443
:104E8000138E6EC581E50E94F93F882351F00E9480
:104E9000218D6093F3057093F4058093F50590934D
:104EA000F60583E50E94F93F882351F00E94C23F36
:104EB0006093FB057093FC058093FD059093FE05C0
:104EC00084E50E94F93F882351F00E94C23F60931D
:104ED000F7057093F8058093F9059093FA0588E536
:104EE0000E94F93F882351F00E94C23F6093C7059A
:104EF0007093C8058093C9059093CA0589E50E94FF
:104F0000F93F882351F00E94C23F6093CB05709314
:104F1000CC058093CD059093CE058AE50E94F93F9C
:104F20008823F1F00E94C23F6093CF057093D005B3
:104F30008093D1059093D2052DEC3CEC4CEC5DE3D5
:104F40000E9496F0181664F0EEEEF5E084918F0161
:104F50000F5F1F4F882321F00E94138EF801F6CFB8
:104F600085E40E94F93F882309F4FAC40E94C23FF5
:104F70006093D3057093D4058093D5059093D6059F
:104F8000EFC41F5FB4E0EB0EF11C133011F40C946E
:104F9000671CF60181916F010E94F93F882389F314
:104FA0000E94C23FD7016D937D938D939C9313977D
:104FB000812F0E949A8CE5CF0E947DB78111D0C4C9
:104FC00008EB15E2E4E5F4E0F9A7E8A7AE014F5FCE
:104FD0005F4F4A0171E1A72E76E2B72E1A01F80160
:104FE0006591759185919491A8A5B9A5CD90DD9015
:104FF000ED90FD90B9A7A8A7A70196010E9412F510
:105000002B013C01F101608371838283938320E053
:1050100030E040EA51EC0E9439F787FD0AC020E0F9
:1050200030E040EA51E4C301B2010E9496F0181644
:105030002CF4F501849118160CF4ECC4D101CD9038
:10504000DD90ED90FD901D0120E030E040EA51EC54
:10505000C701B6010E9439F787FD0AC020E030E0A1
:1050600040EA51E4C701B6010E9496F018164CF5CB
:10507000E6E6F3E284918F010F5F1F4F811103C0B9
:10508000E0E2F6E004C00E94138EF801F3CF8491B1
:105090008F010F5F1F4F882321F00E94138EF801AC
:1050A000F6CF88E290E099A388A388EC90E09DA3D6
:1050B0008CA3BE01605E7F4FCE0184960E947AB8B9
:1050C0004FC40C5F1F4FBFEFAB1ABB0AE4ECF5E215
:1050D000E017F10709F083CF6EE4E62E6FE0F62EBD
:1050E00010E0F40181919191A191B1914F01F701EB
:1050F00081939193A193B1937F01812F0E949A8C08
:105100001F5F133071F70E94C17D83E992E09DA378
:105110008CA304E610E019A308A3BE016C5D7F4FC9
:10512000CE0180960E947AB88AEB92E09DA38CA370
:1051300019A308A3BE016C5D7F4FCE0180960E942B
:105140007AB80EC40E94A16A0BC483E50E94424053
:10515000882309F405C40E94923F70930302609370
:105160000202FEC38DED90E00E941A8E8111F8C3F9
:1051700083E50E944240811103C0EBE7F3E23AC0AD
:105180000091720510E00E94923F000F111FF8017C
:10519000E15CFD4F718360838091720590E07C013A
:1051A000EE0CFF1CEE0CFF1C8701025E1D4F880FEA
:1051B000991FFC01E15CFD4F60817181072E000C9D
:1051C000880B990B0E949CF02AE037ED43E25CE3E8
:1051D0000E94FBF0F701E65FFD4E208131814281A4
:1051E00053810E94FBF0D8016D937D938D939C9326
:1051F0001397B6C384918F010F5F1F4F882321F04F
:105200000E94138EF801F6CF85E40E94138E8091E0
:105210007205805D0E94138EE0917205F0E0EE0F42
:10522000FF1FE15CFD4F608171818EE396E00E947B
:10523000C2CE85E20E94138E8AE00E94138E90C334
:1052400080E50E94F93F882309F48AC30E94923FB7
:105250006B017C0183E50E944240882321F00E947B
:10526000923F8B0102C00FEF1FEFC8010196039719
:1052700008F076C3D7FC74C38C2DE6E4F6E0949175
:10528000891709F4D2C33196B6E0E637FB07B9F7C0
:10529000CFC383E50E944240882319F00E94923FC9
:1052A00002C064E071E079A368A380E50E944240F7
:1052B000882339F00E94923F6938E3E17E0730F499
:1052C00002C068EE73E07A83698304C088E893E1E2
:1052D0009A838983BE01605E7F4FCE0101960E9452
:1052E0007AB83EC385E40E944240811110C080E537
:1052F0000E94F93F882391F00E94C23F60935B05B2
:1053000070935C0580935D0590935E0507C00E94D5
:10531000A23F882361F3E6E6F3E271C089E40E94CC
:10532000F93F882381F00E94C23F2CEA35EC47E226
:105330005EE30E94FBF060935705709358058093DD
:10534000590590935A0584E40E94F93F882381F01F
:105350000E94C23F2CEA35EC47E25EE30E94EFF583
:1053600060935F057093600580936105909362057B
:10537000EBE7F3E284918F010F5F1F4F882321F049
:105380000E94138EF801F6CF40915B0550915C05A9
:1053900060915D0570915E058EE796E00E94A5CE56
:1053A0002CEA35EC47E25EE36091570570915805B1
:1053B0008091590590915A050E94EFF5AB01BC010F
:1053C0008AE796E00E94A5CE2CEA35EC47E25EE340
:1053D00060915F0570916005809161059091620513
:1053E0000E94FBF0AB01BC0186E796E00E94A5CECF
:1053F0008AE00E94138EB4C20E94138EF801849139
:105400008F010F5F1F4F8111F7CFE2E8F6E0849123
:105410008F010F5F1F4F882309F4A2C20E94138ED1
:10542000F801F5CF83E50E94F93F182F882371F02A
:105430000E94C23F0E9457F670933A02609339026D
:1054400021E0672B09F020E02093511180E50E94B4
:10545000F93F882359F02091390230913A02232BE9
:1054600011F00E94B33F809351117AC2111178C29A
:10547000EBE7F3E284918F010F5F1F4F882321F048
:105480000E94138EF801F6CF80915111882319F0F4
:105490006BE173E002C06EE173E089EA96E00E947E
:1054A000DBCE6091390270913A0288E996E00E9461
:1054B000C2CEE4E9F6E084918F010F5F1F4F88238D
:1054C00009F44EC20E94138EF801F5CF0E942865A0
:1054D00047C280E50E94F93F882351F00E94C23FF5
:1054E000609353057093540580935505909356052A
:1054F00089E40E94F93F882381F00E94C23F2CEA90
:1055000035EC47E25EE30E94FBF060934F05709339
:105510005005809351059093520584E40E94F93F11
:10552000882381F00E94C23F2CEA35EC47E25EE31B
:105530000E94EFF560934B0570934C0580934D05E9
:1055400090934E05EBE7F3E284918F010F5F1F4FBD
:10555000882321F00E94138EF801F6CF4091530565
:1055600050915405609155057091560584EC96E074
:105570000E94A5CE2CEA35EC47E25EE360914F0530
:105580007091500580915105909152050E94EFF560
:10559000AB01BC0180EC96E00E94A5CE2CEA35EC74
:1055A00047E25EE360914B0570914C0580914D059B
:1055B00090914E050E94FBF0AB01BC018CEB96E094
:1055C0000E94A5CE8AE00E94138ECAC10E94138E4B
:1055D000F80184918F010F5F1F4F8111F7CFE8EC25
:1055E000F6E084918F010F5F1F4F882309F4B8C143
:1055F0000E94138EF801F5CF0E942463B1C10E946E
:10560000AD98AEC10E94C5D7ABC183E50E94F93FFA
:10561000882321F00E94B33F91E089270E9401D3A3
:105620009FC181E0809315070E946992109215072F
:10563000882309F495C1EBE7F3E284918F010F5FB2
:105640001F4F811103C0E7EDF6E004C00E94138EE6
:10565000F801F3CF84918F010F5F1F4F882309F466
:105660007FC10E94138EF801F5CF8091A509882390
:1056700009F476C181E08093A80972C18BE592E0BC
:105680000E941A8E81116CC185E50E94F93F882322
:10569000D9F10091720510E00E94C23F6B017C01BC
:1056A00020E030E0A9010E9439F787FF04C0F7FA33
:1056B000F094F7F8F094000F111F000F111FF8017C
:1056C000EE5EF64EC082D182E282F38200917205D4
:1056D000F4E00F9F800111240E5E164E20E030E0B2
:1056E00046E154E4D8016D917D918D919C910E9489
:1056F00039F718164CF480E090E0A6E1B4E4F80124
:1057000080839183A283B3838CE40E94F93F882332
:1057100009F426C10091720510E00E94C23F6B019E
:105720007C0120E030E0A9010E9439F787FF04C026
:10573000F7FAF094F7F8F094000F111F000F111F03
:10574000F801EA5EF64EC082D182E282F3820091D5
:105750007205F4E00F9F800111240A5E164E20E0CE
:1057600030E046E154E4D8016D917D918D919C919A
:105770000E9439F718160CF0F3C080E090E0A6E123
:10578000B4E4F80180839183A283B383E9C08AE5FE
:105790000E944240811103C0E5EEF6E00BC00E947A
:1057A000C23F60931A1970931B1980931C19909330
:1057B0001D19D6C084918F010F5F1F4F882321F0E0
:1057C0000E94138EF801F6CF40911A1950911B19BF
:1057D00060911C1970911D1982EE96E00E94A5CE71
:1057E0008AE00E94138EBCC08BE40E94424081116B
:1057F00003C0EBE7F3E236C08BE40E94424088230B
:10580000C1F00E94C23F6B017C0120E030E0A901A1
:105810000E9439F787FD0AC020E030E040E251E401
:10582000C701B6010E9496F0181634F4E4E0F7E0E0
:105830000EC0C12CD12C76010E94B07DC092D7053C
:10584000D092D805E092D905F092DA0589C084910A
:105850008F010F5F1F4F882309F482C00E94138EAF
:10586000F801F5CF84918F010F5F1F4F882321F03E
:105870000E94138EF801F6CF4091D7055091D805BC
:105880006091D9057091DA0583E297E00E94A5CE78
:105890008AE00E94138E64C081E08093190283E540
:1058A0000E944240882339F00E94B33F811158C0C2
:1058B0000E94EBCB55C083E50E94F93FF7CF0E94D1
:1058C000AEB84EC0F09037120E94B07D10915B11BF
:1058D00080E00E943B84FF2029F1EBE7F3E2849112
:1058E0008F010F5F1F4F882321F00E94138EF80154
:1058F000F6CF84E50E94138E6F2D70E080E090E07B
:105900004AE00E944F9180E20E94138EE0E4F7E0AB
:1059100084918F010F5F1F4F882311F10E94138E16
:10592000F801F6CF10920E11812F0E943B84EBE715
:10593000F3E284918F010F5F1F4F882321F00E94B3
:10594000138EF801F6CF60910E1170E08EE297E0B1
:105950000E94C2CE8AE00E94138E02C00E94AEB89E
:10596000109240110E94CECBA1C00E9490820E9452
:10597000D8C7F6CF11110C94981F0C94911F80E09A
:105980000E942CAE0C94C71F0E94923FAB01BC0139
:1059900040931F0C5093200C6093210C7093220CA9
:1059A0008EE69BE00E9482A4DBCF0E94B07D88E55A
:1059B0000E94F93F882331F05F9A809153048E7FD3
:1059C0008093530489E50E94F93F882339F08A9A2D
:1059D000479A809153048D7F809353048AE50E94F7
:1059E000F93F882361F08091080180958170809350
:1059F0000601479A809153048B7F8093530485E47A
:105A00000E94F93F882309F4ABCF129AA9CF0E94D4
:105A10001EBCA6CFF7FAF094F7F8F094D101CD921E
:105A2000DD92ED92FC92139709CB0E9424E498CF6B
:105A30000E94B07DBC2C60E08C2D0E9421B90F3FEC
:105A4000BFEF1B0759F48C2D0E94CBB831E020E04A
:105A5000892B09F030E0032F122F05C0013011050A
:105A600069F401E010E08B2D0E94CBB880179107FC
:105A700009F476CF80E00E942CAEF5CF00E010E074
:105A8000F2CF61E0812F0E9421B96E2D812F0E94FB
:105A9000F3B8F12CB701812F0E945DB9193009F0DC
:105AA0005FCFF0926504E09264045ACFCD5BDF4F84
:105AB0000FB6F894DEBF0FBECDBFDF91CF911F911F
:105AC0000F91FF90EF90DF90CF90BF90AF909F909D
:105AD0008F907F906F905F904F903F902F900895A0
:105AE0002F923F924F925F926F927F928F929F92EE
:105AF000AF92BF92CF92DF92EF92FF920F931F93DC
:105B0000CF93DF93CDB7DEB76F970FB6F894DEBFB4
:105B10000FBECDBFC0906E04D0906F04E0907004B3
:105B2000F090710420E030E040EA50E4C701B60193
:105B30000E9496F087FD19C120E030E041E953E46E
:105B4000C701B6010E9439F718160CF40EC1109265
:105B5000C40D1092C30D809109014091C20D042E15
:105B6000000C550B817021E0822790E048175907FF
:105B700009F433C080910901817028272093C20D58
:105B800081111BC00E940A9FE8E5FEE084918F010D
:105B9000882351F0082E000C990B0E94059F0F5F7F
:105BA0001F4FF8018491F4CF8DE090E00E94059F93
:105BB0008AE090E00E94059F10C0ECE5FEE0849131
:105BC0008F01882389F3082E000C990B0E94059FF2
:105BD0000F5F1F4FF8018491F4CF8091280C833020
:105BE00009F44CC02CF4882351F08130D9F072C0F4
:105BF000843009F43EC0853009F44DC06BC08091FB
:105C0000A509882309F466C081E08093280C0E94CE
:105C100014A46093B90D7093BA0D8093BB0D90934B
:105C2000BC0D58C08091A509811154C08091710BA1
:105C3000882321F082E08093280C4CC01092280C1D
:105C4000E4E5FEE084918F01882351F0082E000CDA
:105C5000990B0E94059F0F5F1F4FF8018491F4CFAD
:105C60008DE090E00E94059F8AE090E00E94059FF1
:105C700031C08091020E8823E9F22CC08091A509E1
:105C8000811128C08091270990912809891B8F7064
:105C900009F496C01FC08091A50981111BC0809195
:105CA000270990912809891B8F7009F4EEC012C052
:105CB0008DE090E00E94059F8AE090E00E94059FA1
:105CC0001092280C80EF9DE090931807809317079F
:105CD0000E947B8E8091AB0D9091AC0D03974CF59B
:105CE0007CEB272E79E0372EE0E68E2EEAEE9E2E14
:105CF000A12CB12C80E19FE00E94963E1816190657
:105D0000C4F48091AB0D9091AC0D049794F480E1B4
:105D10009FE00E945A3E8093B10DE091B20DF09148
:105D2000B30D8A3019F08D3009F0C0C0309709F0FA
:105D3000C6C08091AB0D9091AC0D009711F40C94FE
:105D4000B73D01979093AC0D8093AB0D8091AD0D55
:105D50009091AE0D019664E070E00E94FCF7909384
:105D6000AE0D8093AD0D0C94B73D8091C30D909115
:105D7000C40D8136FAEE9F07E8F01092C40D109220
:105D8000C30DE0E6FEE084918F01882351F0082ED8
:105D9000000C990B0E94059F0F5F1F4FF801849123
:105DA000F4CF8DE090E00E94059F8AE090E00E9491
:105DB000059FD1CE01969093C40D8093C30DCBCE99
:105DC0008091290C81111FC080912A0C811143C040
:105DD00080E59EE090931807809317070E947B8EC2
:105DE00083E49EE090931807809317070E947B8EB0
:105DF00087E39EE090931807809317070E947B8E9D
:105E000083E39EE022C08FE29EE090931807809388
:105E100017070E947B8E82E29EE090931807809382
:105E200017070E947B8E8EE19EE090931807809367
:105E300017070E947B8E8DE09EE090931807809359
:105E400017070E947B8E8CEF9DE09093180780933C
:105E500017070E947B8E8091020E882311F082E04A
:105E600001C084E08093280CE8EFFDE084918F016D
:105E7000882309F4F5CE082E000C990B0E94059F8B
:105E80000F5F1F4FF8018491F3CFE4EFFDE08491A1
:105E90008F01882309F40CCF082E000C990B0E9467
:105EA000059F0F5F1F4FF8018491F3CF8A3309F4E8
:105EB0003DCFEF35F10514F40C949F3B37CF809123
:105EC000AF0D9091B00D20E6289F8001299F100D05
:105ED0001124C801885D934FE80FF91F13829801C0
:105EE000255D334F790161E470E0C9010E9463F8D8
:105EF000009711F40C94833B9093B50D8093B40DEF
:105F00008E199F09800F911F60E070E0845D934FB0
:105F10000E9497EC0E9457F6CB01770FAA0BBB0BA0
:105F20008232910510F00C94833BFC018827EE58D7
:105F3000FF4F8F4F0C940FF8EBEEFDE084918F0133
:105F4000882351F0082E000C990B0E94059F0F5FCB
:105F50001F4FF8018491F4CF20E030E040E05FE390
:105F600060916E0470916F0480917004909171043F
:105F70001EC0E6EEFDE084918F01882351F0082ECB
:105F8000000C990B0E94059F0F5F1F4FF801849131
:105F9000F4CF60916C0470916D04072E000C880B97
:105FA000990B0E949CF020E030E040E05FE30E940B
:105FB00013F50E9457F6CB010E949B410E944BE1D2
:105FC0008DE090E00E94059F8AE090E00E94059F8E
:105FD0000C94833BE1EEFDE084918F01882351F026
:105FE000082E000C990B0E94059F0F5F1F4FF801B0
:105FF0008491F4CF20E030E040E05FE360916804FA
:106000007091690480916A0490916B04D0CFECED9B
:10601000FDE084918F01882351F0082E000C990B2C
:106020000E94059F0F5F1F4FF8018491F4CF60918C
:10603000660470916704B1CF2091640430916504C7
:1060400044E6429FC001439F900D11246FEF70E022
:106050000E94FCF78B016536710510F004E610E034
:10606000E7EDFDE084917F01882359F0082E000CB4
:10607000990B0E94059FFFEFEF1AFF0AF701849129
:10608000F3CFB80180E090E0CBC7E3EDFDE0849171
:106090008F01882351F0082E000C990B0E94059F58
:1060A0000F5F1F4FF8018491F4CF80E290E00E94CF
:1060B000059FEFECFDE084918F01882351F0082EBD
:1060C000000C990B0E94059F0F5F1F4FF8018491F0
:1060D000F4CF6091540470915504809156049091CE
:1060E00057040E944CE180E290E00E94059FEBEC97
:1060F000FDE084918F01882351F0082E000C990B4C
:106100000E94059F0F5F1F4FF8018491F4CF6091AB
:1061100058047091590480915A0490915B040E9434
:106120004CE180E290E00E94059FE7ECFDE0849165
:106130008F01882351F0082E000C990B0E94059FB7
:106140000F5F1F4FF8018491F4CF60915C04709150
:106150005D0480915E0490915F040E944CE180E2B6
:1061600090E026C68091A509882309F450C0E2EC8E
:10617000FDE084918F01882351F0082E000C990BCB
:106180000E94059F0F5F1F4FF8018491F4CF80910B
:10619000A609882359F18091710B882329F18091F8
:1061A0001B0C90911C0CA0911D0CB0911E0C009723
:1061B000A105B105C1F0BC01CD016D597F4F8F4FD5
:1061C0009F4F24E630E040E050E00E94B5F460913B
:1061D0001F0C7091200C8091210C9091220C0E9438
:1061E000B5F4822F01C080E090E0E6CEEEEBFDE05A
:1061F00084918F01882309F4E3CE082E000C990BBB
:106200000E94059F0F5F1F4FF8018491F3CFE6EBCB
:10621000FDE084918F01882309F4D2CE082E000C72
:10622000990B0E94059F0F5F1F4FF8018491F3CFD8
:10623000E1EBFDE084918F01882351F0082E000CE2
:10624000990B0E94059F0F5F1F4FF8018491F4CFB7
:106250008091B90D9091BA0DA091BB0DB091BC0D7C
:10626000892B8A2B8B2B09F477C00E9414A4A501DB
:1062700094010E94B5F469017A016091B90D7091A1
:10628000BA0D8091BB0D9091BC0DA50194010E94A7
:10629000B5F48601021B130BC8016CE370E00E9489
:1062A000E8F7CB019927EAE0F0E0BF010E94FCF794
:1062B000282FCB01BF010E94FCF7805D80934B0427
:1062C000205D20934C0410924D048BE494E00E94D6
:1062D0004BE180E290E00E94059FEFEAFDE08491AF
:1062E0007F01882359F0082E000C990B0E94059F0E
:1062F000FFEFEF1AFF0AF7018491F3CF80E290E0FD
:106300000E94059FC8016CE370E00E94E8F76AE014
:1063100070E00E94FCF7605D60934B04805D8093A9
:106320004C0410924D048BE494E00E944BE180E217
:1063300090E00E94059FEDEAFDE084918F018823A3
:1063400009F43ECE082E000C990B0E94059F0F5FAA
:106350001F4FF8018491F3CF80E290E00E94059FE7
:10636000E5EAFDE084918F01882309F429CE082E07
:10637000000C990B0E94059F0F5F1F4FF80184913D
:10638000F3CF1092E30D8091090180FF11C0E1EA83
:10639000FDE084918F01882309F412CE082E000CB1
:1063A000990B0E94059F0F5F1F4FF8018491F3CF57
:1063B00083E50E9479E0882341F00E94AAE00E94D0
:1063C0005CF67093B80D6093B70DEDE9FDE0849134
:1063D0008F01882351F0082E000C990B0E94059F15
:1063E0000F5F1F4FF8018491F4CF8DE090E00E9481
:1063F000059F8AE090E00E94059F8091010E88230E
:1064000009F4A1C28091B70D9091B80D8430910527
:1064100009F4D2C040F4892B09F03BC4E1ECFBE065
:1064200084918F010CC08830910509F47EC10C97CE
:1064300009F02FC4E9E3FAE084918F012FC2882389
:1064400051F0082E000C990B0E94059F0F5F1F4F03
:10645000F8018491F4CF8DE090E00E94059F8AE0DE
:1064600090E00E94059FE6EBFBE084918F0188237A
:1064700051F0082E000C990B0E94059F0F5F1F4FD3
:10648000F8018491F4CF8DE090E00E94059F8AE0AE
:1064900090E00E94059FEAEAFBE084918F01882347
:1064A00051F0082E000C990B0E94059F0F5F1F4FA3
:1064B000F8018491F4CF8DE090E00E94059F8AE07E
:1064C00090E00E94059FEEE9FBE084918F01882314
:1064D00051F0082E000C990B0E94059F0F5F1F4F73
:1064E000F8018491F4CF8DE090E00E94059F8AE04E
:1064F00090E00E94059FE0E9FBE084918F018823F2
:1065000051F0082E000C990B0E94059F0F5F1F4F42
:10651000F8018491F4CF8DE090E00E94059F8AE01D
:1065200090E00E94059FE2E8FBE084918F018823C0
:1065300051F0082E000C990B0E94059F0F5F1F4F12
:10654000F8018491F4CF8DE090E00E94059F8AE0ED
:1065500090E00E94059FE5E7FBE084918F0188238E
:1065600051F0082E000C990B0E94059F0F5F1F4FE2
:10657000F8018491F4CF8DE090E00E94059F8AE0BD
:1065800090E00E94059FE8E6FBE084918F0188235C
:1065900051F0082E000C990B0E94059F0F5F1F4FB2
:1065A000F8018491F4CF8DE090E00E94059F8AE08D
:1065B00090E00E94059F6DC3EAE5FBE084918F01A6
:1065C000882351F0082E000C990B0E94059F0F5F45
:1065D0001F4FF8018491F4CF8DE090E00E94059F59
:1065E0008AE090E00E94059FECE4FBE084918F013B
:1065F000882351F0082E000C990B0E94059F0F5F15
:106600001F4FF8018491F4CF8DE090E00E94059F28
:106610008AE090E00E94059FE6E3FBE084918F0111
:10662000882351F0082E000C990B0E94059F0F5FE4
:106630001F4FF8018491F4CF8DE090E00E94059FF8
:106640008AE090E00E94059FE0E2FBE084918F01E8
:10665000882351F0082E000C990B0E94059F0F5FB4
:106660001F4FF8018491F4CF8DE090E00E94059FC8
:106670008AE090E00E94059FEEE0FBE084918F01AC
:10668000882351F0082E000C990B0E94059F0F5F84
:106690001F4FF8018491F4CF8DE090E00E94059F98
:1066A0008AE090E00E94059FECEFFAE084918F0170
:1066B000882351F0082E000C990B0E94059F0F5F54
:1066C0001F4FF8018491F4CF8DE090E00E94059F68
:1066D0008AE090E00E94059FEEEEFAE084918F013F
:1066E000882351F0082E000C990B0E94059F0F5F24
:1066F0001F4FF8018491F4CF8DE090E00E94059F38
:106700008AE090E00E94059FE0EEFAE084918F011C
:10671000882309F448CF082E000C990B0E94059F8E
:106720000F5F1F4FF8018491F3CFE9EDFAE08491F8
:106730008F01882351F0082E000C990B0E94059FB1
:106740000F5F1F4FF8018491F4CF8DE090E00E941D
:10675000059F8AE090E00E94059FE2EDFAE08491B7
:106760008F01882351F0082E000C990B0E94059F81
:106770000F5F1F4FF8018491F4CF8DE090E00E94ED
:10678000059F8AE090E00E94059FEBEBFAE0849180
:106790008F01882351F0082E000C990B0E94059F51
:1067A0000F5F1F4FF8018491F4CF8DE090E00E94BD
:1067B000059F8AE090E00E94059FE4EAFAE0849158
:1067C0008F01882351F0082E000C990B0E94059F21
:1067D0000F5F1F4FF8018491F4CF8DE090E00E948D
:1067E000059F8AE090E00E94059FEDE8FAE0849121
:1067F0008F01882351F0082E000C990B0E94059FF1
:106800000F5F1F4FF8018491F4CF8DE090E00E945C
:10681000059F8AE090E00E94059FE6E7FAE08491F8
:106820008F01882351F0082E000C990B0E94059FC0
:106830000F5F1F4FF8018491F4CF8DE090E00E942C
:10684000059F8AE090E00E94059FE3E6FAE08491CC
:106850008F01882351F0082E000C990B0E94059F90
:106860000F5F1F4FF8018491F4CF8DE090E00E94FC
:10687000059F8AE090E00E94059FE0E5FAE08491A0
:106880008F01882309F48FCE082E000C990B0E94EB
:10689000059F0F5F1F4FF8018491F3CF882351F0BC
:1068A000082E000C990B0E94059F0F5F1F4FF801E7
:1068B0008491F4CF8DE090E00E94059F8AE090E003
:1068C0000E94059FE2E2FAE084918F01882351F053
:1068D000082E000C990B0E94059F0F5F1F4FF801B7
:1068E0008491F4CF8DE090E00E94059F8AE090E0D3
:1068F0000E94059FEAE0FAE084918F01882351F01D
:10690000082E000C990B0E94059F0F5F1F4FF80186
:106910008491F4CF8DE090E00E94059F8AE090E0A2
:106920000E94059FE2EFF9E084918F01882309F42A
:106930003ACE082E000C990B0E94059F0F5F1F4F47
:10694000F8018491F3CF8091A609882309F478C1D6
:1069500081E08093230C1092250C1092240C85EF7B
:1069600099E00E94C9A68BE1E5EFF9E0DE011596FA
:1069700001900D928A95E1F78091F3099091F409C5
:106980009C838B838DEE92E09A83898340E050E074
:10699000BE016F5F7F4F80E090E00E942CA1CE018E
:1069A00001960E94C2ADC090240CD090250C00919D
:1069B000B70D1091B80DC601801B910B049720F004
:1069C0006801F3E0CF0ED11C53EE452E59E0552E51
:1069D00064ED662E69E0762EC016D10608F459C122
:1069E0000115110509F09DC069EA79E085EF99E08C
:1069F0000E9491A562E273E089EA99E00E946EF834
:106A0000892B09F048C0F201849143EEE42E49E05D
:106A1000F42E882359F0082E000C990B0E94059F34
:106A2000FFEFEF1AFF0AF7018491F3CF8DE090E0BA
:106A30000E94059F8AE090E00E94059FF3018491E7
:106A400034EDE32E39E0F32E882359F0082E000CA4
:106A5000990B0E94059FFFEFEF1AFF0AF70184913F
:106A6000F3CF8DE090E00E94059F8AE090E00E94C5
:106A7000059F80E090E00E9445E1E4ECF9E084911C
:106A80007F012FEFE21AF20A882309F4D6C00E9490
:106A9000138EF701F4CFE0ECF9E084917F018823B5
:106AA00059F0082E000C990B0E94059FFFEFEF1A7A
:106AB000FF0AF7018491F3CF8DE090E00E94059FDB
:106AC0008AE090E00E94059FF10184912CEBE22E78
:106AD00029E0F22E882359F0082E000C990B0E9411
:106AE000059FFFEFEF1AFF0AF7018491F3CF8DE0C6
:106AF00090E00E94059F8AE090E00E94059F80E060
:106B000090E00E9445E1E7EBF9E084917F012FEFEF
:106B1000E21AF20A882309F490C00E94138EF7014A
:106B2000F4CF60E070E0C80101970E94F2A280916A
:106B3000A709882309F45AC0E5EBF9E084917F01A5
:106B4000882359F0082E000C990B0E94059FFFEF37
:106B5000EF1AFF0AF7018491F3CF89EA99E00E94C6
:106B60004BE18DE090E00E94059F8AE090E00E945A
:106B7000059FE3EBF9E084917F01882359F0082E0B
:106B8000000C990B0E94059FFFEFEF1AFF0AF70117
:106B90008491F3CF86EB99E00E944BE18DE090E089
:106BA0000E94059F8AE090E00E94059FC8010E9414
:106BB00045E1E1EBF9E084917F012FEFE21AF20A5F
:106BC000882321F00E94138EF701F5CF96EBE92E72
:106BD00099E0F92EF70181917F01882319F00E9435
:106BE000138EF8CF8AE00E94138E27C089EA99E0BD
:106BF0000E944BE18DE090E00E94059F8AE090E0CA
:106C00000E94059F86EB99E00E944BE18DE090E0A9
:106C10000E94059F8AE090E00E94059FC8010E94A3
:106C200045E186EBE82E89E0F82EF70181917F019E
:106C30008823C1F20E94138EF8CF0F5F1F4FCCCE76
:106C4000E2EAF9E084918F01882351F0082E000CCC
:106C5000990B0E94059F0F5F1F4FF8018491F4CF9D
:106C60008DE090E00E94059F8AE090E00E94059FE1
:106C7000E3E9F9E084918F01882309F494CC082E8C
:106C8000000C990B0E94059F0F5F1F4FF801849124
:106C9000F3CFE9E9FDE084918F01882309F490C9DD
:106CA000082E000C990B0E94059F0F5F1F4FF801E3
:106CB0008491F3CF8091A509882339F00E943EA0EA
:106CC00022C58091A5098823E9F00E948AB41BC5DA
:106CD0008091280C823019F0833609F014C50E9487
:106CE000F3E0E5E9FDE084918F01882309F468C9A8
:106CF000082E000C990B0E94059F0F5F1F4FF80193
:106D00008491F3CF8091280C833609F0FCC4DDCF49
:106D10008CE89DE00E94E5AD8091280C833609F453
:106D2000F2C40091B40D1091B50D7801F4E0EF0EAE
:106D3000F11C6AE270E0C7010E9463F8F801248147
:106D40002F3221F4B8016B5F7F4F03C02C3331F435
:106D5000B70183EE9DE00E9477F832C91092E30DEF
:106D6000009719F0FC01319710828091B40D909139
:106D7000B50D40E061E004960E94A7DE8091710BA2
:106D80008823C9F0E8E8FDE084918F01882351F061
:106D9000082E000C990B0E94059F0F5F1F4FF801F2
:106DA0008491F4CF8DE090E00E94059F8AE090E00E
:106DB0000E94059F05C9E4E8FDE084918F018823C6
:106DC00089F3082E000C990B0E94059F0F5F1F4F3F
:106DD000F8018491F4CF8091270990912809891BAB
:106DE0008F7009F090C48091280C823009F48BC414
:106DF000833609F488C48091710B8111B8C483C4AF
:106E000083E50E9479E0811126C083E40E9479E045
:106E1000882309F478C48091270990912809891B57
:106E20008F7009F070C420E030E040E251E46091DE
:106E30005C0470915D0480915E0490915F040E94F7
:106E400096F087FF08C089E79DE09093180780932C
:106E500017070E947B8E0E94AAE020E030E0A90183
:106E60000E9496F087FD10C00E94AAE020E030E862
:106E700049E853E40E9439F718164CF00E94AAE042
:106E80000E945CF6CB0105C080E090E002C083E187
:106E900091E00E948F5A37C483E50E9479E08823ED
:106EA00009F431C40E94AAE020E030E0A9010E9468
:106EB00096F087FD10C00E94AAE020E030E046E195
:106EC00053E40E9439F718164CF00E94AAE00E9481
:106ED0005CF6CB0105C080E090E002C086E990E05E
:106EE0000E94D14110C483E50E9479E08823D9F043
:106EF0000E94AAE020E030E04FE753E40E94FBF05C
:106F000020E030E048EC52E40E94EFF50E945CF68D
:106F10006F3F710519F010F06FEF70E0709365042A
:106F2000609364044DC88FEF90E090936504809364
:106F3000640446C88091270990912809891B8F70A5
:106F400009F03EC88091A50981113AC80E94EB64FE
:106F50005F9A809153048E7F809353048A9A479A54
:106F6000809153048D7F8093530480910801809514
:106F7000817080930601479A809153048B7F8093A0
:106F80005304129A1DC883E50E9479E0882319F101
:106F90000E94AAE020E030E040E252E40E9496F035
:106FA00087FD0FC00E94AAE020E030EC49E754E4DE
:106FB0000E9439F7181644F00E94AAE00E9457F682
:106FC00005C068E270E002C067EE73E070930302F0
:106FD0006093020298C3E3E7FDE084918F01882368
:106FE00051F0082E000C990B0E94059F0F5F1F4F58
:106FF000F8018491F4CFC0900202D09003020D2CCE
:10700000000CEE08FF08F7FE0DC06DE280E19FE086
:1070100004D666277727CB016C197D098E099F0955
:107020004AE003C04AE0C701B6010E94B3E00C94F5
:10703000E02F8091270990912809891B8F7009F012
:1070400062C38091280C823009F45DC3833609F055
:1070500028C359C38091270990912809891B8F70F3
:1070600011F00C94E02F8091280C823011F40C94D4
:10707000E02F833609F09DC30C94E02F80912709FF
:1070800090912809891B8F7009F03DC38091280CCD
:10709000823009F438C3833609F0E1C434C38091E7
:1070A000270990912809891B8F7009F02CC38091C2
:1070B000280C823009F427C3833609F006C523C3A0
:1070C0008091270990912809891B8F7009F01BC3B3
:1070D0008091280C823009F416C3833609F02BC541
:1070E00012C38091E30D811103C00E940A9FFEC16B
:1070F0008E3271F58091E40D8E3209F080C180915D
:10710000460B882309F4F2C181508093460B8823F3
:1071100061F090E001974FE1489F9001499F300D49
:107120001124C901805F954F02C082ED99E02BE1E7
:10713000FC013496A5EFB9E001900D922A95E1F794
:10714000FC01828193819093F4098093F309CEC16D
:107150008C3309F054C164E273E083EE9DE00E9439
:107160006EF8892B21F481E08093010EBFC163E3A7
:1071700073E083EE9DE00E946EF8892B79F4EFE6D0
:10718000F9E084918F010F5F1F4F882321F00E9447
:10719000138EF801F6CF82E599E0E4C06AE473E06B
:1071A00083EE9DE00E946EF8892B79F4EEE2F9E01F
:1071B00084918F010F5F1F4F882321F00E94138E4F
:1071C000F801F6CF8BE199E0CDC061E673E083EE84
:1071D0009DE00E946EF8892B79F4E0E0F9E084915B
:1071E0008F010F5F1F4F882321F00E94138EF8013B
:1071F000F6CF8BEF98E0B6C06FE673E083EE9DE0CC
:107200000E946EF8892B79F4EBEDF8E084918F0100
:107210000F5F1F4F882321F00E94138EF801F6CFD5
:1072200086ED98E09FC062E873E083EE9DE00E94E7
:107230006EF8892B79F4EBEBF8E084918F010F5F06
:107240001F4F882321F00E94138EF801F6CF82EBA6
:1072500098E088C060E973E083EE9DE00E946EF8DC
:10726000892B71F40FE818E0F8018491882329F044
:107270000F5F1F4F0E94138EF7CF88E898E072C00F
:1072800066EA73E083EE9DE00E946EF8892B79F444
:10729000E9E6F8E084918F010F5F1F4F882321F00A
:1072A0000E94138EF801F6CF82E698E05BC068EB8F
:1072B00073E083EE9DE00E946EF8892B79F4EAE496
:1072C000F8E084918F010F5F1F4F882321F00E9407
:1072D000138EF801F6CF89E398E044C063EC73E0C5
:1072E00083EE9DE00E946EF8892B79F4E0E2F8E0ED
:1072F00084918F010F5F1F4F882321F00E94138E0E
:10730000F801F6CF8EE098E02DC06FEC73E083EECD
:107310009DE00E946EF8892B79F4E3EFF7E0849109
:107320008F010F5F1F4F882321F00E94138EF801F9
:10733000F6CF81EE97E016C06DED73E083EE9DE031
:107340000E946EF8892BA9F4E7ECF7E084918F0195
:107350000F5F1F4F882321F00E94138EF801F6CF94
:1073600086EB97E090931807809317070E947B8E17
:10737000BDC06AEE73E083EE9DE00E946EF8892B3B
:10738000D9F4E2E9F7E084918F010F5F1F4F882362
:1073900021F00E94138EF801F6CF81E080932A0C31
:1073A00088E697E090931807809317070E947B8EDA
:1073B00083E08093280C9AC061E074E083EE9DE046
:1073C0000E946EF8892B79F4EDE6F7E084918F0145
:1073D0000F5F1F4F882321F00E94138EF801F6CF14
:1073E0000E9494E083C069E174E083EE9DE00E9416
:1073F0006EF8892B09F07AC01092010E77C01D82B9
:1074000018861C821B828DEE92E09A83898380917C
:10741000F809811103C062ED79E002C061EF79E003
:107420006115710519F06C5F7F4F02C060E070E07C
:1074300021E043EE5DE0CE0105960E94F6AA882386
:1074400061F18BE1FE013596A5EFB9E001900D9257
:107450008A95E1F72B813C813093F4092093F3095D
:107460008091460B8A3008F03DC091E0980F9093D0
:10747000460BFFE18F9FC0011124DC01AC5EB54FCC
:107480004BE1E5EFF9E001900D924A95E1F7FC013F
:10749000E05FF54F3383228325C0EBE7F3E284916D
:1074A0008F010F5F1F4F882321F00E94138EF80178
:1074B000F6CFE2E5F7E084918F010F5F1F4F88233D
:1074C00021F00E94138EF801F6CF03EE1DE0F801C3
:1074D00081918F01882319F00E94138EF8CF8AE0E2
:1074E0000E94138ECE0101960E94C2AD1092E30D50
:1074F0008091090180FF07C1E7EBFCE084918F01D7
:10750000882311F40C94E02F082E000C990B0E9494
:10751000059F0F5F1F4FF8018491F2CF8FE40E9407
:1075200079E081110C94E02F83E40E9479E00C94BF
:10753000E02F83E50E9479E0811159C08FE40E9419
:1075400079E0882319F08FE79CE007C084E50E946A
:1075500079E0882349F087E59CE0909318078093B1
:1075600017070E947B8E43C083E40E9479E0882342
:1075700019F08EE29CE0F1CF81E50E9479E088234A
:1075800019F086E09CE0E9CF88E40E9479E0882346
:10759000C9F0E2E0FCE084918F01882351F0082ECD
:1075A000000C990B0E94059F0F5F1F4FF8018491FB
:1075B000F4CF8DE090E00E94059F8AE090E00E9469
:1075C000059F15C08CE40E9479E0882381F0EEEFDE
:1075D000FBE084918F01882361F3082E000C990B46
:1075E0000E94059F0F5F1F4FF8018491F4CFE6ECD6
:1075F000FCE084918F01882311F40C94E02F082E75
:10760000000C990B0E94059F0F5F1F4FF80184919A
:10761000F2CF80912709809128090C94E02F83E50F
:107620000E9479E0882309F46EC086ED9BE0909378
:107630001807809317070E947B8EE6ECFCE084918C
:107640008F01882311F40C94E02F082E000C990B65
:107650000E94059F0F5F1F4FF8018491F2CFE1ED6B
:10766000FBE084918F01882351F0082E000C990BC8
:107670000E94059F0F5F1F4FF8018491F4CFECEC3F
:10768000FBE084918F01882311F40C94E02F082EE5
:10769000000C990B0E94059F0F5F1F4FF80184910A
:1076A000F2CF88E50E9479E0811106C089E50E9449
:1076B00079E0882309F46FC088E50E9479E0882387
:1076C00041F08DE69DE090931807809317070E9484
:1076D0007B8E89E50E9479E0882341F087E69DE072
:1076E00090931807809317070E947B8E8AE50E946B
:1076F00079E0882341F081E69DE09093180780931C
:1077000017070E947B8E8091AF0D9091B00D01966E
:1077100064E070E00E94FCF79093B00D8093AF0D91
:107720008091AB0D9091AC0D01969093AC0D809330
:10773000AB0D1092B30D1092B20D0C947A2E4091B5
:10774000AF0D5091B00D9F012F5F3F4F3093B30DA0
:107750002093B20D90E6949F9001959F300D1124D7
:10776000285D334FE20FF31F83830C947A2E0E941F
:10777000F3E0E0E8FDE084918F01882311F40C949C
:10778000E02F082E000C990B0E94059F0F5F1F4FE2
:10779000F8018491F2CF8AE50E9479E081118CCFC3
:1077A00083E40E9479E0882309F4ADCF8DE59DE064
:1077B000A4CF86E40E9479E0882309F44DC10E9499
:1077C000AAE00E945CF68B0189E59DE09093180782
:1077D000809317070E947B8E88E50E9479E08823BA
:1077E00009F451C00E94AAE02B013C012DEC3CECB5
:1077F0004CE45EE30E9496F09E012F5F3F4F7901BB
:10780000181674F020E030E0A901C301B2010E9413
:1078100039F718162CF41F930F938EE49DE005C1E1
:107820002DEC3CEC4CEC5DEBC301B2010E9496F0F8
:1078300018167CF020E030E040E85FEBC301B201B5
:107840000E9439F718162CF41F930F9382E49DE0E1
:10785000ECC01F930F93C301B2010E9457F67F93B0
:107860006F9388E39DE09F938F93FF92EF920E9426
:1078700068F00FB6F894DEBF0FBECDBFCE01019603
:107880000E94568EDFC089E50E9479E0882309F4C2
:1078900041C00E94AAE02B013C012DEC3CEC4CE4E1
:1078A0005EE30E9496F0FE0131967F01181674F097
:1078B00020E030E0A901C301B2010E9439F7181697
:1078C0002CF41F930F938DE29DE0AFC02DEC3CECA8
:1078D0004CEC5DEBC301B2010E9496F018167CF0EF
:1078E00020E030E040E85FEBC301B2010E9439F7CD
:1078F00018162CF41F930F9381E29DE096C01F93FE
:107900000F93C301B2010E9457F67F936F9387E1F3
:107910009DE0A9CF8AE50E9479E0882309F441C05F
:107920000E94AAE02B013C012DEC3CEC4CE45EE310
:107930000E9496F0FE0131967F01181674F020E047
:1079400030E0A901C301B2010E9439F718162CF4E6
:107950001F930F938CE09DE068C02DEC3CEC4CEC49
:107960005DEBC301B2010E9496F018167CF020E096
:1079700030E040E85FEBC301B2010E9439F718160E
:107980002CF41F930F9380E09DE04FC01F930F9343
:10799000C301B2010E9457F67F936F9386EF9CE07C
:1079A00062CF85E40E9479E0882309F44BC00E94ED
:1079B000AAE02B013C012DEC3CEC4CE45EE30E9480
:1079C00096F0FE0131967F01181674F020E030E049
:1079D000A901C301B2010E9439F718162CF41F93B4
:1079E0000F938BEE9CE021C02DEC3CEC4CEC5DEB5E
:1079F000C301B2010E9496F018167CF020E030E03E
:107A000040E85FEBC301B2010E9439F718162CF46D
:107A10001F930F938FED9CE008C0C301B2010E9439
:107A200057F67F936F9384ED9CE09F938F93FF9223
:107A3000EF920E9468F00F900F900F900F900F90B0
:107A40000F901CCF80ED9CE0909318078093170750
:107A50000E947B8E0C94E02F00E010E0B5CE20E079
:107A600030E040E251E460915C0470915D048091EB
:107A70005E0490915F040E9496F087FF08C089EC35
:107A80009CE090931807809317070E947B8E82E3F7
:107A900090E090936704809366040E94F75988EC05
:107AA00090E00E948F5AE6ECFCE084918F018823DD
:107AB00011F40C94E02F082E000C990B0E94059FE6
:107AC0000F5F1F4FF8018491F2CF20E030E040E2D9
:107AD00051E460915C0470915D0480915E0490912A
:107AE0005F040E9496F087FF08C08FEB9CE09093A4
:107AF0001807809317070E947B8E80E590E0909393
:107B00006704809366040E94F75980EF90E00E941A
:107B10008F5AE6ECFCE084918F01882311F40C94D9
:107B2000E02F082E000C990B0E94059F0F5F1F4F3E
:107B3000F8018491F2CF80E090E00E948F5A109279
:107B40006704109266040E94F759EBEBFCE0849105
:107B50008F01882311F40C94E02F082E000C990B50
:107B60000E94059F0F5F1F4FF8018491F2CF6F961F
:107B70000FB6F894DEBF0FBECDBFDF91CF911F913E
:107B80000F91FF90EF90DF90CF90BF90AF909F90BC
:107B90008F907F906F905F904F903F902F900895BF
:107BA000CF92DF92EF92FF92CF93DF936B017C0134
:107BB000EA0121E338E040EA50EC0E9439F787FD02
:107BC00023C022E430E047E553E4C701B6010E9438
:107BD00096F01816CCF0C880D980EA80FB802FE69A
:107BE00032E143E85AEBC701B6010E9439F787FD3D
:107BF0000BC0C1E022E430E047E553E4C701B60121
:107C00000E9496F018160CF4C0E08C2FDF91CF91F3
:107C1000FF90EF90DF90CF9008950F931F93CF9335
:107C2000DF93FC01A685B7858D0100581F4FE80141
:107C30008881998101968F779927AD014E575F4FC3
:107C4000EA012881398128173907D1F3E801288111
:107C50003981A20FB31F6C93A685B785A058BF4F7B
:107C600011969C938E93A689B7892C9181E090E020
:107C7000078C02C0880F991F0A94E2F7822B8C931D
:107C800081E081A30488F589E02D80818064808370
:107C900081E090E0DF91CF911F910F910895FC0159
:107CA00081A1882329F0A489B5898C9186FFFBCF17
:107CB00011A20895FC01A485B585FD01E058FF4F90
:107CC000208131813296808191812817390779F09E
:107CD00080819181A80FB91F8C91208131812F5F04
:107CE0003F4F2F7733273183208390E008958FEF24
:107CF0009FEF0895DC011C96ED91FC911D97DF012B
:107D0000A058BF4F2D913C91119712968D919C9147
:107D100011972817390739F08D919C91E80FF91FB9
:107D2000808190E008958FEF9FEF0895FC012485F6
:107D30003585F901E058FF4F80819181329620818D
:107D4000318180589F4F821B930B60E870E00C9448
:107D5000FCF70895089580E090E00895CF92DF92B7
:107D6000EF92FF92C0904202D0904302E090440212
:107D7000F0904502FC0180819181A281B3818093C2
:107D8000420290934302A0934402B09345020E94A2
:107D9000D8C7C0924202D0924302E0924402F092CD
:107DA0004502FF90EF90DF90CF900895809190066C
:107DB00090919106981759F0E92FF0E0E05FF94FA4
:107DC00080819F5F9F779093910690E008958FEF59
:107DD0009FEF08951F920F920FB60F9211240BB6CA
:107DE0000F920F931F932F933F934F935F936F9334
:107DF0007F938F939F93AF93BF93CF93DF93EF9333
:107E0000FF9300919106D091900611E01D0F1F770E
:107E1000C091C6009091F404492F092E000C550B17
:107E2000660B770B4C30510508F046C0FA018827E5
:107E3000EC56FF4F8F4F0C940FF8CD3441F0CE34F9
:107E4000B9F481E005C0CA3330F0CD3471F582E079
:107E50008093F40446C0C03308F043C0C03209F434
:107E600040C0CD3211F53DC0C13329F0C43329F0F3
:107E7000C032D9F436C083E0EBCF88E0E9CFC0331D
:107E800021F0C13391F486E0E3CF84E0E1CFC83341
:107E900061F485E0DDCFC23341F487E0D9CFC1334F
:107EA00021F489E0D5CFC03311F08BE0D1CF8AE047
:107EB000CFCFCA30B1F413C0CA3099F4973049F02B
:107EC0009A3059F0953059F41092520210921E19BE
:107ED00006C081E080936B0502C00E94EB641092A3
:107EE000F404011731F0ED2FF0E0E05FF94FC083AB
:107EF000D12FD0939006FF91EF91DF91CF91BF9159
:107F0000AF919F918F917F916F915F914F913F9131
:107F10002F911F910F910F900BBE0F900FBE0F90DE
:107F20001F9018958091920690919306009731F0DA
:107F30004AE050E060E070E00C94EAED60E070E050
:107F4000CB010895EFDF97FD0AC0ECDF6F3F7105AD
:107F50008105910509F02CF4E5DF862F089580E076
:107F600008958FEF08958091920690919306892B42
:107F700031F0E8DF91E0811103C090E001C091E0B1
:107F8000892F08950F931F93CF938091920690911C
:107F90009306009711F1FC018F01C1912C2F2F7DC9
:107FA000A9F0C53411F0C536B9F7F801108260E0C8
:107FB00070E080919206909193060E9497ECF801F0
:107FC000C083562F472F382F292F0BC060E070E059
:107FD000CF911F910F910C9497EC50E040E030E06E
:107FE00020E0652F742F832F922FCF911F910F9137
:107FF000089581548A3108F042C0E82FF0E04091A2
:10800000311250913212609133127091341204C0C7
:1080100076956795579547958A95D2F7842F817005
:1080200040FF2FC0E95EFD4E9081992309F1E09158
:108030003A11F0913B11E90FF11D908120ED290FCC
:108040002A3098F09E3211F491810CC09D3211F0CB
:108050009B3271F4918120ED290F2A3030F09E324D
:1080600039F4928190539A3018F42E2F9F2F02C02A
:1080700020E090E02093920690939306089580E08C
:1080800008950895B6DF882341F081E0209192069B
:1080900030919306232B09F480E0089580E1E4E514
:1080A000F4E0ADE8B1E101900D928A95E1F7089511
:1080B0002F923F924F925F926F927F928F929F92F8
:1080C000AF92BF92CF92DF92EF92FF920F931F93E6
:1080D000CF93DF9300D01F921F92CDB7DEB77C0104
:1080E0008B016A0119018090540490905504A0906E
:1080F0005604B0905704A5019401FC016081718180
:10810000828193810E9496F0F1E0FD83811112C07B
:10811000209158043091590440915A0450915B04C5
:10812000F80160817181828193810E9496F08111B2
:1081300001C01D82F60140805180628073802091D1
:108140000402309105024091060250910702C301DA
:10815000B2010E9496F0882309F453C040920402B1
:1081600050920502609206027092070220E030E011
:1081700040E450E46091EB057091EC058091ED05D1
:108180009091EE050E94EFF569837A838B839C833F
:1081900080928D1190928E11A0928F11B0929011B9
:1081A0008091580490915904A0915A04B0915B04B5
:1081B0008093911190939211A0939311B093941185
:1081C000F60180819181A281B38180939511909372
:1081D0009611A0939711B09398118091600490919B
:1081E0006104A0916204B09163048093991190930B
:1081F0009A11A0939B11B0939C11CE010196AEDD14
:108200004DDFFD81FF2309F16090E7057090E805DF
:108210008090E9059090EA05A090E305B090E40510
:10822000C090E505D090E6059501A601B301C40113
:108230000E9439F7181614F05301640120E030E071
:1082400040E251E4B501C6010CC020E030E040EC52
:108250005FE36091EF057091F0058091F1059091D9
:10826000F2050E94EFF569837A838B839C832091CA
:108270004404222349F0AB01BC0184E69EE00E9445
:10828000A5CE8AE00E94138EF70180819181A281A0
:10829000B38180938D1190938E11A0938F11B09321
:1082A0009011F80180819181A281B3818093911115
:1082B00090939211A0939311B0939411F1012081A6
:1082C0003181428153816091991170919A1180910D
:1082D0009B1190919C110E9413F5609399117093DA
:1082E0009A1180939B1190939C11CE01019636DDDB
:1082F000D5DE0F900F900F900F900F90DF91CF91E0
:108300001F910F91FF90EF90DF90CF90BF90AF90B3
:108310009F908F907F906F905F904F903F902F90A5
:10832000089580E1EDE8F1E1A4E5B4E001900D925B
:108330008A95E1F708959C0197FD0EC0843691055A
:1083400084F064E670E00E94FCF7CB016AE070E024
:108350000E94FCF7805D06C03195219531098DE2C0
:1083600001C080E280934F042A30310564F0EAE0D6
:10837000F0E0C901BF010E94FCF7CB01BF010E94E0
:10838000FCF7805D01C080E280935004C9016AE07F
:1083900070E00E94FCF7805D809351048FE494E0CC
:1083A00008958D3791051CF02DE780E002C0282F3D
:1083B000892F20936604809367040C94F7592F92B9
:1083C0003F924F925F926F927F928F929F92AF9265
:1083D000BF92CF92DF92EF92FF920F931F93CF93B2
:1083E000DF93CDB7DEB7C455D1090FB6F894DEBF21
:1083F0000FBECDBFE3E2F1E184918F010F5F1F4F0C
:10840000882321F00E94138EF801F6CF0E947DB7D9
:1084100081110C94C04B80E090E0A0E8BFE3809312
:10842000851190938611A0938711B093881180E0F5
:1084300090E0A0ECB0E48093891190938A11A0930E
:108440008B11B0938C118DEC9CECACE4BEE380936B
:10845000811190938211A0938311B093841180E0D5
:1084600090E0A8ECB1E48093F0049093F104A09321
:10847000F204B093F3048CE390E09093EF048093C4
:10848000EE0488EC90E09093ED048093EC0410925D
:10849000EB048FE4F7DD882311F074DD04C060E0A5
:1084A00070E080E190E46BAF7CAF8DAF9EAF83E472
:1084B000E9DD882311F057DD02C083E49ADD61967F
:1084C0008FAF61978BE4DEDD882311F04CDD02C0B5
:1084D0008BE48FDD60968FAF609782E4D3DD8823D5
:1084E000E9F050DD0E9457F67093EF046093EE04BC
:1084F0006115710599F0685271096536710570F062
:10850000EEEEF0E184918F010F5F1F4F882311F48D
:108510000C94C04B0E94138EF801F4CF8CE4B2DDB2
:10852000882351F12FDD6B017C01609381117093E1
:108530008211809383119093841120E030E0A9018F
:108540000E9439F787FD0AC020E030E040E050E4A7
:10855000C701B6010E9496F0181674F4E6ECF0E13B
:1085600084918F010F5F1F4F882311F40C94C04B2F
:108570000E94138EF801F4CF81E53BDD882309F4D6
:1085800040C08091920690919306892B19F4EBE9F3
:10859000F0E12BC0F7DC6B017C01609389117093D3
:1085A0008A1180938B1190938C112DEC3CEC4CE450
:1085B0005DE30E9439F787FD0AC020E030E040E724
:1085C00051E4C701B6010E9496F01816D4F4EAE609
:1085D000F0E184918F010F5F1F4F882311F40C94F9
:1085E000C04B0E94138EF801F4CF84918F010F5F6E
:1085F0001F4F882311F40C94C04B0E94138EF80176
:10860000F4CF83E53FDD882319F1BCDC4B015C012D
:108610002DEC3CEC4CEC5DE30E9439F787FD0AC081
:1086200020E030E040E85FE3C501B4010E9496F02D
:108630001816ACF4E3E4F0E184918F010F5F1F4F53
:10864000882311F40C94C04B0E94138EF801F4CFD0
:108650005DEC852E5CEC952EA92C5EE3B52E80E5B5
:10866000C8DC882309F443C0809192069091930658
:10867000892B71F4EBE0F0E184918F010F5F1F4FC4
:10868000882311F40C94C04B0E94138EF801F4CF90
:108690008091EB048F5F8093EB0474DC6B017C01B1
:1086A0006093F0047093F1048093F2049093F304C8
:1086B00020E030E0A9010E9439F787FD0AC020E0E0
:1086C00030E048EC51E4C701B6010E9496F018165C
:1086D00074F4E3EEFFE084918F010F5F1F4F882356
:1086E00011F40C94C04B0E94138EF801F4CF86E471
:1086F000C9DC882319F146DC6B017C0120E030E005
:1087000040E85FE30E9439F787FD0AC020E030E0CF
:1087100040E850E4C701B6010E9496F01816A4F490
:10872000EAEBFFE084918F010F5F1F4F882311F464
:108730000C94C04B0E94138EF801F4CFC12CD12CA5
:1087400040EEE42E4FE3F42EA7019601C701B601D7
:108750000E94FBF09B01AC0160E070E084E490E4D7
:108760000E94EFF52091851130918611409187117B
:10877000509188110E94FBF02B013C01A50194014E
:10878000C501B4010E94FBF0A70196010E94FBF015
:108790002CEE31E548EB5DE30E94EFF59B01AC0167
:1087A000C301B2010E94FBF06093851170938611A2
:1087B000809387119093881188E464DC8823C9F042
:1087C000E1DB0E9457F67093ED046093EC04655A68
:1087D00071096437710568F0ECE8FFE084918F015E
:1087E0000F5F1F4F882309F4CBC70E94138EF80137
:1087F000F5CF85E5FEDB8823E9F00E9414A461151E
:1088000071058105910511F00E948EEC8091920610
:1088100090919306892B11F0B5DB04C060E070E005
:1088200088E492E46093E7047093E8048093E90499
:108830009093EA0482E5DDDB81110DC0E8E5FFE0FD
:1088400084918F010F5F1F4F882309F499C70E94FD
:10885000138EF801F5CF8091920690919306892BA3
:10886000A9F060DB2F967FAF6EAF2F971616170615
:108870009CF0E4E2FFE084918F010F5F1F4F88239B
:1088800009F47EC70E94138EF801F5CF8AE190E0CB
:108890002F969FAF8EAF2F9788E5F4DB882361F08A
:1088A00071DB209138043091390440913A045091A1
:1088B0003B040E9412F508C0609154047091550465
:1088C00080915604909157046093E3047093E404FC
:1088D0008093E5049093E60489E5D4DB882361F076
:1088E00051DB20913C0430913D0440913E04509175
:1088F0003F040E9412F508C0609158047091590419
:1089000080915A0490915B046093DF047093E004BB
:108910008093E1049093E2046091E3047091E40495
:108920008091E5049091E6044FED54E039D981112E
:108930000DC0EAEFFEE084918F010F5F1F4F882387
:1089400009F41EC70E94138EF801F5CF84E451DBB1
:1089500091E089270E943B8420E030E040EA50E427
:1089600060915C0470915D0480915E0490915F045D
:108970000E9496F087FF14C0198A1A8A1B8A1C8AE3
:1089800080E090E0A0EAB0E489839A83AB83BC8363
:10899000BE016F5E7F4FCE0101960E949F85C1DCB4
:1089A0000E9414A46B017C01A8E8CA0EA3E1DA1EA0
:1089B000E11CF11C8091EE049091EF04F2DC6091D7
:1089C000EE047091EF04072E000C880B990B0E94A7
:1089D0009CF09B01AC0160916804709169048091E6
:1089E0006A0490916B040E9412F54B015C0120E037
:1089F00030E0A9010E9439F787FF04C0B7FAB094AC
:108A0000B7F8B09420E030E040E450E4C501B40190
:108A10000E9439F71816FCF40E9414A4DC01CB0163
:108A20008C199D09AE09BF09B7FD0FC00E9414A49F
:108A30006B017C01B8E8CB0EB3E1DB1EE11CF11C3D
:108A40000E943D598AE00E94138E80E00E942CAE65
:108A50000E944592B4CF8091EC049091ED040E9465
:108A60008F5A6091EC047091ED04072E000C880B76
:108A7000990B0E949CF09B01AC0160916E04709177
:108A80006F0480917004909171040E9412F54B0163
:108A90005C0120E030E0A9010E9439F787FF04C0A3
:108AA000B7FAB094B7F8B09420E030E040E450E476
:108AB000C501B4010E9439F71816FCF40E9414A4F1
:108AC000DC01CB018C199D09AE09BF09B7FD0FC0B0
:108AD0000E9414A46B017C01E8E8CE0EE3E1DE1EE7
:108AE000E11CF11C0E943D598AE00E94138E80E037
:108AF0000E942CAE0E944592B4CF10926004109256
:108B00006104109262041092630480E694E00E9473
:108B10001CB78091EB04882399F1C0DA2091991158
:108B200030919A1140919B1150919C116091F004E9
:108B30007091F1048091F2049091F3040E9413F576
:108B40006093991170939A1180939B1190939C114B
:108B500020E030E040E751E46091EF057091F005CE
:108B60008091F1059091F2050E94EFF569837A8377
:108B70008B839C83CE010196F1D890DA0E9429B5AF
:108B800080E2EFEBF4E0DF01282F1D922A95E9F750
:108B9000EFE9F4E0DF01282F1D922A95E9F7EFE7CE
:108BA000F4E0DF011D928A95E9F778DA809181116E
:108BB00090918211A0918311B091841180939511AD
:108BC00090939611A0939711B093981119821A82DD
:108BD0001B821C829E012F5F3F4F45E951E161E9F5
:108BE00071E18DE891E164DA9E01255C3F4F45E932
:108BF00051E161E971E18DE891E15ADA6196BFAD29
:108C00006197BB2329F068E574E084E594E004C033
:108C10006FED74E083EE94E00E94B7E23FAF2D96D3
:108C20002FAF2D972D96EFAD2D97E7FD82C4FFADA9
:108C3000F7FD7FC424E0E202F0011124EF58F64F63
:108C400040805180628073803FAD84E03802F00143
:108C50001124E35AF64FD080C180328023808D2DBD
:108C60009C2DA32DB22D8FAB98AFA9AFBAAFAE019B
:108C7000495C5F4FB201C3010E94D03D882309F4D3
:108C80005AC420E030E040EA50E4B201C3010E943F
:108C900013F5F62E072F182FE92E862F902FA12FD0
:108CA000BE2D8BAB9CABADABBEAB8D2D9C2DA32D48
:108CB000B22D8FA798ABA9ABBAAB2D969FAD2D97D0
:108CC000911152C0AFADA11105C05F2D402F312FC2
:108CD0002E2D04C0542D452D362D272D852F942F54
:108CE000A32FB22F8BAB9CABADABBEABBFADB43043
:108CF00034F4F42C052D162DE72CBB2369F020E06D
:108D000030E040EA50E46D2D7C2D832D922D0E94A1
:108D100012F5362F272F03C09601832D922D432F56
:108D2000522FBC014FA758AB69AB7AABEFADE43023
:108D30000CF0A7C020E030E040EA50E46D2D7C2D1F
:108D4000832D922D0E9413F521966FAF21972396C4
:108D50007FAF239725968FAF259727969FAF2797AD
:108D6000FFADF11185C099C02D962FAD2D97243000
:108D70000CF453C03FAD34305CF020E030E040EA0A
:108D800050E4B201C3010E9412F5362F272F03C011
:108D9000342D252DC301432F522FBC014BAB5CABAF
:108DA0006DAB7EAB8FAD8111E2C420E030E040EAD4
:108DB00050E4B201C3010E9412F5F62E072F182FBE
:108DC000E92E20E030E040EA50E46D2D7C2D832D2B
:108DD000922D0E9413F56FA778AB89AB9AAB9FAD2C
:108DE000992309F44EC020E030E040EA50E46D2DB4
:108DF0007C2D832D922D0E9412F521966FAF219725
:108E000023967FAF239725968FAF259727969FAF01
:108E10002797AFADA43064F140C0BFADB1110DC014
:108E200020E030E040EA50E4B201C3010E9412F5B4
:108E3000F62E072F182FE92E0FC0EFADE430B4F156
:108E400020E030E040EA50E4B201C3010E9412F594
:108E50006BAB7CAB8DAB9EAB2196DFAE219723969F
:108E6000CFAE239725963FAE259727962FAE27970F
:108E700032ED832E33E5932E3BE7A32E31E4B32E60
:108E800029C02196DFAE21972396CFAE2397259652
:108E90003FAE259727962FAE279722ED822E23E50A
:108EA000922E2BEFA22E20E4B22E14C02196DFAE1C
:108EB00021972396CFAE239725963FAE25972796E9
:108EC0002FAE279792ED892E93E5992E9BEFA92E31
:108ED00091E4B92E8BA99CA9ADA9BEA92C968CAF03
:108EE0009DAFAEAFBFAF2C979C01AD01B201C301E6
:108EF0000E9412F5698B7A8B8B8B9C8B4FA458A8A0
:108F000069A87AA8A30192016D2D7C2D832D922D45
:108F10000E9412F56D8B7E8B8F8B988F2C962CADCB
:108F20003DAD4EAD5FAD2C976091540470915504EA
:108F300080915604909157040E9412F52C966CAFC4
:108F40007DAF8EAF9FAF2C97A30192016091580423
:108F50007091590480915A0490915B040E9412F51B
:108F60002B013C018F2D902FA12FBE2D89839A8339
:108F7000AB83BC8321968FAD219723969FAD23971A
:108F80002596AFAD25972796BFAD27978D839E83F6
:108F9000AF83B8878091811190918211A091831144
:108FA000B091841189879A87AB87BC872DEC3CEC04
:108FB0004CEC5CE3C501B4010E94FBF020918511EB
:108FC0003091861140918711509188110E94FBF0D9
:108FD00020916004309161044091620450916304D7
:108FE0000E9413F56D877E878F87988B2C962CAD0A
:108FF0003DAD4EAD5FAD2C97CA01B9010E94FBF0AB
:109000006B017C01A3019201C301B2010E94FBF03C
:109010009B01AC01C701B6010E9413F520E030E0CE
:1090200040E050E40E9439F718160CF046C00E9448
:1090300029B51BA21CA21DA21EA220E030E040E028
:109040005FE360915C0470915D0480915E04909197
:109050005F040E9413F56F8F78A389A39AA39E01E2
:109060002D5D3F4FAE01415E5F4F68E574E084E5E2
:1090700094E01ED81BA21CA21DA21EA220E030E07C
:1090800040E05FE3609181117091821180918311C2
:10909000909184110E9413F56F8F78A389A39AA3EE
:1090A0009E012D5D3F4FAE01415E5F4FBE01615D90
:1090B0007F4FCE01C3960E9458401F8E18A219A25E
:1090C0001AA29E01215E3F4F41E851E1BE01615D60
:1090D0007F4FCE01C3960E9458400E9455B54090E4
:1090E0004202509043026090440270904502E0902A
:1090F000E705F090E8050091E9051091EA05A090D8
:10910000E305B090E405C090E505D090E605950133
:10911000A601B701C8010E9439F7181614F47501A9
:10912000860120E030E040E251E4B701C8010E942E
:10913000EFF5609342027093430280934402909350
:10914000450240E0BE016F5E7F4FCE0101960E9456
:10915000C6C340924202509243026092440270920F
:1091600045020E944E40A1E7B9E02496BFAFAEAFE2
:10917000249722961FAE1EAE229701E010E02196A2
:109180000FAC219702C0000F111F0A94E2F722963C
:10919000EEADFFAD229731962296FFAFEEAF22974C
:1091A00021E030E021960FAC219702C0220F331F3F
:1091B0000A94E2F763963FAF2EAF63978FE7282EAE
:1091C00084E0382E8FEB94E02A969FAF8EAF2A97DB
:1091D000AFE9B4E02896BFAFAEAF2897EDE5F9E070
:1091E0002696FFAFEEAF26972A962EAD3FAD2A9773
:1091F00065963FAF2EAF6597D9018D919C919C01EB
:1092000020233123232B09F4ADC06396EEADFFADCF
:1092100063978E239F23892B09F4A4C02896AEADB3
:10922000BFAD28978D919C9180239123892B09F0C4
:1092300099C020E030E040E050E42496AEADBFADF0
:1092400024976D917D918D919C910E9413F56B01F6
:109250007C0120E030E040E050E42496EEADFFAD2C
:10926000249764817581868197810E9412F54B0154
:109270005C0120E030E040E850ECC701B6010E94FC
:1092800096F087FD6EC120E030E046E553E4C7016B
:10929000B6010E9439F7181634F4C12CD12CB6E56A
:1092A000EB2EB3E4FB2ECBA6DCA6EDA6FEA62696FF
:1092B000AEADBFAD26974D905D906D907C9020E057
:1092C00030E040E85FE3C301B2010E9496F087FD01
:1092D0004FC120E030E046E553E4C301B2010E94F3
:1092E00039F7181634F4412C512CF6E56F2EF3E4BF
:1092F0007F2E4F8E58A269A27AA24FA258A669A6C5
:109300007AA620E030E040E850ECC501B4010E94AC
:1093100096F087FD34C120E030E046E553E4C50116
:10932000B4010E9439F7181634F4812C912C76E59B
:10933000A72E73E4B72E8BA29CA2ADA2BEA2AE0153
:10934000495D5F4FC701B6010E94D03D81111EC12A
:109350002896EEADFFAD289780819181802B912BCF
:10936000918380832A962EAD3FAD2A972E5F3F4F83
:109370002A963FAF2EAF2A976596AEADBFAD6597E3
:109380008D919C9180239123892B09F4A6C0F9012A
:109390008081918180239123892B09F49EC0F10162
:1093A0008081918180239123892B09F096C020E050
:1093B00030E040E050E42696AEADBFAD26976D910B
:1093C0007D918D919C910E9413F52B013C0120E031
:1093D00030E040E050E42696EEADFFAD2697648184
:1093E0007581868197810E9412F54B015C0124965C
:1093F000AEADBFAD2497CD90DD90ED90FC9020E018
:1094000030E040E850ECC701B6010E9496F087FDBD
:10941000FDC020E030E046E553E4C701B6010E94FC
:1094200039F7181634F4C12CD12C56E5E52E53E447
:10943000F52ECBA2DCA2EDA2FEA2CBA6DCA6EDA669
:10944000FEA620E030E040E85FE3C301B2010E94E5
:1094500096F087FDE2C020E030E046E553E4C3012A
:10946000B2010E9439F7181634F4412C512C36E51C
:10947000632E33E4732E4FA258A669A67AA620E085
:1094800030E040E85FE3C501B4010E9496F087FD3B
:10949000CBC020E030E046E553E4C501B4010E94B2
:1094A00039F7181634F4812C912C96E5A92E93E403
:1094B000B92E8F8E98A2A9A2BAA2AE01495D5F4FC4
:1094C000C701B6010E94D03D8111B5C0F101808174
:1094D0009181802B912B91838083F2E02F0E311CA0
:1094E00028962EAD3FAD28972E5F3F4F28963FAF71
:1094F0002EAF289726968EAD9FAD2697049626967A
:109500009FAF8EAF269799E8291694E0390609F0A7
:109510006BCE2496AEADBFAD249714962496BFAF04
:10952000AEAF24972296EEADFFAD2297359709F0A6
:1095300024CE0E9445922F962EAD3FAD2F972150FD
:1095400031092F963FAF2EAF2F97232B09F4B3C0CD
:109550002D963FAD2D9737FDAEC08FAD87FF4ECB1B
:10956000AAC0C12CD12CA0E8EA2EA0ECFA2E9BCEEA
:10957000412C512CE0E86E2EEFE37E2EBACE812CEA
:10958000912C60E8A62E60ECB62ED5CEAE01415EE1
:109590005F4FC501B4010E94D03D882309F4D8CEA5
:1095A00080914404882321F1B701A60184ED9EE057
:1095B0000E94A5CE4FA158A569A57AA58EEC9EE084
:1095C0000E94A5CE4BA15CA16DA17EA184EC9EE082
:1095D0000E94A5CE4F8D58A169A17AA18EEB9EE085
:1095E0000E94A5CE89E20E94138E8AE00E94138E0B
:1095F0009E01215E3F4FAE014D5D5F4FBE01695D33
:109600007F4FCE018B960E9485B5A2CEC12CD12C66
:1096100040E8E42E40ECF42E0CCF412C512C20E8F5
:10962000622E2FE3722E27CF812C912C80E8A82E5A
:109630008FE3B82E3ECFAE01415E5F4FC701B6014A
:109640000E94D03D882309F441CF809144048823AF
:1096500021F1B701A6018AE99EE00E94A5CE4FA1A3
:1096600058A569A57AA584E99EE00E94A5CE4BA1E4
:109670005CA16DA17EA18AE89EE00E94A5CE4F8DDF
:1096800058A169A17AA184E89EE00E94A5CE89E252
:109690000E94138E8AE00E94138E9E01215E3F4F2E
:1096A000AE014D5D5F4FBE01695D7F4FCE018B9670
:1096B0000E9485B50BCF0E9429B580E090E0A0EA1A
:1096C000B0E48093951190939611A0939711B09365
:1096D000981119821A821B821C829E012F5F3F4FB4
:1096E00045E951E161E971E18DE891E10E9458405D
:1096F0008091E3049091E404A091E504B091E60424
:1097000080938D1190938E11A0938F11B09390112F
:109710008091DF049091E004A091E104B091E20413
:109720008093911190939211A0939311B0939411FF
:1097300019821A821B821C829E012F5F3F4F45E9CE
:1097400051E161E971E18DE891E10E945840609634
:10975000FFAD6097F11114C0109267041092660477
:109760000E94F75980E090E00E948F5A09C02FAD07
:10977000F42C052D162DE72C24300CF034CB21CB06
:10978000CC5ADF4F0FB6F894DEBF0FBECDBFDF91CE
:10979000CF911F910F91FF90EF90DF90CF90BF90EE
:1097A000AF909F908F907F906F905F904F903F9081
:1097B0002F9008951F920F920FB60F9211240BB69F
:1097C0000F922F933F938F939F93EF93FF9320914B
:1097D000880E3091890E80918A0E90918B0E2817F9
:1097E000390731F4809131018F7D8093310114C0AC
:1097F000E0918A0EF0918B0EE85FF14F208180910D
:109800008A0E90918B0E01968F77992790938B0EED
:1098100080938A0E20933601FF91EF919F918F9153
:109820003F912F910F900BBE0F900FBE0F901F9086
:1098300018951F920F920FB60F9211240BB60F922C
:109840002F934F935F938F939F93EF93FF93809109
:10985000300182FD1CC02091360180910C0F909147
:109860000D0F40910E0F50910F0F01968F77992792
:109870004817590771F0E0910C0FF0910D0FE45764
:10988000F14F208390930D0F80930C0F02C08091B5
:109890003601FF91EF919F918F915F914F912F91A1
:1098A0000F900BBE0F900FBE0F901F9018952F9228
:1098B0003F924F925F926F927F928F929F92AF9260
:1098C000BF92CF92DF92EF92FF920F931F93CF93AD
:1098D000DF93CDB7DEB762970FB6F894DEBF0FBE49
:1098E000CDBFF8948FEF9FEF90938900809388000D
:1098F0002AE02A8B212C312C789480914705909175
:109900004805A0914905B0914A05892B8A2B8B2BDC
:1099100009F00FC2809127198823E1F010922719CE
:109920008091251990912619892B09F402C2109271
:10993000FF04109226191092251990912709809101
:109940002809981709F4F5C1809128098F5F8F7055
:10995000809328098091251990912619892B09F463
:10996000E8C14091430550914405609145057091CF
:10997000460580913F0590914005A0914105B09129
:1099800042050091360510E020E030E0841B950B85
:10999000A60BB70B081719072A073B0710F4D901C4
:1099A000C801E82F840F951FA61FB71F809343059A
:1099B00090934405A0934505B093460520918400FB
:1099C00030918500245E3F4F40911B0550911C054E
:1099D00060911D0570911E0580910B0590910C05FD
:1099E000A0910D05B0910E05840F951FA61FB71FFE
:1099F00080931B0590931C05A0931D05B0931E0535
:109A0000B7FD1CC0889A8091611190916211A0915C
:109A10006311B091641140910802042E000C550BA3
:109A2000660B770B840F951FA61FB71F80936111DC
:109A300090936211A0936311B093641140911F053C
:109A400050912005609121057091220580910F05AC
:109A500090911005A0911105B0911205840F951FEA
:109A6000A61FB71F80931F0590932005A093210583
:109A7000B0932205B7FD1CC08E9A8091651190911C
:109A80006611A0916711B091681140910902042EEE
:109A9000000C550B660B770B840F951FA61FB71F85
:109AA0008093651190936611A0936711B09368112C
:109AB000409123055091240560912505709126055C
:109AC0008091130590911405A0911505B09116058C
:109AD000840F951FA61FB71F80932305909324051D
:109AE000A0932505B0932605B7FD3FC08091F904EA
:109AF000F0910A028823C9F08091F70482FF02C026
:109B0000F7FD06C08091F604882311F40C94FE55ED
:109B10008091F7049091F80493FF02C0F7FD0CC008
:109B20008091F504811108C006C080910B018095D9
:109B3000887080930901419A4091691150916A118E
:109B400060916B1170916C118F2FFF0F990BAA0B05
:109B5000BB0B840F951FA61FB71F809369119093AD
:109B60006A11A0936B11B0936C114091270550912D
:109B700028056091290570912A058091170590911B
:109B80001805A0911905B0911A05840F951FA61FFD
:109B9000B71F8093270590932805A0932905B093BC
:109BA0002A05B7FD3AC040916D1150916E11609138
:109BB0006F1170917011C0900B020C2C000CDD081D
:109BC000EE08FF084C0D5D1D6E1D7F1D40936D114D
:109BD00050936E1160936F1170937011409107054F
:109BE000509108056091090570910A05841B950B39
:109BF000A60BB70B8093270590932805A093290502
:109C0000B0932A059091FA048091340593FF02C025
:109C1000815001C08F5F8093340580911B05909126
:109C20001C05A0911D05B0911E05B7FD15C0409102
:109C30000705509108056091090570910A05841B7C
:109C4000950BA60BB70B80931B0590931C05A09357
:109C50001D05B0931E05889880911F0590912005E1
:109C6000A0912105B0912205B7FD15C040910705CF
:109C7000509108056091090570910A05841B950BA8
:109C8000A60BB70B80931F0590932005A093210589
:109C9000B09322058E988091230590912405A09180
:109CA0002505B0912605B7FD3AC0409107055091B2
:109CB00008056091090570910A05841B950BA60B98
:109CC000B70B8093230590932405A0932505B093AB
:109CD00026058091F9048823E1F08091F70482FF42
:109CE00004C080910A0287FD05C08091F604882394
:109CF00009F48CC78091F7049091F80493FF04C095
:109D000080910A0287FD0BC08091F504811107C084
:109D100005C080910B018870809309014198E15042
:109D200041F0809184009091850082179307C8F3D9
:109D30004BCE8091150290911602A0911702B0911E
:109D40001802892B8A2B8B2B09F08AC0809135054C
:109D5000882309F453C08090430590904405A09057
:109D60004505B0904605C0903005D0903105E09093
:109D70003205F090330540913405C814D904EA0443
:109D8000FB0480F480910005909101052091040569
:109D9000309105052817390728F4415040933405C0
:109DA000019714C08C149D04AE04BF04E0F48091AC
:109DB000000590910105209102053091030582175D
:109DC000930788F44F5F4093340501969093010503
:109DD000809300054091110250911202609113028C
:109DE000709114020EC08FEF9FEFDC01809311027F
:109DF00090931202A0931302B09314024FEF5FEFFF
:109E0000BA018091340587FD02C0169801C0169AE8
:109E100080918400909185004C96209134052223F6
:109E2000B9F0149A2091340527FF02C02F5F01C0BA
:109E3000215020933405149820913405222369F38E
:109E4000209184003091850028173907C8F3E5CFA9
:109E500040931502509316026093170270931802F4
:109E60008091470590914805A0914905B0914A0518
:109E7000892B8A2B8B2B09F046C6A0912519B0910E
:109E80002619109711F40C94A857809043059090D0
:109E90004405A0904505B090460540913F0550917E
:109EA0004005609141057091420584169506A6060D
:109EB000B706D8F01092FF041092261910922519B7
:109EC0009091270980912809981711F40C94A857AC
:109ED000809128098F5F8F708093280940EDC42EF0
:109EE00047E0D42EE12CF12C1AC440913B0550914F
:109EF0003C0560913D0570913E05481559056A0580
:109F00007B0508F4AAC1409137055091380560914E
:109F1000390570913A05D6960D911D912D913C9180
:109F2000D997401751076207730708F077C14115A9
:109F300051056105710549F48090FB049090FC0483
:109F4000A090FD04B090FE0464C1E12CF980842E41
:109F5000952F862F0A811B81FD81EE813F81288507
:109F60009C80E0910A19E89D912CFF2730910B19F4
:109F7000389D900CF11D10900C19189CF00DE99F64
:109F8000900CF11D399FF00DE89FF00D092D1F2F4A
:109F9000099DE12D332722270F9FE00D311D2E1D36
:109FA000199DE00D311D2E1D1F9F300D211D032F0A
:109FB000122F099DF12C332722270F9FF00C311D02
:109FC0002E1D199DF00C311D2E1D1F9F300D211DC2
:109FD000032F122FEE278090FB049091FC048091B8
:109FE000FD0400907E040E2809F483C030917A04A9
:109FF000309FE1198E089E098E0920917B04209FD5
:10A00000E01981089E098E09F0907C04F09E80186A
:10A0100091098E09319FE01981089E098E09219FBF
:10A02000801891098E09F19E90198109099DF12CE2
:10A03000332722270F9FF00C311D2E1D199DF00C88
:10A04000311D2E1D1F9F300D211D032F122F30910A
:10A050007604309FE10D8E1C9E1D8E1D209177048D
:10A06000209FE00D811C9E1D8E1DF0907804F09EB7
:10A07000800C911D8E1D319FE00D811C9E1D8E1D3B
:10A08000219F800C911D8E1DF19E900D811D099DBB
:10A09000F12C332722270F9FF00C311D2E1D199D07
:10A0A000F00C311D2E1D1F9F300D211D032F122F6F
:10A0B00030917204309FE1198E089E098E0920911B
:10A0C0007304209FE01981089E098E09F0907404A2
:10A0D000F09E801891098E09319FE01981089E0930
:10A0E0008E09219F801891098E09F19E901981098E
:10A0F00082C030917A04309FE10D8E1C9E1D8E1D12
:10A1000020917B04209FE00D811C9E1D8E1DF090F0
:10A110007C04F09E800C911D8E1D319FE00D811CF2
:10A120009E1D8E1D219F800C911D8E1DF19E900DF8
:10A13000811D099DF12C332722270F9FF00C311D23
:10A140002E1D199DF00C311D2E1D1F9F300D211D40
:10A15000032F122F30917604309FE1198E089E094B
:10A160008E0920917704209FE01981089E098E09AD
:10A17000F0907804F09E801891098E09319FE019C3
:10A1800081089E098E09219F801891098E09F19EF0
:10A1900090198109099DF12C332722270F9FF00C7C
:10A1A000311D2E1D199DF00C311D2E1D1F9F300DD0
:10A1B000211D032F122F30917204309FE10D8E1C50
:10A1C0009E1D8E1D20917304209FE00D811C9E1DFD
:10A1D0008E1DF0907404F09E800C911D8E1D319F99
:10A1E000E00D811C9E1D8E1D219F800C911D8E1DDA
:10A1F000F19E900D811D11249C82F9820A831B839C
:10A20000FD83EE833F832887912C992AA12CB12CC2
:10A21000A82A80E599E121E0298B14C0D2968D907F
:10A220009D90AD90BC90D597F4CFB694A794979499
:10A230008794D988DD0CD98A049629E18C36920757
:10A2400009F4EAC4FC010591159125913491081592
:10A2500019052A053B0548F3DFC4409030055090AE
:10A2600031056090320570903305481459046A0432
:10A270007B0408F0C3C180912F05811121C0FD012D
:10A28000EE5BFF4FE080F1800281138178962081A0
:10A29000318142815381D2966D917D918D919C91B6
:10A2A000D5970E94D4CDDD24D394D0922F05E09190
:10A2B0002519F091261982A993A9A4A9B5A98EC13F
:10A2C00040912B0550912C0560912D0570912E0524
:10A2D000DA960D911D912D913C91DD974017510714
:10A2E0006207730708F073C14115510561057105D7
:10A2F00049F48091FB049091FC04A091FD04B0917D
:10A30000FE046CC1F0E0E985842F352F262FAA8545
:10A310007B856C855D85BE854F859889B0910A19CE
:10A32000B89F612D552740910B19489F600D511D15
:10A3300010900C19189E500DB39F600D511D439F36
:10A34000500DB29F500DA62F752FA69FB12D4427FB
:10A350009927A59FB00D411D9F1F769FB00D411DF0
:10A360009F1F759F400D911DA42F792FA69FE12D52
:10A3700044279927A59FE00D411D9F1F769FE00D63
:10A38000411D9F1F759F400D911DA42F792FBB2745
:10A390008091FB043091FC042091FD0400907E0428
:10A3A0000F2A09F483C040917A044A9FB1198F0B98
:10A3B0003F0B2F0B90917B049A9FB01981093F0BA3
:10A3C0002F0BE0917C04EA9F801931092F0B479FE6
:10A3D000B01981093F0B2F0B979F801931092F0B63
:10A3E000E79F30192109A69FE12D44279927A59FB2
:10A3F000E00D411D9F1F769FE00D411D9F1F759F22
:10A40000400D911DA42F792F409176044A9FB10DE4
:10A410008F1F3F1F2F1F909177049A9FB00D811DB2
:10A420003F1F2F1FE0917804EA9F800D311D2F1FE1
:10A43000479FB00D811D3F1F2F1F979F800D311D1E
:10A440002F1FE79F300D211DA69FE12D442799273F
:10A45000A59FE00D411D9F1F769FE00D411D9F1F91
:10A46000759F400D911DA42F792F409172044A9F32
:10A47000B1198F0B3F0B2F0B909173049A9FB0195A
:10A4800081093F0B2F0BE0917404EA9F8019310979
:10A490002F0B479FB01981093F0B2F0B979F8019F6
:10A4A00031092F0BE79F3019210982C040917A04AE
:10A4B0004A9FB10D8F1F3F1F2F1F90917B049A9FC2
:10A4C000B00D811D3F1F2F1FE0917C04EA9F800D7E
:10A4D000311D2F1F479FB00D811D3F1F2F1F979FBD
:10A4E000800D311D2F1FE79F300D211DA69FE12DEF
:10A4F00044279927A59FE00D411D9F1F769FE00DE2
:10A50000411D9F1F759F400D911DA42F792F4091D4
:10A5100076044A9FB1198F0B3F0B2F0B9091770454
:10A520009A9FB01981093F0B2F0BE0917804EA9FA5
:10A53000801931092F0B479FB01981093F0B2F0B51
:10A54000979F801931092F0BE79F30192109A69F8A
:10A55000E12D44279927A59FE00D411D9F1F769F60
:10A56000E00D411D9F1F759F400D911DA42F792F58
:10A57000409172044A9FB10D8F1F3F1F2F1F909172
:10A5800073049A9FB00D811D3F1F2F1FE09174042B
:10A59000EA9F800D311D2F1F479FB00D811D3F1F6A
:10A5A0002F1F979F800D311D2F1FE79F300D211DFD
:10A5B0001124E987AA877B876C875D87BE874F87D1
:10A5C000988B90E0932BA0E0B0E0A22B07C0A65A96
:10A5D000BF4F8D919D910D90BC91A02D20E539E14B
:10A5E00041E0498BF9014591559165917491481766
:10A5F00059076A077B0708F499C3A7C380913405FC
:10A600008823E1F0FD01E85BFF4F4081518160E06C
:10A6100070E000911102109112022091130230910A
:10A620001402401751076207730741F01092150298
:10A6300010921602109217021092180240910D0209
:10A6400050910E0260910F027091100277FF5FC06F
:10A65000AE5ABF4FCD90DD90ED90FC9080E599E132
:10A6600021E0FC0145915591659174914C155D0572
:10A670006E057F0550F4F694E794D794C794220FA3
:10A68000049679E18C36970761F72093360580E2CE
:10A69000C816D104E104F10428F470E2C72ED12CCD
:10A6A000E12CF12C90E2C91AD108E108F108C1149B
:10A6B000A8E0DA06E104F10408F403C4B4E0DB9E88
:10A6C000C0011124805B9A4EFC0132962591349191
:10A6D000EC2D6627E39FA001E29F410D561F0694D3
:10A6E000461F561F112460E070E0FC012591349153
:10A6F000C901A0E0B0E0841B950BA60BB70B8093BB
:10A700000D0290930E02A0930F02B0931002C0901E
:10A710000D02D0900E02E0900F02F0901002809196
:10A72000251990912619892B09F0E5C10E9453CE75
:10A730009093261980932519892B09F4DCC1E091A7
:10A740002519F0912619808183FF3EC0858996895D
:10A75000A789B08D8093611190936211A0936311CA
:10A76000B0936411818D928DA38DB48D809365110A
:10A7700090936611A0936711B0936811858D968DA3
:10A78000A78DB0A18093691190936A11A0936B116A
:10A79000B0936C1181A192A1A3A1B4A180936D117A
:10A7A00090936E11A0936F11B0937011909127093F
:10A7B00080912809981709F4B9CF809128098F5FF3
:10A7C0008F7080932809B2CFC588D688E788F08C2F
:10A7D00081E0C114D104E104F10409F480E0018DA9
:10A7E000128D238D348D011511052105310509F0D8
:10A7F0008260458D568D678D70A1411551056105AB
:10A80000710509F084608093FF0410922B0510926B
:10A810002C0510922D0510922E05109237051092DE
:10A8200038051092390510923A0585A196A1A7A185
:10A83000B0A580933F0590934005A0934105B09348
:10A840004205882499245401881A990AAA0ABB0A45
:10A850008092270590922805A0922905B0922A059A
:10A860008092230590922405A0922505B09226059A
:10A8700080921F0590922005A0922105B09222059A
:10A8800080921B0590921C05A0921D05B0921E059A
:10A89000CC0CDD1CEE1CFF1CC0920B05D0920C05ED
:10A8A000E0920D05F0920E05000F111F221F331FBD
:10A8B00000930F0510931005209311053093120596
:10A8C000440F551F661F771F4093130550931405BF
:10A8D000609315057093160541A152A163A174A15F
:10A8E000440F551F661F771F409317055093180597
:10A8F0006093190570931A05880F991FAA1FBB1F33
:10A900008093070590930805A0930905B0930A0565
:10A910001092430510924405109245051092460589
:10A9200082A593A5A4A5B5A580933B0590933C056E
:10A93000A0933D05B0933E0586A597A5A0A9B1A912
:10A940008093300590933105A0933205B093330581
:10A9500081A580930605DF01A95BBF4F9C91909371
:10A960003505992339F115962D913C911197309326
:10A9700005052093040512972D913C911197309372
:10A9800003052093020510921502109216021092F0
:10A9900017021092180212972D913C91A90160E0C4
:10A9A00070E040931102509312026093130270936F
:10A9B00014020CC088248A94982C540180921102AD
:10A9C00090921202A0921302B0921402EA5BFF4F1F
:10A9D00090812091FA0492130AC020910C0230E079
:10A9E000482F082E000C550B4217530731F0909357
:10A9F000FA0480930C020E9426CE0E94E1C22FEF3F
:10AA00003FEFA90120930D0230930E0240930F02F5
:10AA100050931002E0912519F0912619DF01DE967E
:10AA2000ED90FD900D911C9122A933A944A955A93F
:10AA3000EA5AFF4F60817181828193810E94D4CD57
:10AA400010922F05E0912519F0912619EA5AFF4F2F
:10AA500080809180A280B38080E599E121E0FC01B3
:10AA60004591559165917491481559056A057B0585
:10AA700058F4B694A79497948794220F0496ACE662
:10AA8000B9E1A817B90759F72093360590E289165E
:10AA90009104A104B10428F4B0E28B2E912CA12CD6
:10AAA000B12C30E2831A9108A108B108811448E062
:10AAB0009406A104B10408F428C254E0959EC00194
:10AAC0001124805B9A4EFC01329625913491782DA9
:10AAD0006627739FA001729F410D561F0694461F63
:10AAE000561F1124FC01C590D490E12CF12CC41AFE
:10AAF000D50AE108F108C0924705D0924805E092D6
:10AB00004905F0924A0500914705109148052091AA
:10AB1000490530914A054091150250911602609105
:10AB2000170270911802F02E198BF22FE32F4017A5
:10AB300051076207730720F4F42E598BF62FE72F85
:10AB40008F2D9989AF2FBE2F0097E1E0AE07B10599
:10AB500020F08FEF9FEFA0E0B0E0081B190B2A0B4D
:10AB60003B0B00934705109348052093490530930C
:10AB70004A054F3FFFEF5F076F077F0761F0481BF4
:10AB8000590B6A0B7B0B409315025093160260938E
:10AB9000170270931802F894209184003091850078
:10ABA000205F3F4F4A8941504A8B442341F0280E91
:10ABB000391E2216330610F40C947C4C01C0190186
:10ABC0003092890020928800789462960FB6F894AB
:10ABD000DEBF0FBECDBFDF91CF911F910F91FF90D0
:10ABE000EF90DF90CF90BF90AF909F908F907F902D
:10ABF0006F905F904F903F902F90089580910B0140
:10AC000080958870809309010C94884D80910B0188
:10AC10008870809309016EC839893093360580E2C7
:10AC200088169104A104B10428F430E2832E912CFB
:10AC3000A12CB12C30E2831A9108A108B10881142B
:10AC400088E09806A104B10420F1E4E09E9EC001D2
:10AC50001124805B9A4EFC01329625913491F82D97
:10AC6000EE27F39F7001F29FE10CFE1E0694EE1E8C
:10AC7000FE1E1124FC01C590D490860120E030E036
:10AC8000480159018E189F08A108B1087501640197
:10AC900022C0950184013695279517950795F801EF
:10ACA000EC7FCF01805B9E4EFC01C590D490FC01EF
:10ACB000329625913491E82DE770E29FC001E39F21
:10ACC000900D112423E0969587952A95E1F7C81AEF
:10ACD000D90AE12CF12C4C0D5D1D6E1D7F1D40939A
:10ACE0003705509338056093390570933A05909174
:10ACF000350580913405992309F474C0882309F43B
:10AD00000ECDA85BBF4F8D919C91A0E0B0E040912B
:10AD10001102509112026091130270911402841773
:10AD20009507A607B70709F060C0F9CCB695A795B7
:10AD300097958795D988DD0CD98A2C5F3F4F4CE6D3
:10AD400059E14217530709F04DCC59895093360504
:10AD500080329105A105B10520F480E290E0A0E0E9
:10AD6000B0E08097A109B109811558E09507A105C8
:10AD7000B10508F443C074E0979F90011124205B53
:10AD80003A4EF901329645915491EE27859FB001D4
:10AD9000849F610D7E1F06946E1F7E1F1124F90192
:10ADA000C590D490E12CF12CC61AD70AE108F1081D
:10ADB00080912B0590912C05A0912D05B0912E0529
:10ADC0008C0D9D1DAE1DBF1D80932B0590932C05F2
:10ADD000A0932D05B0932E0580913505811130C0CB
:10ADE00080913405882309F49ACC109215021092B0
:10ADF0001602109217021092180291CCAC01BD01FC
:10AE00007695679557954795FA01EC7F9F01205BF2
:10AE10003E4EF901C590D490F90132964591549176
:10AE20008770849F9001859F300D1124F3E0369543
:10AE30002795FA95E1F7C21AD30AE12CF12CB8CF85
:10AE40008989480E511C611C711C809125199091B3
:10AE50002619481459046A047B04D8F42091340557
:10AE6000222309F45CCCFC01E85BFF4F2081318197
:10AE7000A90160E070E0009111021091120220918E
:10AE8000130230911402401751076207730709F447
:10AE900046CC1092150210921602109217021092D0
:10AEA0001802FC01E85BFF4F80819181A0E0B0E0D7
:10AEB0008093110290931202A0931302B093140294
:10AEC0002ECCD701C601B695A79597958795FC011D
:10AED000EC7FCF01805B9E4EFC0125913491FC01FB
:10AEE0003296459154916C2D6770649FC001659FA7
:10AEF000900D112463E0969587956A95E1F7281BDC
:10AF0000390BC901A0E0B0E0FACBD501C401B69578
:10AF1000A79597958795FC01EC7FCF01805B9E4EAE
:10AF2000FC01C590D490FC01329625913491482DB6
:10AF30004770429FC001439F900D1124A3E0969556
:10AF40008795AA95E1F7C81AD90AE12CF12CD3CD3F
:10AF500080EDC82E87E0D82EE12CF12CE7CBCF92E4
:10AF6000DF92EF92FF920F931F93CF93DF936C01C9
:10AF70007A018B01C0E0D0E0CE15DF0581F0D80169
:10AF80006D918D01D601ED91FC910190F081E02D44
:10AF9000C6011995892B11F02196EECF7E01C701CC
:10AFA000DF91CF911F910F91FF90EF90DF90CF90A5
:10AFB0000895FF920F931F93CF93DF938C01EB01C2
:10AFC000F42E80E20E94138E8FEFF81611F084E5C4
:10AFD00001C082E40E94138E8AE30E94138EF8015E
:10AFE000608171818281938142E00E94D491488185
:10AFF00059816A817B8184E19CE10E94A5CE62E057
:10B0000070E080E090E0DF91CF911F910F91FF9071
:10B010000C9424BA1F920F920FB60F9211240BB604
:10B020000F922F933F934F935F936F937F938F93E1
:10B030009F93AF93BF93EF93FF9380917605909189
:10B040007705A0917805B0917905892B8A2B8B2BF8
:10B0500059F190917505E0917305F0917405808127
:10B06000892780838091760590917705A091780556
:10B07000B0917905181619061A061B060CF056C071
:10B080008091760590917705A0917805B09179052A
:10B090000197A109B1098093760590937705A09354
:10B0A0007805B093790542C080911D02E0E2FCE191
:10B0B000E4919FEF90931D02E230C9F050F4EE232B
:10B0C00099F0E13081F590916F009D7F90936F0032
:10B0D0002AC0E43019F1E0F0E53029F590917300D1
:10B0E0009D7F909373001FC010926E001CC09091C2
:10B0F00070009D7F9093700091E09093B0009091CC
:10B10000B100987F94609093B1001092B3000BC08F
:10B11000909171009D7F9093710005C09091720095
:10B120009D7F9093720060E00E94F3B8FF91EF91D1
:10B13000BF91AF919F918F917F916F915F914F914F
:10B140003F912F910F900BBE0F900FBE0F901F904D
:10B1500018958F929F92AF92BF92CF92DF92EF920B
:10B16000FF920F931F93CF93DF93F0E2FF2EE12C1A
:10B17000AE2DB0E0BD016F0D711D759567956E1513
:10B1800011F0F6120BC0EEEEF9E165917491072E05
:10B19000000C880B990B0E949CF062C09B0121500F
:10B1A0003109220F331F220F331FF901E059F64EE8
:10B1B00005911491AB01440F551F440F551FFA011F
:10B1C000E059F64EC591D4918017910714F4F62EEC
:10B1D000D1CFC817D90714F4E62ECACFF901EE581B
:10B1E000F64EE590F490FA01EE58F64EC590D490E4
:10B1F000BC01601B710B072E000C880B990B0E9481
:10B200009CF04B015C01B6016E197F09072E000C02
:10B21000880B990B0E949CF09B01AC01C501B40105
:10B220000E94FBF04B015C01C01BD10BBE01DD0F86
:10B23000880B990B0E949CF09B01AC01C501B401E5
:10B240000E94EFF54B015C01B701FF0C880B990BD5
:10B250000E949CF09B01AC01C501B4010E9413F552
:10B26000DF91CF911F910F91FF90EF90DF90CF90E2
:10B27000BF90AF909F908F9008950F931F93CF939F
:10B28000DF93CDB7DEB728970FB6F894DEBF0FBEB9
:10B29000CDBF60916C0470916D04072E000C880B7B
:10B2A000990B0E949CF06D837E838F839887809199
:10B2B0006E0490916F04A0917004B0917104898321
:10B2C0009A83AB83BC834DEFBE016B5F7F4FCE0192
:10B2D00001966FDE6091660470916704072E000C82
:10B2E000880B990B0E949CF06D837E838F839887D7
:10B2F0008091680490916904A0916A04B0916B04F4
:10B3000089839A83AB83BC834FEFBE016B5F7F4F12
:10B31000CE0101964EDEECE1FCE184918F010F5FDE
:10B320001F4F882321F00E94138EF801F6CFE09181
:10B330007205F0E0E059FA4F608170E080E090E043
:10B340000E94BA91E7E1FCE184918F010F5F1F4FEA
:10B35000882321F00E94138EF801F6CF60917105C9
:10B3600070E080E090E00E94BA9128960FB6F894C1
:10B37000DEBF0FBECDBFDF91CF911F910F9108951A
:10B380000F930FB70F9300916E000B7F00936E0029
:10B3900078940F930BB70F930CB70F921F922F93C4
:10B3A0003F934F935F936F937F938F939F93AF934D
:10B3B000BF93EF93FF931124F0D1FF91EF91BF91D1
:10B3C000AF919F918F917F916F915F914F913F913D
:10B3D0002F911F900F900CBF0F910BBF0F91046026
:10B3E000F89400936E000F910FBF0F911895CF92B4
:10B3F000DF92EF92FF92C0906804D0906904E090D1
:10B400006A04F0906B046091660470916704665062
:10B410007109072E000C880B990B0E949CF09B0170
:10B42000AC01C701B6010E9496F087FF1FC020E063
:10B4300030E040E050E4C701B6010E9413F50E94DD
:10B440005CF67093A9056093A8050E9414A4DC0122
:10B45000CB01805A9541AF4FBF4F8093A405909385
:10B46000A505A093A605B093A70508C01092A40552
:10B470001092A5051092A6051092A705FF90EF90D7
:10B48000DF90CF900895CF92DF92EF92FF92C0901D
:10B490006E04D0906F04E0907004F090710460919D
:10B4A0006C0470916D0467507109072E000C880BB5
:10B4B000990B0E949CF09B01AC01C701B6010E9450
:10B4C00096F087FF1FC020E030E040E450E4C70161
:10B4D000B6010E9413F50E945CF67093A305609379
:10B4E000A2050E9414A4DC01CB01805A9541AF4F04
:10B4F000BF4F80939E0590939F05A093A005B093A6
:10B50000A10508C010929E0510929F051092A005FB
:10B510001092A105FF90EF90DF90CF9008952091B9
:10B520002602309127022A503109821793070CF422
:10B530009C0130936D0420936C0480E0A4CF1092A2
:10B540006C0580E090E0EBDF1092670410926604D7
:10B550004EDF0E943DCF80E090E0E1DF1092700569
:10B560002C981092670410926604109271058091D5
:10B57000020180728093000108958F929F92AF9292
:10B58000BF92CF92DF92EF92FF920F931F93CF93D0
:10B59000DF93F0E4FF2EE12CAE2DB0E0BD016F0D86
:10B5A000711D759567956E1511F0F6120BC0E9E6E1
:10B5B000FBE165917491072E000C880B990B0E949A
:10B5C0009CF062C09B0121503109220F331F220FD2
:10B5D000331FF901E559F54E05911491AB01440F64
:10B5E000551F440F551FFA01E559F54EC591D491E9
:10B5F0008017910714F4F62ED1CFC817D90714F489
:10B60000E62ECACFF901E359F54EE590F490FA0120
:10B61000E359F54EC590D490BC01601B710B072E09
:10B62000000C880B990B0E949CF04B015C01B60149
:10B630006E197F09072E000C880B990B0E949CF055
:10B640009B01AC01C501B4010E94FBF04B015C0100
:10B65000C01BD10BBE01DD0F880B990B0E949CF023
:10B660009B01AC01C501B4010E94EFF54B015C01E7
:10B67000B701FF0C880B990B0E949CF09B01AC0159
:10B68000C501B4010E9413F5DF91CF911F910F9175
:10B69000FF90EF90DF90CF90BF90AF909F908F90F2
:10B6A000089560E08091B5059091B60552DD6093F4
:10B6B0006E0470936F048093700490937104809172
:10B6C000B3059091B40559DF6093680470936904E1
:10B6D00080936A0490936B04A89510926D05089569
:10B6E000DF92EF92FF920F931F93CF93DF93F82E89
:10B6F000D62EE72E8A0180911902882309F439C0D9
:10B70000E6E6F3E28491EF012196882321F00E947E
:10B71000138EFE01F7CFED2DFE2D8491EF012196C2
:10B72000882321F00E94138EFE01F7CFE1E0FAE1B9
:10B730008491EF012196882321F00E94138EFE014F
:10B74000F7CFF7FC0BC06F2DFF0C770B880B990B15
:10B750000E94BA918AE00E94138E0BC0ECEFF9E1CF
:10B760008491EF012196882321F00E94138EFE011F
:10B77000F7CF80917A05811108C01092190281E0FB
:10B7800080937A05C8010E94E5ADDF91CF911F91AA
:10B790000F91FF90EF90DF90D2CE0F931F93CF9336
:10B7A000DF9380911C028F37A0F08F579091700526
:10B7B0009093C605992311F02C9A01C02C982091E2
:10B7C00071052093C50590910201222369F090959F
:10B7D0000BC09091C605891708F02C989091C5056B
:10B7E000891728F0909102019072909300018F5F69
:10B7F00080931C029091C40581E089278093C40541
:10B8000080911B0285301CF4C1E0C80F01C0C0E06C
:10B81000823009F4B8C054F4882301F1813009F072
:10B82000E7C088E080937B0085E4C4C0843009F4DD
:10B83000C9C00CF4BBC0853009F0DAC09091C305D3
:10B84000911102C08093C3058091C30581508093FC
:10B85000C305882309F4CCC0C5E0CAC080911A0290
:10B860008F5F80311CF480931A02C2C010921A02BA
:10B8700080916D05811113C08091B9059091BA0531
:10B880009093B6058093B5058091B7059091B80562
:10B890009093B4058093B30581E080936D058AE0B1
:10B8A000E9EBF5E0DF011D928A95E9F71092B80502
:10B8B0001092B7050091B5051091B6051195019547
:10B8C000110980916C0490916D04D1E0181619064D
:10B8D0002CF080917005811101C0D0E08091370F6C
:10B8E0009091380F9195819591098017910734F4C3
:10B8F00042EA5BE163EC7BE180E0F2DE80912402CE
:10B90000909125029195819591090817190744F4A2
:10B91000DD2331F045ED5BE166EF7BE180E0E0DEC9
:10B92000809166049091670411E0181619062CF0B6
:10B9300080917105811101C010E02091B305309113
:10B94000B4058091350F9091360F8217930734F02C
:10B9500042EB5BE163EC7BE18FEFC2DE20912202E0
:10B96000309123028091B3059091B405821793071B
:10B970000CF43EC01123E1F145EE5BE166EF7BE1A3
:10B980008FEFAEDE35C080917A0086FD2EC08091AB
:10B990007800909179002091B9053091BA05820F15
:10B9A000931F9093BA058093B90522C088E08093D5
:10B9B0007B0086E480937C0080917A008064809391
:10B9C0007A0016C080917A0086FD11C080917800BF
:10B9D000909179002091B7053091B805820F931F9F
:10B9E0009093B8058093B70503C0C2E001C0C4E0DE
:10B9F000C0931B020E94E1C280916E0590916F0579
:10BA0000009799F0019790936F0580936E05892BAD
:10BA100061F488E09CE19093180780931707DF9109
:10BA2000CF911F910F910C947B8EDF91CF911F913D
:10BA30000F9108952F923F924F925F926F927F9253
:10BA40008F929F92AF92BF92CF92DF92EF92FF922E
:10BA50000F931F93CF93DF9300D01F92CDB7DEB724
:10BA60005C017A8369831A0107FD0DC0802F002EC7
:10BA7000000C990B9C838B83FC01EE5AFE4E808157
:10BA80008823E1F008C08091B205882399F0E1E0B5
:10BA9000F0E0FC83EB83F5011082EB81FC81EE0F7B
:10BAA000FF1FEE0FFF1FE655FA4F10821182128220
:10BAB000138230C081E090E09C838B83F901408049
:10BAC0005180628073808B819C81880F991F880FC1
:10BAD000991F9C0126553A4F4901A3019201F40197
:10BAE00060817181828193810E9496F0882391F018
:10BAF000F401408251826282738211E020E030E0E2
:10BB0000A901C301B2010E9439F718160CF010E028
:10BB1000F5011083F50180818230F1F0833009F462
:10BB200066C0813009F084C0EB81FC81EE0FFF1FFD
:10BB3000EE0FFF1FE655FA4F20813181428153817C
:10BB4000F10160817181828193810E9496F087FD6D
:10BB50006FC082E0F50180832B813C81220F331F6F
:10BB6000220F331F26553A4F3C832B83B60180E0CA
:10BB700090E00E949AF09B01AC01EB81FC81608116
:10BB80007181828193810E9412F59B01AC01F101C8
:10BB900060817181828193810E9439F787FD14C091
:10BBA0000E9414A44B015C019701A8EEB3E00E942F
:10BBB00003F5860E971EA81EB91EE981FA818082C0
:10BBC0009182A282B38234C00E9414A4E981FA81D6
:10BBD000C080D180E280F380DC01CB018C199D090B
:10BBE000AE09BF09B7FD24C083E0F50180830F3F94
:10BBF00019F04BE65BE102C04EE75BE162E97BE1F5
:10BC0000802F0F900F900F900F90DF91CF911F9189
:10BC10000F91FF90EF90DF90CF90BF90AF909F90EB
:10BC20008F907F906F905F904F903F902F9058CD66
:10BC30000F900F900F900F90DF91CF911F910F9168
:10BC4000FF90EF90DF90CF90BF90AF909F908F903C
:10BC50007F906F905F904F903F902F9008957F92CC
:10BC60008F929F92AF92BF92CF92DF92EF92FF920C
:10BC70000F931F93CF93DF9320E030E048E452E42A
:10BC800060916E0470916F048091700490917104C2
:10BC90000E9439F718164CF4E6EFF9E1E491C1E09F
:10BCA00001C0CC0FEA95EAF701C0C0E080EFE82EB2
:10BCB00089E1F82E06EF19E196E0A92E912CD0E04B
:10BCC000CC24C394D12CF7017490F801849077FCB4
:10BCD00023C0892D90E0082C02C0959587950A9481
:10BCE000E2F780FD19C0BE01082C02C0759567956A
:10BCF0000A94E2F76170B62EB1946B2D872D0E94E5
:10BD0000F3B86B2D70E0872D0E945DB9C60101C0AC
:10BD1000880F8A94EAF7982AAA94FFEFEF1AFF0A8D
:10BD20000F5F1F4FA110CFCFDF91CF911F910F91C8
:10BD3000FF90EF90DF90CF90BF90AF909F908F904B
:10BD40007F9008954F925F926F927F928F929F9211
:10BD5000AF92BF92CF92DF92EF92FF920F931F9319
:10BD6000CF93DF93CDB7DEB760970FB6F894DEBF01
:10BD70000FBECDBF80916B05811139C180916D05DA
:10BD8000811117C060960FB6F894DEBF0FBECDBF0D
:10BD9000DF91CF911F910F91FF90EF90DF90CF90A7
:10BDA000BF90AF909F908F907F906F905F904F90DB
:10BDB000089577DC0E9414A44B015C01809152111C
:10BDC000811117C08091670590916805A091690560
:10BDD000B0916A050097A105B10559F0A50194013C
:10BDE000281B390B4A0B5B0B57FD03C081E0809386
:10BDF000521160916C0470916D04072E000C880B39
:10BE0000990B0E949CF069837A838B839C8344E125
:10BE1000C42ED12C5CE3E52EF12C00E09E012F5FB7
:10BE20003F4F4EE654E06AE975E089E995E002DEAD
:10BE300040906E0450906F04609070047090710494
:10BE40006091390F70913A0F072E000C880B990BF7
:10BE50000E949CF09B01AC01C301B2010E9439F722
:10BE600018160CF4C8C060E06093700580919E05C0
:10BE700090919F05A091A005B091A1050097A10503
:10BE8000B10521F1A5019401281B390B4A0B5B0B6D
:10BE900057FD1CC06091A2057091A30580E090E061
:10BEA0000E949AF09B01AC0160916E0470916F0446
:10BEB00080917004909171040E9496F087FF4BC2AC
:10BEC00041E45AE163E57AE180E00ADC80916305B0
:10BED00090916405A0916505B0916605A501940156
:10BEE000281B390B4A0B5B0B57FD0FC0B8DED50181
:10BEF000C4018C53964FAF4FBF4F8093630590930F
:10BF00006405A0936505B09366058091A4059091A2
:10BF1000A505A091A605B091A7050097A105B105BB
:10BF200011F1881A990AAA0ABB0AB7FC1CC06091D1
:10BF3000A8057091A90580E090E00E949AF09B010D
:10BF4000AC01609168047091690480916A049091D9
:10BF50006B040E9496F087FF3BC14FE15AE162E318
:10BF60007AE18FEFBDDB6091660470916704072E64
:10BF7000000C880B990B0E949CF069837A838B8359
:10BF80009C8395E0C92ED12C24E1E22EF12C0FEFF9
:10BF90009E012F5F3F4F48E654E064E975E088E971
:10BFA00095E048DD8091B20581110FC1C090680411
:10BFB000D0906904E0906A04F0906B0420E030E0D7
:10BFC00040EA50E4C701B6010E9439F787FD0BC073
:10BFD00020E030E047E053E4C701B6010E9496F04C
:10BFE00018160CF0F7C060E060937105CBCE82E6C6
:10BFF0009AE10E94E5AD6091260270912702072E1A
:10C00000000C880B990B0E949CF09B01AC01C301B2
:10C01000B2010E9496F087FF26CF00916C04109128
:10C020006D0420ED3CEC4CE45DE360915F057091A4
:10C03000600580916105909162050E94FBF06B01A3
:10C040007C0120919005309191054091920550918D
:10C050009305C301B2010E9412F59B01AC01C70117
:10C06000B6010E94FBF06B017C0123E333E343E75D
:10C070005FE360918C0570918D0580918E059091A4
:10C080008F050E94FBF09B01AC01C701B6010E9425
:10C0900013F56B017C0160938C0570938D05809383
:10C0A0008E0590938F054092900550929105609275
:10C0B0009205709293058091521181114FC1B80180
:10C0C000012E000C880B990B0E949CF0A301920199
:10C0D0000E9412F52B013C0120E030E040E251E4E7
:10C0E0000E9439F718160CF44AC120E030E040E213
:10C0F00051ECC301B2010E9496F087FD2FC1012BC4
:10C1000009F42CC180918B05811170C18091870544
:10C1100090918805A0918905B0918A058D839E83B1
:10C12000AF83B88720915B0530915C0540915D0538
:10C1300050915E05C301B2010E94FBF069877A87C6
:10C140008B879C87A30192016D817E818F81988569
:10C150000E9413F56D837E838F8398876093870594
:10C16000709388058093890590938A0520915705DF
:10C17000309158054091590550915A050E94FBF0A5
:10C1800029853A854B855C850E9413F5A7019601A8
:10C190000E9412F56B017C0120E030E04FE753E490
:10C1A0000E9439F720E030E0A90118160CF406C10E
:10C1B000C701B6010E9496F087FD1FC1C701B601F5
:10C1C0000E9457F6759567954FCE10927105DACD9E
:10C1D0000ED9C9CE6091660470916704072E000CD9
:10C1E000880B990B0E949CF0A70196010E9412F502
:10C1F0004B015C0120915305309154054091550548
:10C20000509156050E94FBF069877A878B879C873F
:10C2100020918305309184054091850550918605D4
:10C22000C501B4010E9413F56D837E838F839887C7
:10C2300060938305709384058093850590938605AC
:10C2400020914F0530915005409151055091520574
:10C250000E94FBF06D877E878F87988B20ED3CECEA
:10C260004CE45DE360914B0570914C0580914D0568
:10C2700090914E050E94FBF02B013C0120917F051F
:10C28000309180054091810550918205C701B6012A
:10C290000E9412F59B01AC01C301B2010E94FBF0A8
:10C2A0002B013C0123E333E343E75FE360917B052C
:10C2B00070917C0580917D0590917E050E94FBF038
:10C2C0009B01AC01C301B2010E9413F52B013C019B
:10C2D00060937B0570937C0580937D0590937E052C
:10C2E000C0927F05D0928005E0928105F092820590
:10C2F0002D853E854F85588969857A858B859C85F6
:10C300000E9413F5A30192010E9412F56B017C01BA
:10C3100020E030E04FE753E40E9439F720E030E0BE
:10C32000A9011816FCF4C501B4010E9439F71816CA
:10C3300084F4A50194016D817E818F8198850E948E
:10C3400012F560938305709384058093850590931F
:10C3500086056FE749CE80E096D8B8CD81E080931E
:10C360008B0581CDC701B6010E9496F087FD0CC0F8
:10C37000C701B6010E9457F67595679535CE81E0E5
:10C3800080938B056FE770CD20E030E0A901C501F7
:10C39000B4010E9496F087FF26CEA50194016D811D
:10C3A0007E818F8198850E9412F56093830570933A
:10C3B0008405809385059093860515CEC301B2014F
:10C3C0000E9439F71816F4F6A30192016D817E815F
:10C3D0008F8198850E9412F5609387057093880578
:10C3E0008093890590938A056FE73ECD10928B0567
:10C3F0001D821E821F82188695CE20E030E0A901A2
:10C40000C301B2010E9496F087FF2DCDA3019201D6
:10C410006D817E818F8198850E9412F560938705DA
:10C42000709388058093890590938A051CCDCF92DF
:10C43000DF92EF92FF926B017C0183E3C816D10477
:10C44000E104F10468F082E3C81AD108E108F108B8
:10C4500062E370E080E090E00E9424BA73DCEDCFEC
:10C46000C701B6010E9424BAFF90EF90DF90CF90F1
:10C4700069CCCF92DF92EF92FF920F931F93CF93ED
:10C48000DF9388E50E94F93FD82E89E40E94F93FA6
:10C49000C82E882319F00E94923F1CC0DD20C1F0F5
:10C4A0000E94C23F20E030E040E251E40E9412F5D9
:10C4B00020E030E040EC51E40E9413F52BEA3AEA28
:10C4C0004AEA5CE30E94FBF00E9457F6653010F0E8
:10C4D0001FEF01C0162F89E50E94F93F082F8AE45B
:10C4E0000E94F93FC82F882319F00E94923F1CC078
:10C4F0000023C1F00E94C23F20E030E040E251E45E
:10C500000E9412F520E030E040EC51E40E9413F567
:10C510002BEA3AEA4AEA5CE30E94FBF00E9457F6F3
:10C52000653010F0DFEF01C0D62F8AE50E94F93F99
:10C53000E82E811105C081E50E94F93FF82E01C067
:10C54000F12CC11001C0C0E02C2F30E0D11001C08F
:10C5500000E0200F311D2130310521F4E1101AC017
:10C56000F11018C0E6E6F3E28491EF012196811103
:10C5700003C0E6EDFEE104C00E94138EFE01F4CF7D
:10C580008491EF012196882309F455C00E94138EEF
:10C59000FE01F6CF17FD02C0D7FF17C0E6E6F3E2B3
:10C5A0008491EF012196811103C0E7EBFEE104C005
:10C5B0000E94138EFE01F4CF8491EF01219688230F
:10C5C000D1F10E94138EFE01F7CF0E94C23F9B0162
:10C5D000AC01012F110F110BAD2FDD0FBB0BFF2095
:10C5E00099F085E0809FF001819FF00D1124EA0F02
:10C5F000FB1FEE0FFF1FEE0FFF1FEB55FE4E60817E
:10C6000071818281938103C060E070E0CB01E5E03D
:10C61000E09FE001E19FD00D1124CA0FDB1FCC0F7A
:10C62000DD1FCC0FDD1FCB55DE4E0E9413F5688356
:10C6300079838A839B83DF91CF911F910F91FF9024
:10C64000EF90DF90CF9008952F923F924F925F929C
:10C650006F927F928F929F92AF92BF92CF92DF9212
:10C66000EF92FF920F931F93CF93DF93CDB7DEB777
:10C6700061970FB6F894DEBF0FBECDBF83E50E9471
:10C68000F93F882349F00E94B33F182F811106C05B
:10C6900080E00E943B8402C010915B1180915404A1
:10C6A00090915504A0915604B091570489839A83C0
:10C6B000AB83BC838091580490915904A0915A0493
:10C6C000B0915B048D839E83AF83B88780915C04B7
:10C6D00090915D04A0915E04B0915F0489879A8770
:10C6E000AB87BC870E940E84882309F49AC083E438
:10C6F0000E94F93F882309F494C00E94C23F1B01A5
:10C700002C0105E0612C712C38EC388B82EC898B84
:10C71000A12CB12C98EC9E87E2E4EF87015080F1C8
:10C7200025E02D87209F400111243D8531503D8714
:10C730003F3FA1F3F401E30FF11DEE0FFF1FEE0FDA
:10C74000FF1FEB55FE4EC080D180E280F380960142
:10C75000A701B5018E859F850E9439F718161CF434
:10C760005601EE86FF869601A701B3018889998953
:10C770000E9496F087FFD9CF3601E88AF98AD5CF93
:10C78000930148895989B5018E859F850E9413F5CB
:10C7900020E030E040E05FE30E94FBF0A201910165
:10C7A0000E9413F52B013C012DEB37E346E855EBD6
:10C7B0000E9439F787FD0AC02DEB37E346E855E3C1
:10C7C000C301B2010E9496F018165CF580E00E9449
:10C7D0003B8435E0D32E45E0C42EDA949FEFD91682
:10C7E00001F105E0CD9C500111240150B0F3750119
:10C7F000E00EF11CC701880F991F880F991FFC01DB
:10C80000EB55FE4E7F01A30192016081718182810F
:10C8100093810E9412F5F701608371838283938371
:10C82000E4CF86E50E94F93F882399F00E940E84A8
:10C83000882379F0E1EAFEE184917F012FEFE21A8B
:10C84000F20A882321F00E94138EF701F5CF0E948F
:10C850001EC28AE50E94F93F882321F00E94C23F50
:10C860000E94E5B7812F0E943B84111103C0EBE7C2
:10C87000F3E21CC080915B118111F9CFE6E6F3E28F
:10C8800084918F010F5F1F4F882321F00E94138E28
:10C89000F801F6CFE2E8FEE184918F010F5F1F4FB0
:10C8A000882329F30E94138EF801F6CF84918F011B
:10C8B0000F5F1F4F882321F00E94138EF801F6CFDF
:10C8C00080915B11811103C067E173E002C063E1F5
:10C8D00073E084E79EE10E94DBCE8AE00E94138E23
:10C8E000EBE7F3E284918F010F5F1F4F882321F064
:10C8F0000E94138EF801F6CFE7E6FEE184918F01E6
:10C900000F5F1F4F882321F00E94138EF801F6CF8E
:10C91000C0905C11D0905D11E0905E11F0905F11BD
:10C9200020E030E0A901C701B6010E9439F71816CE
:10C930004CF442E0C701B6010E94D4918AE00E9403
:10C94000138E0CC0E2E6FEE184918F010F5F1F4F52
:10C95000882321F00E94138EF801F6CF4CE050E0BE
:10C9600064E574E0CE0101960E942FF8892BD1F086
:10C9700061960FB6F894DEBF0FBECDBFDF91CF91A9
:10C980001F910F91FF90EF90DF90CF90BF90AF90ED
:10C990009F908F907F906F905F904F903F902F90DF
:10C9A0000C94C17D61960FB6F894DEBF0FBECDBF6B
:10C9B000DF91CF911F910F91FF90EF90DF90CF907B
:10C9C000BF90AF909F908F907F906F905F904F90AF
:10C9D0003F902F90089580916F00982F927081FF63
:10C9E00005C080916F008D7F80936F008091280932
:10C9F00080932709809326098093250984E68093F4
:10CA0000240928EE33E030936F0520936E059923B7
:10CA100029F080916F00826080936F0081E08093A5
:10CA200027190E94B07D0E94B2CB80915B118823B0
:10CA300021F08AE392E10E94BDCF8CE0EAE3F2E1CB
:10CA4000A4E5B4E001900D928A95E1F70C94DA8C9C
:10CA50002F923F924F925F926F927F928F929F920E
:10CA6000AF92BF92CF92DF92EF92FF920F931F93FC
:10CA7000CF93DF93CDB7DEB7CD54D1090FB6F8947D
:10CA8000DEBF0FBECDBF85E40E944240882321F067
:10CA90000E94923F8B0102C000E010E083E40E94FC
:10CAA0004240882321F00E94923F6AA302C025E001
:10CAB0002AA385E50E944240882319F00E94B33FD3
:10CAC00003C085E50E94F93F8CA717FD07C0C12C64
:10CAD000D12CB6E1EB2EB3E4FB2E06C0C12CD12C39
:10CAE000ACE8EA2EA2E4FA2E83E50E9442408823B5
:10CAF00021F00E94C23F6B017C010115110511F468
:10CB00001092720510924011102F0E9414A42B0154
:10CB10003C01302F331F3327331F83E0831B89836E
:10CB2000D301C2018C53964FAF4FBF4F8093630523
:10CB300090936405A0936505B09366050F5F02307E
:10CB400080F0E8E3FEE18491AF014F5F5F4F5A83CD
:10CB50004983882309F473C30E94138EE981FA8103
:10CB6000F2CF17FD12C0E12FEE0FFF0BEA5DFD4F74
:10CB7000608171816A507109072E000C880B990B36
:10CB80000E949CF04B015C0106C0812C912CFAEFB5
:10CB9000AF2EF2E4BF2EC701B6010E9457F6072E52
:10CBA000000C880B990B0E949CF069877A878B8711
:10CBB0009C87A50194010E9439F718167CF4E9EFCF
:10CBC000FDE18491DF011196BA83A983882309F4DA
:10CBD00036C30E94138EE981FA81F3CFE4E2FEE1CD
:10CBE00084917F01BFEFEB1AFB0A882321F00E949A
:10CBF000138EF701F5CF0E949F5A17FF04C08FE7ED
:10CC00008093710508C0E12F012E000CFF0BE05945
:10CC1000FA4F8FE78083E9818E2F90E0A301920184
:10CC2000205A35414F4F5F4F2EAB3FAB48AF59AF06
:10CC300021E0209352021F3F49F443E65DE15BAFE0
:10CC40004AAFADE2BDE1BDAFACAF08C0E1E5FDE18B
:10CC5000FBAFEAAF2AE13DE13DAF2CAF4CA25DA2B4
:10CC60006EA27FA24DA65EA66FA678AA19AA1AAADE
:10CC70001BAA1CAA1DAA2A961FAE2A9730E4398F38
:10CC80004CE14A8F56E45B8F1C8E1D8E1E8E1F8ECC
:10CC90001D8A1E8A1F8A188E198A1A8A1B8A1C8A64
:10CCA00019821A821B821C822FE730E040E050E09C
:10CCB0002D833E834F8358877FE7C72ED12CE12CED
:10CCC000F12C18A619A61AA61BA631E03D87188AD2
:10CCD0001F8629961FAE2997212C312C00E0212F89
:10CCE000012E000C330BA90140595A4F5FAF4EAFD4
:10CCF000220F331F220F331FD901A259BB4FB9A3F3
:10CD0000A8A39C01092E000C440B550B24962CAFB4
:10CD10003DAF4EAF5FAF249704969C01990F440B33
:10CD2000550B28962CAF3DAF4EAF5FAF28974AA169
:10CD3000042E000C550B5BA34AA38091520288235A
:10CD400009F47BC20E9414A44B015C0180916D0523
:10CD5000882309F4D8C00E94515B17FD0CC0A8A11C
:10CD6000B9A1BC912996BFAF2997E8A1F9A121806B
:10CD7000328003810BC0F09168042996FFAF299798
:10CD80002090690430906A0400916B0429962FADBD
:10CD90002997322D432D502F6C8D7D8D8E8D9F8D3B
:10CDA0000E9496F087FF07C029962FAD29972C8FF8
:10CDB0002D8E3E8E0F8F2A962FAD2A97398D4A8D54
:10CDC0005B8D29966FAD2997722D832D902F0E9430
:10CDD00096F087FF09C029963FAD29972A963FAF65
:10CDE0002A97298E3A8E0B8F809163059091640566
:10CDF000A0916505B0916605A5019401281B390B2A
:10CE00004A0B5B0B57FD10C00E942F5ED501C40179
:10CE10008C53964FAF4FBF4F80936305909364053B
:10CE2000A0936505B09366053D8529962FAD29979A
:10CE3000332309F44BC0322D432D502F69857A8559
:10CE40008B859C850E9496F087FF5DC0D501C4014B
:10CE500084199509A609B7092E968CAF9DAFAEAF80
:10CE6000BFAF2E9788589341A109B109B7FD4BC0B8
:10CE7000D701C6012D813E814F815885821B930BBE
:10CE8000A40BB50BB595A7959795879517FF03C08C
:10CE90008093710503C0EEADFFAD80832E962CAD5F
:10CEA0003DAD4EAD5FAD2E9728A739A74AA75BA72A
:10CEB00039853C8F4A854D8F5B855E8F8C858F8F42
:10CEC0008CA29DA2AEA2BFA21D861DC0322D432DF5
:10CED000502F69857A858B859C850E9439F71816B5
:10CEE00094F4D501C4012CA13DA14EA15FA1821BE8
:10CEF000930BA40BB50BAC01BD014858534161091C
:10CF0000710977FFB9C120E030E040EA51E469855A
:10CF10007A858B859C850E9413F529962FAD2997DC
:10CF2000322D432D502F0E9496F087FF0FC0E5E869
:10CF3000FDE18491DF011196BA83A983882309F466
:10CF40007CC10E94138EE981FA81F3CFD501C4011F
:10CF50002DA53EA54FA558A9821B930BA40BB50B7D
:10CF6000B7FD89C00E943D598AE00E94138ED50109
:10CF7000C4018053984FAF4FBF4F8DA79EA7AFA757
:10CF8000B8AB99A991115AC02AA93BA94CA95DA98E
:10CF900029966FAD2997722D832D902F0E9439F716
:10CFA0001816DCF524966CAD7DAD8EAD9FAD249743
:10CFB0000E949CF029962FAD2997322D432D502F9A
:10CFC0000E9413F56AAB7BAB8CAB9DABA5019401C2
:10CFD000205A35414F4F5F4F2EAB3FAB48AF59AF53
:10CFE00028966CAD7DAD8EAD9FAD28970E949CF0CC
:10CFF0009B01AC0169857A858B859C850E9412F521
:10D0000029962FAD2997322D432D502F0E9496F04F
:10D01000881F8827881F89AB2EC0D501C4012EA97F
:10D020003FA948AD59AD821B930BA40BB50BB7FDBF
:10D0300022C04AAD5BAD66E77DE11AC020E030E07A
:10D0400040EA51E469857A858B859C850E9412F5BA
:10D050009B01AC0129966FAD2997722D832D902FDE
:10D060000E9496F087FF07C04CAD5DAD61E47DE1A5
:10D07000812F0E94705BD501C401880F991FAA1FE0
:10D08000BB1F2CA13DA14EA15FA1821B930BA40B42
:10D09000B50B84199509A609B70981309F49A442A7
:10D0A000B10580F0ECEFFCE18491AF014F5F5F4F81
:10D0B0005A834983882309F4C0C00E94138EE981F2
:10D0C000FA81F2CF8AA19BA1AF85B8898A179B0705
:10D0D0000CF033CEEFE9FCE184913F01BFEF6B1A16
:10D0E0007B0A882321F00E94138EF301F5CF17FDF0
:10D0F00005C0E6E1F3E0FE83ED8304C020E234E006
:10D100003E832D836D817E818EE89CE10E94DBCE83
:10D1100049815A816B817C818AE89CE10E94A5CE7D
:10D120008AE00E94138E6D817E8189E79CE10E94D6
:10D13000DBCE49895A896B897C8985E79CE10E940D
:10D14000A5CE8AE00E94138E6D817E8184E69CE1EB
:10D150000E94DBCE4D895E896F89788D80E69CE1E7
:10D160000E94A5CE8AE00E94138E3CA5332309F4C9
:10D1700066C017FF31C089819A81AB81BC818093E1
:10D18000530590935405A0935505B09356052CEA8A
:10D1900035EC47E25EE369897A898B899C890E9434
:10D1A000FBF060934F057093500580935105909369
:10D1B00052052CEA35EC47E25EE36D897E898F8962
:10D1C000988D0E94EFF560934B0570934C0580930A
:10D1D0004D0590934E0533C029813A814B815C8186
:10D1E00020935B0530935C0540935D0550935E058D
:10D1F0002CEA35EC47E25EE369897A898B899C8960
:10D200000E94FBF060935705709358058093590571
:10D2100090935A052CEA35EC47E25EE36D897E89EE
:10D220008F89988D0E94EFF560935F05709360057C
:10D23000809361059093620502C00E949F5A81E02D
:10D2400080934011C35BDF4F0FB6F894DEBF0FBE73
:10D25000CDBFDF91CF911F910F91FF90EF90DF90A5
:10D26000CF90BF90AF909F908F907F906F905F9086
:10D270004F903F902F9008954F855889452B09F482
:10D2800037C148A459A46AA47BA4480E591E6A1E3B
:10D290007B1E28A539A54AA55BA5281B390B4A0B7F
:10D2A0005B0B6D817E818F8198850E94A6F4A3011E
:10D2B00092010E94D7F4DA01C9018C0D9D1DAE1DAB
:10D2C000BF1D84319105A105B105FCF06C017D0104
:10D2D0008C3E9105A105B1052CF05BEEC52ED12C3D
:10D2E000E12CF12C80E8C816D104E104F104DCF053
:10D2F0002EEF30E040E050E02C193D094E095F0967
:10D300002D833E834F83588712C044E1C42ED12C15
:10D31000E12CF12C84E190E0A0E0B0E08D839E83CD
:10D32000AF83B88704C0CD82DE82EF82F886E1EF5A
:10D33000FDE18491DF011196BE87AD87882329F036
:10D340000E94138EED85FE85F4CFC701B6010E94C1
:10D35000BA91ECEEFDE184919F012F5F3F4F3E8734
:10D360002D87882329F00E94138EED85FE85F3CF4B
:10D370006D817E818F8198850E94BA912A964FADEA
:10D380002A97598D6A8D7B8D85EE9DE10E94A5CEF1
:10D390004C8D5D8D6E8D7F8D8EED9DE10E94A5CEB5
:10D3A0004F855889433051050CF4A2C06D817E81B0
:10D3B0008F8198850E949CF020E030E040E850E4A6
:10D3C0000E94FBF069837A838B839C832A962FAD1E
:10D3D0002A97398D4A8D5B8D6C8D7D8D8E8D9F8DBD
:10D3E0000E9412F52BED3FE049E450E40E94FBF06F
:10D3F00020E030E040E05FE30E94FBF09B01AC01E5
:10D4000069817A818B819C810E94EFF569837A839F
:10D410008B839C83C301B2010E949CF02FE632E112
:10D4200043E85AE30E94FBF02B013C0149815A81F9
:10D430006B817C8188ED9DE10E94A5CEB301A201A4
:10D4400082ED9DE10E94A5CE2AE939E949E15FE339
:10D4500069817A818B819C810E94FBF069837A8348
:10D460008B839C839B01AC010E9413F5A301920165
:10D470000E94EFF5698B7A8B8B8B9C8B29813A818B
:10D480004B815C81C301B2010E94FBF020E030E0DF
:10D4900040E05EE30E94FBF06D8B7E8B8F8B988F5C
:10D4A000E2ECFDE184913F015FEF651A750A882384
:10D4B00021F00E94138EF301F5CF49815A816B81CF
:10D4C0007C818CEB9DE10E94A5CE49895A896B89AC
:10D4D0007C8986EB9DE10E94A5CE4D895E896F898E
:10D4E000788D80EB9DE10E94A5CE8AE00E94138E8C
:10D4F0008D819E81AF81B8858C0D9D1DAE1DBF1D98
:10D50000B595A7959795879517FF03C080937105EB
:10D5100003C0EEADFFAD80832F8538892F5F3F4F6D
:10D52000388B2F8739852A963FAF2A974A85498FAE
:10D530005B855A8F8C858B8F2401350191E09D8707
:10D54000E2CCCF93DF93EBE7F3E28491EF012196F6
:10D55000882321F00E94138EFE01F7CF83E50E94FD
:10D56000F93F882321F00E94B33F80934102E0E518
:10D57000FCE18491EF012196882321F00E94138E13
:10D58000FE01F7CF80914102811103C0ECE4FCE180
:10D5900002C0E8E4FCE18491EF012196882321F0A8
:10D5A0000E94138EFE01F7CFE0E4FCE18491EF01CD
:10D5B0002196882321F00E94138EFE01F7CF20913F
:10D5C00038043091390440913A0450913B04609101
:10D5D00002117091031180910411909105110E9424
:10D5E00013F5AB01BC018EE39CE10E94A5CE209116
:10D5F0003C0430913D0440913E0450913F046091C1
:10D6000006117091071180910811909109110E94E3
:10D6100013F5AB01BC018BE39CE10E94A5CE2091E8
:10D620004004309141044091420450914304609180
:10D630000A1170910B1180910C1190910D110E94A3
:10D6400013F5AB01BC0188E39CE10E94A5CEE0E3A9
:10D65000FCE18491EF012196882321F00E94138E32
:10D66000FE01F7CF209138043091390440913A04FB
:10D6700050913B0460912D0270912E0280912F02F7
:10D68000909130020E9413F5AB01BC018EE29CE147
:10D690000E94A5CE20913C0430913D0440913E046F
:10D6A00050913F04609131027091320280913302B7
:10D6B000909134020E9413F5AB01BC018BE29CE116
:10D6C0000E94A5CE20914004309141044091420433
:10D6D0005091430460913502709136028091370277
:10D6E000909138020E9413F5AB01BC0188E29CE1E5
:10D6F0000E94A5CE8AE0DF91CF910C94138EFF9209
:10D700000F931F93CF93DF93F82E092F162FE3E289
:10D71000FCE18491EF012196882321F00E94138E71
:10D72000FE01F7CFEF2DF02F8491EF012196882392
:10D7300021F00E94138EFE01F7CFE1E2FCE184911B
:10D74000EF012196882321F00E94138EFE01F7CF6E
:10D75000612F70E080E090E00E94BA918AE0DF9152
:10D76000CF911F910F91FF900C94138ECF92DF9267
:10D77000EF92FF920F931F93CF93DF93CDB7DEB756
:10D78000A0970FB6F894DEBF0FBECDBF8091A5095C
:10D79000882331F083E08093280C81E080932A0C69
:10D7A00080E090E0A0EAB0E489839A83AB83BC83F5
:10D7B00080E090E0ADE4B3E48D839E83AF83B887CF
:10D7C00080E090E0A0EAB1E489879A87AB87BC87C4
:10D7D00088E592E00E941A8E81118DC185E40E9435
:10D7E000F93F882381F00E94C23F6B017C0120E059
:10D7F00030E0A9010E9439F787FF0BC0F7FAF094D7
:10D80000F7F8F09406C0C12CD12C80E8E82E80E413
:10D81000F82EF7FAF094F7F8F094C98ADA8AEB8ACE
:10D82000FC8A8AE50E944240882379F08AE50E94BA
:10D830004240882319F00E94C23F03C060E070E0BC
:10D84000CB0169877A878B879C8788E50E94424055
:10D85000882379F088E50E944240882319F00E94CD
:10D86000C23F03C060E070E0CB0169837A838B83A1
:10D870009C8389E50E944240882379F089E50E94D3
:10D880004240882319F00E94C23F03C060E070E06C
:10D89000CB016D837E838F83988785E50E94F93F56
:10D8A000882329F00E94C23F6B017C010CC0E091EB
:10D8B0000E1184E0E89FF0011124EE5EF64EC08068
:10D8C000D180E280F38020E030E0A901C701B601F9
:10D8D0000E9439F787FF04C0F7FAF094F7F8F09444
:10D8E000F7FAF094F7F8F094CD8ADE8AEF8AF88E92
:10D8F000198E1A8E1B8E1C8E8CE40E94F93F882391
:10D9000029F00E94C23F6B017C010CC0E0910E1116
:10D9100094E0E99FF0011124EA5EF64EC080D180C8
:10D92000E280F38020E030E0A901C701B6010E9447
:10D9300039F787FF04C0F7FAF094F7F8F094CD8E2A
:10D94000DE8EEF8EF8A282E40E944240882321F00E
:10D950000E94923F162F01C01AE000914019AE01BB
:10D960004B5E5F4FBE016F5F7F4FCE0141960E94BD
:10D9700007B3882309F4BBC0EBE7F3E284917F018E
:10D980009FEFE91AF90A882321F00E94138EF7010C
:10D99000F5CFEFE2FFE184917F019FEFE91AF90AE9
:10D9A000882321F00E94138EF701F5CF61E0812FCB
:10D9B0000E9485810E9414A4DC01CB0180529C4608
:10D9C000AB4FBF4F8093670590936805A09369059F
:10D9D000B0936A051092521183E08093401181E068
:10D9E00080931E1980911E19882309F466C060E097
:10D9F000812F0E94858180915211882309F459C09A
:10DA0000EBE7F3E284917F019FEFE91AF90A88239B
:10DA100021F00E94138EF701F5CFE5E1FFE184913B
:10DA20007F019FEFE91AF90A882339F00E94138ECB
:10DA3000F701F5CF81E00E942CAE80911E19811173
:10DA4000F9CF0E94B5AD0E948DB2EBE7F3E284916D
:10DA50007F019FEFE91AF90A882321F00E94138EB3
:10DA6000F701F5CFE6EFFEE184917F019FEFE91A20
:10DA7000F90A81111AC00E9414A4DC01CB01805262
:10DA80009C46AB4FBF4F8093670590936805A0936A
:10DA90006905B0936A051092521181E080931E19B6
:10DAA00061E0812F0E94858104C00E94138EF701DE
:10DAB000DBCF81E00E942CAE95CF81E080934011B6
:10DAC00080E090E0A0E0B0E48D879E87AF87B88BC0
:10DAD00080911607882359F0212FAE01435F5F4FD5
:10DAE000BE01635E7F4FCE0149960E945EBA01304F
:10DAF00011F40E94F6CEA0960FB6F894DEBF0FBECA
:10DB0000CDBFDF91CF911F910F91FF90EF90DF90EC
:10DB1000CF9008952F923F924F925F926F927F9293
:10DB20008F929F92AF92BF92CF92DF92EF92FF922D
:10DB30000F931F93CF93DF93CDB7DEB7C857D109AB
:10DB40000FB6F894DEBF0FBECDBFE0916E05F09129
:10DB50006F05EF2B11F00C944B762896DFAECEAE0E
:10DB600028976E2C79016A015B01FC0120813181CB
:10DB7000428153816C962CAF3DAF4EAF5FAF6C9737
:10DB80002091711130917211409173115091741163
:10DB90006C966CAD7DAD8EAD9FAD6C970E94FBF029
:10DBA0000E9444F7E0966CAF7DAF8EAF9FAFE097D9
:10DBB000D5018D919D910D90BC91A02DA0968CAF1B
:10DBC0009DAFAEAFBFAFA097209175113091761188
:10DBD0004091771150917811BC01CD010E94FBF06A
:10DBE0000E9444F7E4966CAF7DAF8EAF9FAFE49791
:10DBF000D6012D913D914D915C91A4962CAF3DAFF6
:10DC00004EAF5FAFA4972091791130917A11409176
:10DC10007B1150917C11A4966CAD7DAD8EAD9FAD06
:10DC2000A4970E94FBF00E9444F7E8966CAF7DAF8A
:10DC30008EAF9FAFE897D7012D913D914D915C91AB
:10DC400022962CAF3DAF4EAF5FAF229720917D1152
:10DC500030917E1140917F115091801122966CADD0
:10DC60007DAD8EAD9FAD22970E94FBF00E9444F7E0
:10DC700060966CAF7DAF8EAF9FAF60978091FF05D0
:10DC800083FF1CC060962CAD3DAD4EAD5FAD60977F
:10DC90002093590930935A0940935B0950935C09CA
:10DCA00022968CAD9DADAEADBFAD22978093490954
:10DCB00090934A09A0934B09B0934C09D801BC91A9
:10DCC000B9A7F801F181F9ABD8011296BC91BEABAE
:10DCD000F801F381FAAF8091270990912809891BF7
:10DCE0008F708F3021F480E00E942CAEF4CF009131
:10DCF0002709E9960FAFE99780912709082F10E0CF
:10DD00001CA30BA380914D0990914E09A0914F093E
:10DD1000B0915009E0968CAC9DACAEACBFACE09736
:10DD2000881A990AAA0ABB0A80915109909152094E
:10DD3000A0915309B0915409E4962CAC3DAC4EAC83
:10DD40005FACE497281A390A4A0A5B0A80915509A0
:10DD500090915609A0915709B0915809E8962CADB9
:10DD60003DAD4EAD5FADE897281B390B4A0B5B0B01
:10DD70002DA33EA34FA358A78091590990915A090A
:10DD8000A0915B09B0915C0960960CAD1DAD2EAD04
:10DD90003FAD6097081B190B2A0B3B0B0DA71EA765
:10DDA0002FA738AB012B022B032B09F4BCC08091A9
:10DDB000511181114BC060916E0470916F0480917C
:10DDC0007004909171040E9457F6209139023091AD
:10DDD0003A02621773070CF039C060962CAD3DAD66
:10DDE0004EAD5FAD60972093590930935A09409327
:10DDF0005B0950935C0922968CAD9DADAEADBFAD75
:10DE000022978093490990934A09A0934B09B093B4
:10DE10004C09EBE7F3E284918F010F5F1F4F8111F3
:10DE200003C0EAE7FFE104C00E94138EF801F3CFBC
:10DE300084918F010F5F1F4F882321F00E94138E62
:10DE4000F801F6CF1DA61EA61FA618AA94E0699E8B
:10DE500080011124025E1D4F6DA57EA58FA598A996
:10DE60000E949CF0D8012D913D914D915C910E94B2
:10DE7000FBF06B017C0120E030E0A9010E9439F742
:10DE800087FF04C0F7FAF094F7F8F09460917D11E1
:10DE900070917E1180917F11909180110E9457F6B0
:10DEA0009B01AC01A8E5B2E00E94F3F40E949CF053
:10DEB000A70196010E9496F087FF39C060960CADCD
:10DEC0001DAD2EAD3FAD60970093590910935A09CF
:10DED00020935B0930935C0922962CAD3DAD4EAD8D
:10DEE0005FAD22972093490930934A0940934B092B
:10DEF00050934C09EBE7F3E284918F010F5F1F4FC2
:10DF0000811103C0EBE5FFE104C00E94138EF8010C
:10DF1000F3CF84918F010F5F1F4F882321F00E9460
:10DF2000138EF801F6CF1DA61EA61FA618AAD501AE
:10DF3000C4018827B7FD83959927AA27BB27782E88
:10DF400057FE03C0382F3260732E8DA19EA1AFA162
:10DF5000B8A5B7FF03C0972D9460792E0DA51EA517
:10DF60002FA538A937FF03C0172D1860712E24E0A4
:10DF7000629E80011124025E1D4F6DA57EA58FA5B6
:10DF800098A90E949CF0D8012D913D914D915C91F2
:10DF90000E94FBF06B017C0120E030E0A9010E94AF
:10DFA00039F787FF04C0C701B601905802C0C70106
:10DFB000B60120E030E040E05FE30E9413F50E94EC
:10DFC0005CF66AAB7BAB8CAB9DAB88E60BA11CA16E
:10DFD000809FF001819FF00D1124E657FD4E1082C5
:10DFE000EA5BFF4F7082B501A401B7FE07C044276A
:10DFF0005527BA01481959096A097B0988E60BA116
:10E000001CA1809FF001819FF00D1124E657FD4E69
:10E01000458B568B678B708F2C962CAE3DAE4EAEDB
:10E020005FAE2C9757FE0DC088279927DC01821917
:10E030009309A409B5092C968CAF9DAFAEAFBFAFC5
:10E040002C9728E60BA11CA1209FF001219FF00D29
:10E050001124E657FD4E2C968CAD9DADAEADBFADF7
:10E060002C97818F928FA38FB48F0DA11EA12FA10A
:10E0700038A537FF07C030952095109501951F4FA3
:10E080002F4F3F4FE8E67E2EABA1BCA17A9EF00158
:10E090007B9EF00D1124E657FD4E058F168F278FBE
:10E0A00030A38AA99BA9ACA9BDA981A392A3A3A3CC
:10E0B000B4A323964FAF2397752EF62FE72F2C96F8
:10E0C0008CAD9DADAEADBFAD2C97481759076A0713
:10E0D0007B0778F429969FAD299723969FAF2397C6
:10E0E0002A967FAC2A972B96FFAD2B972C96EFADF7
:10E0F0002C9723968FAD2397972DAF2FBE2F801788
:10E100009107A207B30710F4D901C8010AA91BA9F6
:10E110002CA93DA980179107A207B30710F4D901D4
:10E12000C80128E60BA11CA1209FF001219FF00D42
:10E130001124E657FD4E85A396A3A7A3B0A7069783
:10E14000A105B10508F4A0C5DF01AE59BF4F80910C
:10E150006404909165048D939C9361A6452B462B96
:10E16000472B09F05F9888E60BA11CA1809FF00166
:10E17000819FF00D1124E657FD4E818D928DA38D68
:10E18000B48D892B8A2B8B2B11F08A98479888E6BF
:10E190000BA11CA1809FF001819FF00D1124E65777
:10E1A000FD4E858D968DA78DB0A1892B8A2B8B2B4B
:10E1B00031F08091080181708093060147982AA967
:10E1C0003BA94CA95DA9232B242B252B09F465C55C
:10E1D00080910406882319F0815080930406611011
:10E1E00004C0129880E2809304066090FB05709052
:10E1F000FC050091FD051091FE059301A80169A59C
:10E2000079A98EA99AAD0E9496F087FF04C069A6ED
:10E2100079AA0EAB1AAFC501B4010E949CF02091FF
:10E2200076123091771240917812509179120E94B3
:10E23000FBF026966CAF7DAF8EAF9FAF2697698BB4
:10E240007A8B8B8B9C8BC201B1010E949CF0209138
:10E250007A1230917B1240917C1250917D120E9473
:10E26000FBF02B013C016D8B7E8B8F8B988F6DA10A
:10E270007EA18FA198A50E949CF020917E123091E2
:10E280007F1240918012509181120E94FBF04B014D
:10E290005C01698F7A8F8B8F9C8F209182123091D5
:10E2A00083124091841250918512C701B6010E94D9
:10E2B000FBF06B017C016D8F7E8F8F8F98A388E6BA
:10E2C0000BA11CA1809FF001819FF00D1124E65746
:10E2D000FD4E258936894789508D2DA33EA34FA336
:10E2E00058A7263031054105510508F4DFC42896AA
:10E2F000AEADBFAD2897CD90DD90ED90FC9020E0C5
:10E3000030E0A901C701B6010E9496F08111EDC469
:10E3100026962CAD3DAD4EAD5FAD2697CA01B90135
:10E320000E94FBF06B017C01A3019201C301B201C9
:10E330000E94FBF09B01AC01C701B6010E9413F5DE
:10E340006B017C01A5019401C501B4010E94FBF0A1
:10E350009B01AC01C701B6010E9413F50E947EF734
:10E3600028E60BA11CA1209FF001219FF00D112494
:10E37000E657FD4E658776878787908B88E60BA1E9
:10E380001CA1809FF001819FF00D1124E657FD4EE6
:10E390004584568467847088A301920160E070E030
:10E3A00080E89FE30E94EFF564966CAF7DAF8EAF7F
:10E3B0009FAF649729A539A94EA95AAD0E94FBF0D9
:10E3C0004B015C018091270990912509891B8F7071
:10E3D00027968FAF2797A501940160E074E284E748
:10E3E00099E40E94EFF50E9444F76B017C012796A7
:10E3F0008FAD27978250863008F486C4A50194011A
:10E40000C301B2010E94FBF09B01AC010E94FBF032
:10E4100068966CAF7DAF8EAF9FAF689788E6ABA173
:10E42000BCA18A9F80018B9F100D112406571D4EA1
:10E4300068962CAD3DAD4EAD5FAD6897D801119695
:10E440002D933D934D935C93149795962D913D910B
:10E450004D915C9198972EAB3FAB48AF59AFCA0135
:10E46000B9010E949AF06AAF7BAF8CAF9DAF9B0160
:10E47000AC01C501B4010E94FBF00E94D9F50E94D5
:10E480005CF6A8966CAF7DAF8EAF9FAFA897F801F2
:10E49000EE5AFF4F60837183828393838E010F5EF8
:10E4A0001F4F2A961FAF0EAF2A97005111092496CD
:10E4B0001FAF0EAF249703EE15E0AC961FAF0EAF63
:10E4C000AC978E010F5D1F4F1AA309A324960EADC2
:10E4D0001FAD2497AA961FAF0EAFAA97312C212CFF
:10E4E00010E819A70FE309AB2A96AEADBFAD2A9786
:10E4F0002D913D914D915D912A96BFAFAEAF2A9778
:10E50000C501B4010E94FBF06B017C01AA96EEAD3F
:10E51000FFADAA976193719381939193AA96FFAFF0
:10E52000EEAFAA9720E030E0A9010E9439F787FFFB
:10E5300004C0F7FAF094F7F8F094AC96AEADBFAD26
:10E54000AC974D905D906D907D90AC96BFAFAEAFA7
:10E55000AC97A7019601C301B2010E9496F087FD16
:10E560000DC409A11AA12A962EAD3FAD2A97021714
:10E57000130709F0B9CF20E030E040E85FE3632DF6
:10E58000722D89A599A90E9496F087FF58C07E0137
:10E5900031E1E30EF11C24960EAD1FAD2497232D1F
:10E5A000322D49A559A9D8016D917D918D919C91EC
:10E5B0000E94FBF0F80161937193819391938F0115
:10E5C000EE16FF0661F728E60BA11CA1209FC001F3
:10E5D000219F900D11249C0126573D4E7901890100
:10E5E0000E5A1F4FA8966CAD7DAD8EAD9FADA8970E
:10E5F0000E949AF0232D322D49A559A90E94FBF0C3
:10E600000E945CF6D8016D937D938D939C93139734
:10E61000232D322D49A559A9632D722D89A599A9BC
:10E620000E94FBF068962CAD3DAD4EAD5FAD689796
:10E630000E94FBF0F70161837283838394832AAD88
:10E640003BAD4CAD5DAD64966CAD7DAD8EAD9FAD1B
:10E6500064970E94FBF069A77AA78BA79CA70DA1DE
:10E660001EA12FA138A5012B022B032B09F09EC35D
:10E6700088E62BA13CA1829F8001839F100D11246D
:10E6800006571D4EF801818D928DA38DB48D892B77
:10E690008A2B8B2B09F08AC3858D968DA78DB0A10F
:10E6A000892B8A2B8B2B09F081C320913C1130914F
:10E6B0003D1140913E1150913F1169A57AA58BA55E
:10E6C0009CA50E94FBF00E94D9F50E945CF62B01EC
:10E6D0003C01F801E95BFF4F108288E62BA13CA1C9
:10E6E000829F8001839F100D112406571D4EF80153
:10E6F000E25AFF4F4082518262827382C301B201AB
:10E700000E949AF029A53AA54BA55CA50E94EFF5B9
:10E710006AAF7BAF8CAF9DAFD80151966D937D935F
:10E720008D939C935497F801E95BFF4F8081882378
:10E7300081F17801B8E4EB0EF11C37962091D705F2
:10E740003091D8054091D9055091DA0560817181E9
:10E75000828193810E94FBF02AAD3BAD4CAD5DAD53
:10E760000E94FBF020917D1130917E1140917F112C
:10E77000509180110E94FBF09B01AC0160E074E2BB
:10E7800084EF99E40E94EFF50E945CF6F701718333
:10E79000608388E60BA11CA1809FF001819FF00D92
:10E7A0001124E657FD4E21813281438154812C96FC
:10E7B0002CAF3DAF4EAF5FAF2C97CA01B9010E949D
:10E7C0007EF7362E272E8C0147EC55E062965FAF20
:10E7D0004EAF62973E0151E1650E711C87EC95E0EA
:10E7E0009FAB8EAB24964EAC5FAC24973DA62DA27A
:10E7F00009A719AB1AAAD201CD90DD90ED90FD903A
:10E800002D0120E030E0A901C701B6010E9439F7CF
:10E8100087FF04C0F7FAF094F7F8F094EEA9FFA987
:10E8200081909190A190B190FFABEEABA7019601C2
:10E83000C501B4010E9496F087FDD8C56414750423
:10E84000D1F627965FAD2797552309F448C6C090A7
:10E850002909D0902A09E0902B09F0902C092DEB82
:10E8600037E346E855E3C701B6010E9496F087FDFD
:10E8700036C6C701B6010E947EF76B017C019B0181
:10E88000AC01632D722DC8010E9496F087FD03C074
:10E890003C2C2D2C87019601A701632D722DC801F8
:10E8A0000E94EFF568966CAF7DAF8EAF9FAF689713
:10E8B0008DE299E028969FAF8EAF289720E030E058
:10E8C00040E85FE32AAB3BAB4CAB5DAB1EAA28969E
:10E8D000AEADBFAD28972D913D914D915D9128969C
:10E8E000BFAFAEAF289768966CAD7DAD8EAD9FADD6
:10E8F00068970E94FBF04B015C012496EEADFFADE2
:10E900002497C190D190E190F1902496FFAFEEAFA3
:10E910002497FEA9FF2391F02AA93BA94CA95DA940
:10E920000E94FBF04B015C012AA93BA94CA95DA9FF
:10E93000C701B6010E94FBF06B017C01A7019601A3
:10E94000C501B4010E9439F720E030E0A901181692
:10E950000CF092C5C701B6010E9439F718160CF4E5
:10E9600086C520E030E0A901C501B4010E9496F0FF
:10E9700087FD7DC52601370177FA709477F870948A
:10E98000A3019201C501B4010E9439F7181614F4CD
:10E99000240135016296AEADBFAD6297CD90DD909A
:10E9A000ED90FD906296BFAFAEAF6297A30192016A
:10E9B000C701B6010E9496F087FF15C0A30192011E
:10E9C000C701B6010E94EFF59B01AC016AA97BA9C2
:10E9D0008CA99DA90E94FBF06AAB7BAB8CAB9DAB75
:10E9E000BEA9BF5FBEABEDE3F9E028962EAD3FAD0B
:10E9F0002897E217F30709F06ACF3EA9332361F0A5
:10EA00002AA93BA94CA95DA9632D722DC8010E94BA
:10EA1000FBF0362E272E8C0124EA30E74DE75FE32A
:10EA2000632D722DC8010E94FBF06B017C012091C7
:10EA300000063091010640910206509103060E94A3
:10EA400096F087FD42C58DA59DA1A9A5B9A9809382
:10EA5000000690930106A0930206B093030628E6F1
:10EA60004BA15CA1249FC001259F900D1124DC01C6
:10EA7000A657BD4E7D01232D322DA801632D722D89
:10EA8000C8010E94FBF0F701618772878387948732
:10EA90006AAD7BAD8CAD9DAD90589B01AC010E94E1
:10EAA00013F5D7011D962D913D914D915C91509795
:10EAB0000E94FBF09B01AC016BE077ED83E29BE3EE
:10EAC0000E9412F59B01AC018BE097EDA3E2BBE342
:10EAD000F70185839683A783B08710812C966CAD50
:10EAE0007DAD8EAD9FAD2C970E9496F018160CF45C
:10EAF000FBC483E0182B88E62BA13CA1829FF00188
:10EB0000839FF00D1124E657FD4E108380E1FE0136
:10EB10003196ADE2B9E001900D928A95E1F72C961D
:10EB20008CAD9DADAEADBFAD2C9780932909909370
:10EB30002A09A0932B09B0932C09E0960CAD1DADCA
:10EB40002EAD3FADE09700934D0910934E092093F1
:10EB50004F0930935009E4962CAD3DAD4EAD5FADFD
:10EB6000E4972093510930935209409353095093ED
:10EB70005409E8968CAD9DADAEADBFADE8978093DE
:10EB8000550990935609A0935709B0935809609678
:10EB90000CAD1DAD2EAD3FAD60970093590910939C
:10EBA0005A0920935B0930935C096C962CAD3DADFE
:10EBB0004EAD5FAD6C9720933D0930933E09409375
:10EBC0003F0950934009A0968CAD9DADAEADBFAD51
:10EBD000A0978093410990934209A0934309B09371
:10EBE0004409A4960CAD1DAD2EAD3FADA497009386
:10EBF0004509109346092093470930934809229606
:10EC00002CAD3DAD4EAD5FAD2297209349093093B9
:10EC10004A0940934B0950934C09909127098091E0
:10EC20002809981303C084E680932409E9968FADE0
:10EC3000E9978F5F8F7080932709809127099091C2
:10EC4000260981508F70891351C4109128091BA384
:10EC5000009127090DA728E61BA10DA51013D1C40B
:10EC6000812C912CA12CB12C1DA219A619AA1EAE83
:10EC7000212C312C00E010E02DA53BA12313CEC4A4
:10EC80002114310409F07FC580916F008260809368
:10EC90006F0081E0ECC680E0EAC66090F7057090F6
:10ECA000F8050091F9051091FA05A7CA818D928D9A
:10ECB000A38DB48D0697A105B10508F018CB858DFD
:10ECC000968DA78DB0A10697A105B10508F00FCBD1
:10ECD00020E030E0A901C701B6010E9439F787FFA3
:10ECE00004C0F7FAF094F7F8F09488E60BA11CA1A1
:10ECF000809FF001819FF00D1124E657FD4EC586DF
:10ED0000D686E786F08A3ACB8091F3059091F40598
:10ED1000A091F505B091F605C816D906EA06FB06DE
:10ED200008F06CCB8C199D09AE09BF09BC01CD015F
:10ED3000660F771F881F991F27964FAD2797042FBF
:10ED400010E020E030E0A90198010E94B5F4CA016A
:10ED5000B9010E949AF00E9444F76C0D7D1D8E1D32
:10ED60009F1D0E949AF09B01AC0160E074E284E771
:10ED700099E40E94EFF54B015C0140CBA70196019D
:10ED8000C301B2010E94EFF57B018C019B01AC0134
:10ED9000632D722D89A599A90E9439F718160CF0D8
:10EDA000E0CB3E2C2F2C09A719ABDBCB0AA91BA962
:10EDB0002CA93DA9012B022B032B49F02091DF0543
:10EDC0003091E0054091E1055091E20508C02091A5
:10EDD000DB053091DC054091DD055091DE0569A52C
:10EDE0007AA58BA59CA50E94FBF00E94D9F50E94F4
:10EDF0005CF62B013C012AA93BA94CA95DA9232B58
:10EE0000242B252BC9F020E030E0A9016091D70523
:10EE10007091D8058091D9059091DA050E9496F0FD
:10EE2000882351F081E00DA51EA52FA538A9101645
:10EE30001106120613060CF080E098E62BA13CA107
:10EE4000929F8001939F100D112406571D4E1801AB
:10EE500037E4230E311CD1018C93882309F4B3C00D
:10EE600020913D0930913E0940913F095091400960
:10EE70006C966CAD7DAD8EAD9FAD6C970E9412F51A
:10EE80006DA77EA78FA798AB2091410930914209C9
:10EE90004091430950914409A0966CAD7DAD8EAD73
:10EEA0009FADA0970E9412F54B015C01209145098E
:10EEB000309146094091470950914809A4966CAD9C
:10EEC0007DAD8EAD9FADA4970E9412F56B017C01C4
:10EED0002DA53EA54FA558A9CA01B9010E94FBF076
:10EEE0006DA77EA78FA798ABA5019401C501B401BA
:10EEF0000E94FBF09B01AC016DA57EA58FA598A992
:10EF00000E9413F54B015C01A7019601C701B601F0
:10EF10000E94FBF09B01AC01C501B4010E9413F5F6
:10EF20000E947EF76B017C012091490930914A09CA
:10EF300040914B0950914C0922966CAD7DAD8EAD40
:10EF40009FAD22970E9412F5A70196010E94EFF54E
:10EF50006B017C01F801E25BFF4F60837183828368
:10EF6000938320E030E040E450E40E9439F7181623
:10EF70001CF4F101108227C02091D7053091D805EB
:10EF80004091D9055091DA05C701B6010E94FBF006
:10EF90009B01AC016091D3057091D4058091D5059A
:10EFA0009091D6050E94EFF529A53AA54BA55CA541
:10EFB0000E94FBF00E945CF66415750586059705B6
:10EFC00010F42B013C018091521290915312A091A8
:10EFD0005412B09155120EA91FA928AD39AD801752
:10EFE0009107A207B30708F4DFC02DA13EA14FA1EE
:10EFF00058A5232B242B252B41F16091561270919B
:10F000005712809158129091591264157505860512
:10F010009705D8F42EA93FA948AD59AD0E94A6F492
:10F020006B017C012DA13EA14FA158A5C301B201E6
:10F030000E94A6F4C616D706E806F90630F4C70102
:10F04000B6010E94B5F429013A0188E60BA11CA182
:10F05000809FF001819FF00D1124E657FD4EC18C79
:10F06000D28CE38CF48CC114D104E104F10431F1AD
:10F0700060915A1270915B1280915C1290915D12B6
:10F080006415750586059705C8F42EA93FA948ADF6
:10F0900059AD0E94A6F44B015C01A7019601C30182
:10F0A000B2010E94A6F486169706A806B90630F4A7
:10F0B000C501B4010E94B5F429013A0188E60BA10B
:10F0C0001CA1809FF001819FF00D1124E657FD4E99
:10F0D000C58CD68CE78CF0A0C114D104E104F104F6
:10F0E00031F160915E1270915F1280916012909187
:10F0F00061126415750586059705C8F42EA93FA908
:10F1000048AD59AD0E94A6F44B015C01A7019601E0
:10F11000C301B2010E94A6F486169706A806B90696
:10F1200030F4C501B4010E94B5F429013A0188E622
:10F130000BA11CA1809FF001819FF00D1124E657C7
:10F14000FD4EC1A0D2A0E3A0F4A0C114D104E104FB
:10F15000F10409F4C2CA6091621270916312809145
:10F16000641290916512641575058605970508F07F
:10F17000B4CA2EA93FA948AD59AD0E94A6F44B01CF
:10F180005C01A7019601C301B2010E94A6F4861694
:10F190009706A806B90608F0A0CAC501B4010E94E6
:10F1A000B5F429013A0199CA2DA13EA14FA158A554
:10F1B000232B242B252BC9F16091561270915712E5
:10F1C000809158129091591264157505860597051E
:10F1D00060F50E949AF02AAD3BAD4CAD5DAD0E944A
:10F1E000FBF06B017C016DA17EA18FA198A50E940F
:10F1F0009AF04B015C01C301B2010E949AF0A50193
:10F2000094010E94FBF09B01AC01C701B6010E9472
:10F2100096F087FF0AC0A5019401C701B6010E94BC
:10F22000EFF50E945CF62B013C0188E60BA11CA1C6
:10F23000809FF001819FF00D1124E657FD4E818CD7
:10F24000928CA38CB48C81149104A104B104B9F103
:10F2500060915A1270915B1280915C1290915D12D4
:10F26000641575058605970550F50E949AF02AAD3C
:10F270003BAD4CAD5DAD0E94FBF06B017C01C50167
:10F28000B4010E949AF04B015C01C301B2010E94DB
:10F290009AF0A50194010E94FBF09B01AC01C7010B
:10F2A000B6010E9496F087FF0AC0A5019401C7012C
:10F2B000B6010E94EFF50E945CF62B013C0188E646
:10F2C0000BA11CA1809FF001819FF00D1124E65736
:10F2D000FD4E858C968CA78CB0A081149104A1045E
:10F2E000B104B9F160915E1270915F128091601269
:10F2F00090916112641575058605970550F50E9479
:10F300009AF02AAD3BAD4CAD5DAD0E94FBF06B01B8
:10F310007C01C501B4010E949AF04B015C01C3015C
:10F32000B2010E949AF0A50194010E94FBF09B019A
:10F33000AC01C701B6010E9496F087FF0AC0A50183
:10F340009401C701B6010E94EFF50E945CF62B0103
:10F350003C0188E60BA11CA1809FF001819FF00D6C
:10F360001124E657FD4EC1A0D2A0E3A0F4A0C11421
:10F37000D104E104F10409F4B0C960916212709102
:10F38000631280916412909165126415750586056B
:10F39000970508F0A2C90E949AF02AAD3BAD4CAD8A
:10F3A0005DAD0E94FBF04B015C01C701B6010E94FC
:10F3B0009AF06B017C01C301B2010E949AF0A7018F
:10F3C00096010E94FBF09B01AC01C501B4010E94B3
:10F3D00096F087FF82C9A7019601C501B4010E947A
:10F3E000EFF50E945CF62B013C0177C9FAA9FF23D7
:10F3F00031F1A5019401632D722DC8010E94FBF02B
:10F400004B015C012DA53DA149A559A9C701B60134
:10F410000E94FBF09B01AC01C501B4010E9496F073
:10F4200087FF22C0A7019601C501B4010E94EFF534
:10F430006DA77DA389A799AB21E02AABFFC9A701DE
:10F440009601C501B4010E94EFF59B01AC016DA5C9
:10F450007DA189A599A90E94FBF06DA77DA389A72D
:10F4600099AB31E03AABEAC941E04AABE7C9A70141
:10F470009601C501B40113C0C701B6010E9496F000
:10F4800087FD09C020E030E0A901C501B4010E9458
:10F4900039F718164CF4A5019401C701B6010E9472
:10F4A00012F52B013C0176CA2401350177FA7094DC
:10F4B00077F87094A3019201C701B6010E9496F0FB
:10F4C00087FD68CA2601370165CA2DA53DA149A55A
:10F4D00059A9C701B6010E9496F087FFB4CA3DA49E
:10F4E0002DA009A519A9AFCA81E004CBF090270986
:10F4F0008FEF8F0D8F708BA3B09026098091270915
:10F50000B81609F454C0C12CD12C0BA10B1509F469
:10F510004EC0602E712C28E6269D8001279D100D7F
:10F52000112406571D4ED8018C9183FD2BC00EAFC0
:10F530001AAB0115110541F11996BC91BDA7F8014F
:10F54000F285FDA3D8011B96BC91B9A7F801F485FB
:10F55000F9ABD80115962D903D904D905C90189781
:10F56000A20191016DA57DA189A59F2F0E9496F012
:10F57000811186C1C114D10439F0F601808180FD6A
:10F580007FC102C0CEAEDAAA8BA181508F708BA34F
:10F59000809126098B1103C0CEACDAA8B6CF0BA19F
:10F5A0000B1529F081E08B0D8F70B82EF1CF1091E3
:10F5B00026091BA3C12CD12C809127090BA18017F0
:10F5C00009F443CB802E912C28E6289D8001299DAB
:10F5D000100D112406571D4ED8018C9183FD0AC0D1
:10F5E0005801C114D10439F0C6010E94A3E281116F
:10F5F00002C0C5C156018BA18F5F8F708BA36501BF
:10F60000DBCF802F81508F70289FF0011124E657A7
:10F61000FD4E908193FF24CB8DA71ECB48E6439FE0
:10F62000C0011124DC01A657BD4E1D018C9183FD44
:10F6300019C015966D917D918D919C9118970E949E
:10F640007EF7F62EE72ED82EC92E0115110509F4E6
:10F650008CC0F801808180FD0AC0D1018C9180FDB1
:10F6600006C083C0FDA0E9A4D9A8CEAC83C0F80130
:10F67000808181608083C8010E94A3E2811171C0F2
:10F68000F80161817281838194810E947EF72B0150
:10F690003C019B01AC0160E070E080E89FE30E94C8
:10F6A000EFF54B015C019B01AC016F2D7E2D8D2D83
:10F6B0009C2D0E94FBF069837A838B839C832DA110
:10F6C00039A549A95EADC501B4010E94FBF0698B63
:10F6D0007A8B8B8B9C8BAE014F5F5F4FBE016F5E51
:10F6E0007F4FC8010E94C2BCF801E95BFF4F8081D7
:10F6F0008823B9F12091D7053091D8054091D905DB
:10F700005091DA05379660817181828193810E94E0
:10F71000FBF020917D1130917E1140917F1150912D
:10F7200080110E94FBF04B015C019B01AC01C30105
:10F73000B2010E94FBF00E945CF6F801E65BFF4F0D
:10F7400071836083A50194016F2D7E2D8D2D9C2DDD
:10F750000E94FBF00E945CF6F801E45BFF4F7183AE
:10F760006083D8018C918E7F8C938F2C9E2CAD2C36
:10F77000BC2C81018BA18F5F8F708BA3FDA2E9A6AA
:10F78000D9AACEAE79CAF101808181608083C80197
:10F790000E94A3E281116FC0D10111966D917D91FC
:10F7A0008D919C9114970E947EF76B017C019B01C7
:10F7B000AC0160E070E080E89FE30E94EFF52B0170
:10F7C0003C012DEC3CEC4CE45DE30E94FBF06983D2
:10F7D0007A838B839C839401A501C301B2010E94AB
:10F7E000FBF0698B7A8B8B8B9C8BAE014F5F5F4FED
:10F7F000BE016F5E7F4FC1010E94C2BCF101E95B97
:10F80000FF4F80818823B9F12091D7053091D80529
:10F810004091D9055091DA053796608171818281D6
:10F8200093810E94FBF020917D1130917E114091D7
:10F830007F11509180110E94FBF04B015C019B01F4
:10F84000AC01C701B6010E94FBF00E945CF6F10119
:10F85000E65BFF4F718360832DEC3CEC4CE45DE391
:10F86000C501B4010E94FBF00E945CF6F101E45B6B
:10F87000FF4F71836083F10180818E7F808304CA92
:10F8800028E6269DF001279DF00D1124E657FD4E38
:10F89000808181FD43C0C114D10441F0D601159689
:10F8A000CD90DD90ED90FC90189708C08BE0C82EAD
:10F8B00087EDD82E83E2E82E8BE3F82EB8E6B69DCE
:10F8C000F001B79DF00D1124E657FD4E8189928914
:10F8D000A389B489BC01CD0190589B01AC010E9461
:10F8E00013F5F80125853685478550890E94FBF080
:10F8F0009B01AC01C701B6010E9412F5E62E872ECE
:10F90000982EA92E262F372F482F592F6DA57DA170
:10F9100089A599A90E9496F087FF04C0EDA48DA047
:10F9200099A4A9A82E2D382D492D5A2DC201B10117
:10F930000E9496F0882309F427CEF8E6F69DC001D0
:10F94000F79D900D11249C0126573D4E6901D90168
:10F950008C9181608C93C8010E94A3E2882329F0D6
:10F96000F60180818E7F80830FCE8E2D982DA92D5C
:10F97000BA2DF60185839683A783B08705CED6017D
:10F980008C9181FD52C0D60115962D913D914D91DE
:10F990005C9118972DA73EA74FA758AB1501B5E06E
:10F9A0002B0E311CF8014580568067807084A301BE
:10F9B00092016DA57EA58FA598A90E9496F087FF5C
:10F9C00034C0F60181899289A389B489BC01CD0133
:10F9D00090589B01AC010E9413F5D6011D962D9104
:10F9E0003D914D915C9150970E94FBF09B01AC01C1
:10F9F0006DA57EA58FA598A90E9412F56B017C01CB
:10FA00009B01AC01C301B2010E9439F718166CF4D6
:10FA1000D8018C9181608C93C5010E94A3E2882358
:10FA2000E1F0F80180818E7F808318E6189DF00157
:10FA3000199DF00D1124E657FD4E21853285438531
:10FA4000548565817681878190850E9496F0811129
:10FA5000D2CD0BA100932609CECDD101CD92DD925E
:10FA6000ED92FC9213970BA100932609DECFC858A4
:10FA7000DF4F0FB6F894DEBF0FBECDBFDF91CF9141
:10FA80001F910F91FF90EF90DF90CF90BF90AF90BC
:10FA90009F908F907F906F905F904F903F902F90AE
:10FAA00008958091270990912809891B8F708F30C4
:10FAB00021F480E00E942CAEF4CF809127098F5F63
:10FAC0008F70E091270998E69E9FF0011124E65778
:10FAD000FD4EDF011D929A95E9F798E090834091E1
:10FAE0004D0950914E0960914F0970915009458B15
:10FAF000568B678B708F40915109509152096091DC
:10FB0000530970915409418F528F638F748F4091C4
:10FB10005509509156096091570970915809458FC0
:10FB2000568F678F70A34091590950915A0960917F
:10FB30005B0970915C0941A352A363A374A3209154
:10FB4000270990912809291303C094E6909324096A
:10FB50008093270980916F00826080936F000895E1
:10FB60009091270980912809981306C080916E050D
:10FB700090916F05892B21F080E00E942CAEF0CF90
:10FB800008954F925F926F927F928F929F92AF9261
:10FB9000BF92CF92DF92EF92FF92CF93DF932091AB
:10FBA00038043091390440913A0450913B046091FB
:10FBB00054047091550480915604909157040E940A
:10FBC00013F5AB01BC0181E690E20E94A5CE209125
:10FBD0003C0430913D0440913E0450913F046091BB
:10FBE00058047091590480915A0490915B040E94CA
:10FBF00013F5AB01BC018DE590E20E94A5CE2091EA
:10FC0000400430914104409142045091430460917A
:10FC10005C0470915D0480915E0490915F040E9489
:10FC200013F5AB01BC0189E590E20E94A5CE40919D
:10FC3000600450916104609162047091630485E5F1
:10FC400090E20E94A5CE80916F00982F927081FF64
:10FC500005C080916F008D7F80936F00409061118F
:10FC600050906211609063117090641180906511E2
:10FC700090906611A0906711B0906811C0906911C2
:10FC8000D0906A11E0906B11F0906C11992329F0DB
:10FC900080916F00826080936F00EBE4F0E28491CA
:10FCA000EF012196882321F00E94138EFE01F7CFE9
:10FCB000C301B2010E94BA91E7E4F0E28491EF013E
:10FCC0002196882321F00E94138EFE01F7CFC501F3
:10FCD000B4010E94BA91E3E4F0E28491EF0121962D
:10FCE000882321F00E94138EFE01F7CFC701B601D1
:10FCF0000E94BA918AE0DF91CF91FF90EF90DF9060
:10FD0000CF90BF90AF909F908F907F906F905F90BB
:10FD10004F900C94138E2F923F924F925F926F925E
:10FD20007F928F929F92AF92BF92CF92DF92EF928B
:10FD3000FF920F931F93CF93DF93CDB7DEB76297F8
:10FD40000FB6F894DEBF0FBECDBF8091FF0583FDD7
:10FD5000B4C183E50E9442408C87811106C082E5D0
:10FD60000E944240882309F4A8C10E94C23F0E9419
:10FD700057F6CB010E94D1410E94C23F20E030E003
:10FD800040EA50E40E9439F7181614F40E94F6CEA7
:10FD9000E7E3F0E28491FB83EA83882371F0082E85
:10FDA000000C990B0E94059F4A815B814F5F5F4F5A
:10FDB0005B834A83FA018491F0CF8DE090E00E944A
:10FDC000059F8AE090E00E94059F81E080935202A7
:10FDD0001092401180910E11809372051A821B823D
:10FDE0001C821D82188619861A861B8619821D861A
:10FDF000FCE3FE872CE12F8736E4388B312C212C55
:10FE000040E8498B5FEB5A8B812C912C5401609117
:10FE1000660470916704072E000C880B990B0E94F2
:10FE20009CF07B018C019B01AC01632D722D8989B3
:10FE30009A890E9496F0882341F1209168043091BC
:10FE4000690440916A0450916B048C85B70181115B
:10FE50000CC0C8010E9496F0881F8827881F8983DC
:10FE60003E2C2F2C098B1A8B10C0C8010E9496F0D3
:10FE700087FF06C0EBE3F0E28491FB83EA83E8C0EE
:10FE80003E2C2F2C098B1A8B19820E9414A46B0113
:10FE90007C01DC01CB01288539854A855B85821B85
:10FEA000930BA40BB50BB7FD3BC0D701C60188511E
:10FEB0009C4FAF4FBF4F88879987AA87BB870E9407
:10FEC0003D59EFE3F0E284913F019FEF691A790A0F
:10FED000882321F00E94138EF301F5CF8114910441
:10FEE000A104B104B9F0D501C401805F984DAF4FB2
:10FEF000BF4FBC01CD016C197D098E099F0928EE09
:10FF000033E040E050E00E94B5F4CA01B9010E941C
:10FF1000BA9103C08FE30E94138E8AE00E94138E71
:10FF200080E00E942CAE0E9414A46093E9107093AC
:10FF3000EA108093EB109093EC10A0916804AE83CC
:10FF4000B0916904BF8300916A0410916B040E9410
:10FF5000702D2E813F81A801632D722D89899A8988
:10FF60000E9412F52B013C0120E030E0A9010E9423
:10FF700039F787FF04C077FA709477F8709481148A
:10FF80009104A104B10459F420E030E040E85FE3BB
:10FF9000C301B2010E9496F087FF0DC00AC020E0A5
:10FFA00030E040E450E4C301B2010E9439F7181672
:10FFB00014F446015701E981EE2391F12A813B8136
:10FFC0004C815D81211531054105510541F0D70175
:10FFD000C601821B930BA40BB50BB7FD21C02E816C
:10FFE0003F81A8016D857E858F8598890E9412F5D5
:10FFF00020E030E040EC5FE30E9496F087FD3ACFCE
:020000021000EC
:10000000D701C601805A9541AF4FBF4F8A839B836A
:10001000AC83BD839E819D87AF81AE870F87188B90
:1000200080915202882309F425CF81149104A10400
:10003000B10409F4ECCEB0E1CB1AB7E2DB0AE10877
:10004000F108C818D908EA08FB08F7FE13CFDFCE7D
:10005000882361F0082E000C990B0E94059FEA810D
:10006000FB813196FB83EA838491F2CF8DE090E0AF
:100070000E94059F8AE090E00E94059F80915202B5
:1000800081E08093401162960FB6F894DEBF0FBEF8
:10009000CDBFDF91CF911F910F91FF90EF90DF9037
:1000A000CF90BF90AF909F908F907F906F905F9018
:1000B0004F903F902F900C94459262960FB6F89413
:1000C000DEBF0FBECDBFDF91CF911F910F91FF908B
:1000D000EF90DF90CF90BF90AF909F908F907F90E8
:1000E0006F905F904F903F902F900895EF92FF9206
:1000F0000F931F93CF93DF93CDB7DEB769970FB6FA
:10010000F894DEBF0FBECDBF83E50E94424081114F
:1001100003C0EFE1F0E208C00E94923F6E34710527
:10012000C1F70E94ADCFE4C084918F010F5F1F4FD4
:10013000882321F00E94138EF801F6CFE6E1F0E269
:1001400084918F010F5F1F4F882321F00E94138E2F
:10015000F801F6CF80913C0F90913D0F0E9445E150
:10016000E9E0F0E284918F010F5F1F4F882321F0B7
:100170000E94138EF801F6CF80913E0F90913F0FB1
:100180000E9445E1EEEFFFE184918F010F5F1F4F69
:10019000882321F00E94138EF801F6CF80913C0F46
:1001A00090913D0F20913E0F30913F0F821B930B9A
:1001B00020914019215041E050E0223010F040E001
:1001C00050E0841B950B0E9445E18AE00E94138E4B
:1001D000E6EFFFE184918F010F5F1F4F882321F02D
:1001E0000E94138EF801F6CF8091400F9091410F3D
:1001F000A091420FB091430F8E8B9F8BA88FB98F28
:10020000BE016F5F7F4FCE0146960E94318DE9EEB1
:10021000FFE184918F010F5F1F4F882321F00E941F
:10022000138EF801F6CFCE0101967C018C01F80106
:1002300081918F01882319F00E94138EF8CF80914D
:10024000440F9091450FA091460FB091470F8E8BB0
:100250009F8BA88FB98FBE016F5F7F4FCE014696EF
:100260000E94318DE9EDFFE184918F010F5F1F4FF7
:10027000882321F00E94138EF801F6CFF7018191B7
:100280007F01882319F00E94138EF8CF8AE00E9424
:10029000138EE1EDFFE184918F010F5F1F4F8823E3
:1002A00021F00E94138EF801F6CFE1ECFFE184917A
:1002B0008F010F5F1F4F882321F00E94138EF801DA
:1002C000F6CF20E030E04AE754E46091480F7091A7
:1002D000490F80914A0F90914B0F0E94EFF542E039
:1002E0000E94D4918DE60E94138E8AE00E94138EA4
:1002F00069960FB6F894DEBF0FBECDBFDF91CF91E8
:100300001F910F91FF90EF9008958F929F92AF925F
:10031000BF92CF92DF92EF92FF920F931F93CF93F2
:10032000DF9300D01F92CDB7DEB7F82E662351F0D1
:1003300010920F0610920B0610920C0610920D06EA
:1003400010920E060E9414A480900B0690900C064A
:10035000A0900D06B0900E069B01AC01281939093A
:100360004A095B0957FD4CC020910F06F7FC16C0E7
:100370004F2D0F2C000C550B4C5F5F4FE22F022EC0
:10038000000CFF0B4E175F07DCF12F153CF044EF1C
:10039000C42EDD24D394E12CF12C06C038EEC32EFC
:1003A00033E0D32EE12CF12CDC01CB018C0D9D1D13
:1003B000AE1DBF1D80930B0690930C06A0930D06F7
:1003C000B0930E06022F017010E024E2209FC001BE
:1003D000219F900D901B112480599C4F9C838B83EF
:1003E00082E390E09A838983BE016D5F7F4FCE01E7
:1003F00001960E947AB880910F068F5F80930F0656
:100400000F900F900F900F90DF91CF911F910F9150
:10041000FF90EF90DF90CF90BF90AF909F908F9024
:100420000895AF92BF92CF92DF92EF920F931F93F6
:10043000CF93DF93CDB7DEB760970FB6F894DEBFEA
:100440000FBECDBF5C018B010E944E40E0900E11AB
:100450008DE8C82E81E1D82E84E0E89EF0011124B9
:10046000E25EFD4F2081318142815381F50160813F
:100470007181828193810E94EFF5F6012485358593
:10048000468557850E9413F5F60164877587868730
:1004900097871D861E861F86188A80819181A2817A
:1004A000B38189839A83AB83BC8384819581A68140
:1004B000B7818D839E83AF83B88780859185A28520
:1004C000B38589879A87AB87BC87AE01475F5F4F4B
:1004D000BE016B5F7F4FCE0101960E943DC1CE01F0
:1004E0000D966C0129E931E1AE01475F5F4FBE0116
:1004F0006B5F7F4F0C970E948A6D0E94914130DBA9
:1005000060960FB6F894DEBF0FBECDBFDF91CF91DE
:100510001F910F91EF90DF90CF90BF90AF90089513
:100520009F92AF92BF92CF92DF92EF92FF920F9382
:100530001F93CF93DF9387E5A82E82E0B82E0DE8B6
:1005400011E1C4E5D4E098E3C92E94E0D92E25E466
:10055000E22E24E0F22E912CF50181915F010E94A0
:10056000F93F882309F10E94C23FF7012081211140
:1005700004C020914904222339F0288139814A811D
:100580005B810E9413F50AC0F3E09F1639F0F60173
:1005900020813181428153810E9412F5F8016083EC
:1005A00071838283938309C088819981AA81BB81E9
:1005B000F80180839183A283B38393940C5F1F4FD0
:1005C0002496F4E0CF0ED11C2FEFE21AF20A84E059
:1005D0009812C2CF86E40E9442408823C9F00E944C
:1005E000C23F20E030E0A9010E9439F7181684F4D8
:1005F0000E94C23F20E030E040E752E40E94EFF565
:1006000060934202709343028093440290934502A8
:100610008091FF0583FD28C080913B0F882321F145
:100620002091600430916104409162045091630410
:100630006091991170919A1180919B1190919C11E8
:100640000E9412F52091480F3091490F40914A0FB6
:1006500050914B0F0E9413F56093480F7093490F10
:1006600080934A0F90934B0FDF91CF911F910F9181
:10067000FF90EF90DF90CF90BF90AF909F90089544
:100680002F923F924F925F926F927F929F92AF9282
:10069000BF92CF92DF92EF92FF920F931F93CF936F
:1006A000DF93CDB7DEB764970FB6F894DEBF0FBE09
:1006B000CDBF1A012B01922EF32EC82ED12CF6019C
:1006C000EF5EF94DE491AA24A3941E160CF4A12C1C
:1006D000BB24B39420E030E0A901C201B1010E9423
:1006E00039F718160CF0B12CCC0CDD1CCC0CDD1C31
:1006F000C6018C5A9B4F3C01FC0110821182128270
:1007000013820E94DA8CF30120823182428253826A
:10071000E0900E1120E030E0A901B801892D9F2D55
:100720000E9496F081110AC0F601EC53FA4D8591B2
:100730009591A591B4918C019A2EFB2EC801A92DFB
:10074000BF2D898B9A8BAB8BBC8B80915C04909175
:100750005D04A0915E04B0915F04409158045091F3
:10076000590460915A0470915B04009154041091F3
:100770005504209156043091570409831A832B8322
:100780003C834D835E836F83788789879A87AB87A5
:10079000BC871D861E861F86188AAE01475F5F4F85
:1007A000BE016B5F7F4FCE0101960E943DC1CE011D
:1007B0000D966C018E010F5E1F4F20E634E0AE01F6
:1007C000475F5F4FBE016B5F7F4F0C970E948A6D42
:1007D000C7D9AB1459F080915E0F882319F010929D
:1007E0005E0F04C085E99FE10E94E5AD64960FB6F7
:1007F000F894DEBF0FBECDBFDF91CF911F910F9157
:10080000FF90EF90DF90CF90BF90AF909F907F9040
:100810006F905F904F903F902F900895EF92FF92CE
:100820001F93CF93DF9385EAE82E81E1F82E15E040
:10083000C0E0D0E020E030E0A901F701EC0FFD1F9F
:1008400060817181828193810E9496F081110CC038
:100850002496C431D10571F7115084E1E80EF11CE2
:100860001111E6CF80E001C081E0DF91CF911F91AF
:10087000FF90EF900895CF9390915B119817C1F07E
:10088000C82F6ED9C11112C04CE554E068E574E080
:1008900084E594E00E943DC180E080935B11882351
:1008A00039F084E594E0CF910C94BDCFB7DFF5CF5C
:1008B000CF910895CF92DF92EF920F931F93CF9332
:1008C000DF93CDB7DEB760970FB6F894DEBF0FBEEB
:1008D000CDBFE0900E11E4E5F4E080859185A2851E
:1008E000B3854481558166817781008111812281A0
:1008F000338109831A832B833C834D835E836F830B
:10090000788789879A87AB87BC871D861E861F8656
:10091000188AAE01475F5F4FBE016B5F7F4FCE010C
:1009200001960E943DC1CE010D966C0102E412E0D9
:1009300020E634E0AE01475F5F4FBE016B5F7F4F43
:100940000C970E948A6D60960FB6F894DEBF0FBEBA
:10095000CDBFDF91CF911F910F91EF90DF90CF909E
:1009600008952F923F924F925F926F927F928F9253
:100970009F92AF92BF92CF92DF92EF92FF920F932E
:100980001F93CF93DF93CDB7DEB72A970FB6F894B6
:10099000DEBF0FBECDBF2B013C012D833E834F83B5
:1009A000588747015801DA86C986809142029091A2
:1009B0004302A0914402B091450289839A83AB839C
:1009C000BC83D6011C9111960C91119712963C9004
:1009D000129713962C9020E030E0A901612F702F20
:1009E000832D922D0E9496F081110AC0ECECF5E265
:1009F00085919591A591B491182F092F3A2E2B2E00
:100A0000A501940160915C0470915D0480915E0485
:100A100090915F040E9496F087FF15C0812F902F60
:100A2000A32DB22D8093420290934302A0934402DF
:100A3000B093450280925C0490925D04A0925E04A3
:100A4000B0925F0437DFE985FA85C080D180E2800B
:100A5000F38020E030E0A901C701B6010E9496F0C2
:100A6000811107C085E5C82EDC2C85E0E82E83E4E3
:100A7000F82EC0924202D0924302E0924402F092D9
:100A8000450240925404509255046092560470926C
:100A900057048D819E81AF81B885809358049093CF
:100AA0005904A0935A04B0935B0404DF20915C04C2
:100AB00030915D0440915E0450915F04C501B40122
:100AC0000E9496F087FF15C0812F902FA32DB22D85
:100AD0008093420290934302A0934402B093450254
:100AE00080925C0490925D04A0925E04B0925F04D8
:100AF000E1DE36D889819A81AB81BC818093420244
:100B000090934302A0934402B09345022A960FB6F5
:100B1000F894DEBF0FBECDBFDF91CF911F910F9133
:100B2000FF90EF90DF90CF90BF90AF909F908F900D
:100B30007F906F905F904F903F902F900895CF924D
:100B4000DF92EF92FF920F931F936B01FC01E08005
:100B5000F18002811381E4E5F4E02481358146814E
:100B600057816081718182819381FBDE1F910F919A
:100B7000FF90EF90DF90CF9008958F929F92AF9269
:100B8000BF92EF92FF920F931F93CF93DF9300D00A
:100B90001F92CDB7DEB7182F80915304877087302E
:100BA00069F48FE40E944240882319F00E94B33F09
:100BB00003C08FE40E94F93F8111BCC00E94B07D48
:100BC00080E059DE8091420290914302A09144025C
:100BD000B09145028093070690930806A0930906FA
:100BE000B0930A0680910202909103029093060648
:100BF0008093050684E690E09093030280930202BE
:100C000081E080934D0F11111BC088E50E94F93FD0
:100C1000F82E89E50E94F93F082F8AE50E94F93FE6
:100C2000E82EF11006C0011109C0811107C0F02E95
:100C30000CC0002319F0F02E182F08C010E006C0D9
:100C4000FF24F39401E0EE24E39411E00E944E406F
:100C500082E50E944240882361F00E94C23F4B011E
:100C60005C0120E030E0A9010E9496F0882369F140
:100C700006C0812C912C80EAA82E80E4B82E111198
:100C800004C0F11002C0002389F180929511909266
:100C90009611A0929711B0929811A50194016091BC
:100CA0005C0470915D0480915E0490915F040E94E9
:100CB00096F087FF0AC019821A821B821C82BE012D
:100CC0006F5F7F4F85E991E13ADF111105C0F110A7
:100CD00003C0011106C00AC080E00E947CAC112351
:100CE000C1F381E00E947CAC111102C0EE2019F02A
:100CF00082E00E947CAC5ED680914C0F80934D0FB9
:100D00008091070690910806A0910906B0910A0605
:100D10008093420290934302A0934402B093450211
:100D2000809105069091060690930302809302023B
:100D30000E94C17D0F900F900F900F90DF91CF9187
:100D40001F910F91FF90EF90BF90AF909F908F9069
:100D500008952F923F924F925F926F927F928F925F
:100D60009F92AF92BF92CF92DF92EF92FF920F933A
:100D70001F93CF93DF93CDB7DEB762970FB6F8948A
:100D8000DEBF0FBECDBF8DE690E054D78111DCC130
:100D90008091FF0583FDD8C183E50E9442408C8786
:100DA000811106C082E50E94424089838823B1F008
:100DB0000E94C23F0E9457F6CB010E948F5A0E94A8
:100DC000C23F20E030E04AEA52E40E9496F0181652
:100DD0000CF4B5C10E943DCF21E02983E7E2F0E2A7
:100DE00084918F01882351F0082E000C990B0E94EA
:100DF000059F0F5F1F4FF8018491F4CF8DE090E0C5
:100E00000E94059F8AE090E00E94059F0E94EFD01B
:100E1000F981FF2309F498C181E080935202109276
:100E200040111A821B821C821D82188619861A861E
:100E30001B8619821D862CE32E873CE13F8746E402
:100E4000488B312C212C50E8598B8FEB8A8B812CCD
:100E5000912C540160916C0470916D04072E000C6C
:100E6000880B990B0E949CF07B018C019B01AC01CB
:100E7000632D722D89899A890E9496F0882359F1F1
:100E800020916E0430916F04409170045091710470
:100E90009C85B701802F91110CC0912F0E9496F074
:100EA000881F8827881F89833E2C2F2C098B1A8B3B
:100EB00012C0912F0E9496F087FF08C080915202C5
:100EC000EFE2F0E28491FB83EA83E5C03E2C2F2C15
:100ED000098B1A8B19820E9414A46B017C01DC011E
:100EE000CB01288539854A855B85821B930BA40B32
:100EF000B50BB7FD38C0D701C60188519C4FAF4F25
:100F0000BF4F88879987AA87BB870E943D59E3E333
:100F1000F0E284913F019FEF691A790A882319F062
:100F200082D6F301F6CF81149104A104B104B9F083
:100F3000D501C401805F984DAF4FBF4FBC01CD01BB
:100F40006C197D098E099F0928EE33E040E050E0DE
:100F50000E94B5F4CA01B9010E94BA9102C08FE3A0
:100F600062D68AE060D680E00E942CAE0E9414A473
:100F70006093E9107093EA108093EB109093EC105B
:100F8000A0916E04AE83B0916F04BF830091700492
:100F9000109171040E94702D2E813F81A801632D54
:100FA000722D89899A890E9412F52B013C0120E05B
:100FB00030E0A9010E9439F787FF04C077FA7094E6
:100FC00077F8709481149104A104B10459F420E0DD
:100FD00030E040E85FE3C301B2010E9496F087FF72
:100FE0000DC00AC020E030E040E450E4C301B2018B
:100FF0000E9439F7181614F446015701E981EE23CF
:1010000091F12A813B814C815D812115310541059A
:10101000510541F0D701C601821B930BA40BB50B00
:10102000B7FD21C02E813F81A8016D857E858F850A
:1010300098890E9412F520E030E040EC5FE30E94C6
:1010400096F087FD3BCFD701C601805A9541AF4F3F
:10105000BF4F8A839B83AC83BD839E819D87AF8175
:10106000AE870F87188B80915202882309F426CF10
:1010700081149104A104B10409F4ECCEB0E1CB1ABF
:10108000B7E2DB0AE108F108C818D908EA08FB084A
:10109000F7FE14CFDFCE882361F0082E000C990BE9
:1010A0000E94059FEA81FB813196FB83EA8384914C
:1010B000F2CF8DE090E00E94059F8AE090E00E94D0
:1010C000059F8091280C8130E9F4EBE2F0E28491F5
:1010D000FB83EA83882371F0082E000C990B0E9491
:1010E000059F4A815B814F5F5F4F5B834A83FA01B3
:1010F0008491F0CF8DE090E00E94059F8AE090E01F
:101100000E94059F81E08093401162960FB6F8948B
:10111000DEBF0FBECDBFDF91CF911F910F91FF902A
:10112000EF90DF90CF90BF90AF909F908F907F9087
:101130006F905F904F903F902F900C9445920E943B
:10114000F6CE31E039834ACE62960FB6F894DEBF10
:101150000FBECDBFDF91CF911F910F91FF90EF9008
:10116000DF90CF90BF90AF909F908F907F906F90C7
:101170005F904F903F902F90089590919E11E92F8E
:10118000F0E0E65AF04F80839F5F943018F490931C
:101190009E1102C010929E1180919F118F5F8093CB
:1011A0009F110895CF93FC0120812B33A1F0209152
:1011B0009F11243080F4C62FBC0180919E11F0E66F
:1011C0008F9FC0011124815A904F0E9477F88C2F75
:1011D000D4DF81E001C080E0CF9108952F923F924B
:1011E0004F925F926F927F928F929F92AF92BF9237
:1011F000CF92DF92EF92FF920F931F93CF93DF93E3
:1012000000D000D0CDB7DEB79A8389830E9414A4A2
:10121000E981FA81C680D780E084F184C114D104C9
:10122000E104F10409F0ACC22485222309F469C366
:1012300032852150248721E0230F228745852413FE
:1012400001C01286E981FA8124E0329FE00DF11D90
:101250001124C684D784E088F188E981FA81C282AA
:10126000D382E482F582DC01CB018C0D9D1DA11D92
:10127000B11D86839783A087B18784819581892B4F
:1012800009F43FC3FFB7FD83F894E981FA81228016
:1012900033802101612C712C0481158180911D0204
:1012A0008F3121F08F3F09F068C205C0E0E2FCE118
:1012B00024912E83DAC08FE180931D02E0E2FCE1ED
:1012C00084918E838F3F09F458C2823009F469C03B
:1012D00030F5882309F44CC0813009F0C6C0109263
:1012E000800010928100809181008860809381004D
:1012F00080918100816080938100E3EAF6E2E491CD
:10130000F0E0EE0FFF1FE05BF94D85919491E9EE5F
:10131000F6E2E491E0939706E1E0EE8330C19E812E
:10132000943009F482C008F460C0953009F09DC083
:1013300010922001109221018091210188608093F8
:10134000210180912101816080932101E3EAF6E28D
:10135000E491F0E0EE0FFF1FE05BF94D8591949171
:10136000E9EEF6E2E491E093940695E09E8307C1EE
:1013700014BC15BC84B5826084BD85B5816085BD13
:10138000E3EAF6E2E491F0E0EE0FFF1FE05BF94DD7
:1013900085919491E9EEF6E2E491E09398061E823D
:1013A000ABC21092B0001092B1008091B000826088
:1013B0008093B0008091B10081608093B100E3EA36
:1013C000F6E2E491F0E0EE0FFF1FE05BF94D85914E
:1013D00094919093740580937305E9EEF6E2E4919D
:1013E000E0937505F2E0FE8387C2109290001092A0
:1013F000910080919100886080939100809191008C
:10140000816080939100E3EAF6E2E491F0E0EE0F70
:10141000FF1FE05BF94D85919491E9EEF6E2E491CE
:10142000E093960623E02E83AAC01092A0001092AB
:10143000A1008091A10088608093A1008091A1000B
:1014400081608093A100E3EAF6E2E491F0E0EE0F20
:10145000FF1FE05BF94D85919491E9EEF6E2E4918E
:10146000E093950684E08E838AC0EE81E7FD85C116
:1014700061E08FE10E9421B98E818D7F09F083C0E8
:101480004801A12CB12C60E072E18AE790E0A5014F
:1014900094010E94D7F429833A834B835C836901CA
:1014A0007A01F1E0CF1AD108E108F1082FEFC21656
:1014B000D104E104F10409F008F44EC060E472E4E0
:1014C0008FE090E0A50194010E94D7F469017A01B0
:1014D00081E0C81AD108E108F1089E81923009F52F
:1014E000EFEFCE16D104E104F10409F008F4CBC10A
:1014F00060E970ED83E090E0A50194010E94D7F4CB
:1015000069017A01F1E0CF1AD108E108F1082FEF63
:10151000C216D104E104F10411F008F041C183E0E6
:1015200027C08FEFC816D104E104F104B9F0B0F080
:1015300068E478EE81E090E0A50194010E94D7F480
:1015400069017A0191E0C91AD108E108F108EE8138
:10155000EE2309F49AC163C181E001C082E09E815B
:10156000911106C095B5987F892B85BD7AC085E01D
:101570009091B100987F892B8093B10072C061E097
:101580008FE10E9421B94801A12CB12C60E072E1E9
:101590008AE790E0A50194010E94D7F469017A01DD
:1015A000E1E0CE1AD108E108F108C114D104F1E05C
:1015B000EF06F10488F068E478EE81E090E0A501A0
:1015C00094010E94D7F469017A0181E0C81AD10818
:1015D000E108F10883E001C081E09E81913071F45F
:1015E00090918100987F892B80938100452846281F
:1015F0004728D9F52FEF3FEFA90168C0EE81E3300E
:1016000071F490919100987F892B809391004528E7
:101610004628472851F52FEF3FEFA90179C0FE81F9
:10162000F43071F49091A100987F892B8093A100F0
:10163000452846284728C9F42FEF3FEFA9017AC073
:101640002E81253071F490912101987F892B809310
:10165000210145284628472841F42FEF3FEFA901F3
:101660007BC045284628472869F0D801AA0FBB1F30
:1016700091010E9403F528EE33E040E050E00E9423
:10168000B5F403C02FEF3FEFA9018E81823081F1C5
:101690002CF4882361F08130C9F06FC09E819430B2
:1016A00009F448C0ACF1953009F456C066C0C7BC17
:1016B0002093A9063093AA064093AB065093AC063C
:1016C00080916E00826080936E0057C0D092890036
:1016D000C09288002093A5063093A6064093A706E3
:1016E0005093A80680916F00826080936F0045C080
:1016F000C092B30020937605309377054093780528
:10170000509379058091700082608093700035C09D
:10171000D0929900C09298002093A1063093A2061F
:101720004093A3065093A406809171008260809339
:10173000710023C0D092A900C092A80020939D06FA
:1017400030939E0640939F065093A00680917200AE
:1017500082608093720011C0D0922901C09228014A
:101760002093990630939A0640939B0650939C06CB
:1017700080917300826080937300ED81EFBFC1C0E0
:10178000DC01CB018C199D09AE09BF09B7FDB9C0B9
:101790004698E981FA811682178210861186B1C0B7
:1017A00068E478EE81E090E0A50194010E94D7F40E
:1017B00069017A01F1E0CF1AD108E108F1082FEFB1
:1017C000C216D104E104F10441F138F164E274EF8E
:1017D00080E090E0A50194010E94D7F469017A01AC
:1017E000F1E0CF1AD108E108F1082FEFC216D104B9
:1017F000E104F10409F008F4BACE62E17AE780E08E
:1018000090E0A50194010E94D7F469017A0181E07A
:10181000C81AD108E108F10819C084E0A9CE2FEF59
:10182000C216D104E104F10409F008F463C062E1D6
:101830007AE780E090E0A50194010E94D7F4690165
:101840007A01F1E0CF1AD108E108F1082FEFC216B2
:10185000D104E104F104A9F0A0F089819A81AB815F
:10186000BC812AE0B595A795979587952A95D1F7DC
:101870006C017D01F1E0CF1AD108E108F10887E0A1
:1018800077CE86E075CE82E073CEEFEFCE16D10430
:10189000E104F10469F160F162E17AE780E090E04F
:1018A000A50194010E94D7F469017A0181E0C81A68
:1018B000D108E108F1089FEFC916D104E104F10451
:1018C000A9F0A0F089819A81AB81BC813AE0B595FD
:1018D000A795979587953A95D1F76C017D01E1E041
:1018E000CE1AD108E108F10885E03CCE84E03ACE7A
:1018F00083E038CE84E033CE61E08FE10E9421B9ED
:10190000BFCD26960FB6F894DEBF0FBECDBFDF91D8
:10191000CF911F910F91FF90EF90DF90CF90BF90EC
:10192000AF909F908F907F906F905F904F903F907F
:101930002F9008950F931F93CF93DF9394E0899F87
:10194000E00111248E01085C1B4FFE01E25BF04FA9
:10195000DE01AA50BF4E2D913D914D915C91608169
:101960007181828193810E9413F5F80160837183F4
:1019700082839383FE01E75FFD4D85919591A5914B
:10198000B491FE01EE5FFE4E80839183A283B38308
:10199000FE01EB5EFD4D85919591A591B491C35DDE
:1019A000DD4F88839983AA83BB83DF91CF911F91F9
:1019B0000F9108950F931F93CF93DF93CDB7DEB7A9
:1019C0002C970FB6F894DEBF0FBECDBFE4E5F4E070
:1019D00080859185A285B385448155816681778113
:1019E000008111812281338109831A832B833C83F7
:1019F0004D835E836F83788789879A87AB87BC879F
:101A0000AE01475F5F4FBE016B5F7F4FCE01019616
:101A10000E943DC120E634E0AE01475F5F4FBE014A
:101A20006B5F7F4FCE0101960E947AD12C960FB644
:101A3000F894DEBF0FBECDBFDF91CF911F910F9104
:101A400008958091920690919306009731F04AE0B4
:101A500050E060E070E00C9415EF60E070E0CB01C6
:101A600008952F923F924F925F926F927F928F9242
:101A70009F92AF92BF92CF92DF92EF92FF920F931D
:101A80001F93CF93DF93EB01FC0180809180A280B4
:101A9000B380C501B40120E831E541E050E00E9487
:101AA000B5F4C9016DE671E00E94E8F76B017C01B5
:101AB000C501B40120E13EE040E050E00E94B5F4F1
:101AC000CA01B90128E130E040E050E00E94B5F4DD
:101AD000362E272E062F172F8CE3482E512C612CE3
:101AE000712CC501B401A30192010E94B5F4B62E78
:101AF000A72ECA01B901A30192010E94B5F4CB013E
:101B0000C114D104D9F0AF92BF927F936F932F92FB
:101B10003F92FF92EF92DF92CF928CE890E29F93F8
:101B20008F93DF93CF930E9468F08DB79EB70E9688
:101B30000FB6F8949EBF0FBE8DBF5CC0E114F104D8
:101B4000C9F0AF92BF927F936F932F923F92FF9213
:101B5000EF928CE790E29F938F93DF93CF930E9455
:101B600068F0EDB7FEB73C960FB6F894FEBF0FBE17
:101B7000EDBF40C0012BB9F0AF92BF927F936F933E
:101B80002F923F9280E790E29F938F93DF93CF93C2
:101B90000E9468F08DB79EB70A960FB6F8949EBF64
:101BA0000FBE8DBF27C0892BA9F0AF92BF927F9344
:101BB0006F9388E690E29F938F93DF93CF930E9479
:101BC00068F0EDB7FEB738960FB6F894FEBF0FBEBB
:101BD000EDBF10C0AF92BF9284E690E29F938F93C7
:101BE000DF93CF930E9468F00F900F900F900F90AB
:101BF0000F900F90DF91CF911F910F91FF90EF9079
:101C0000DF90CF90BF90AF909F908F907F906F901C
